:020000040800F2
:1000000000040020A51F0008F71F0008F71F0008C4
:10001000F71F0008F71F0008F71F00080000000086
:10002000000000000000000000000000F71F0008B2
:10003000F71F000800000000F71F0008F5BC0108CA
:100040008DBE01088FBE010891BE010895BE010852
:10005000B5BE0108B7BE0108B9BE0108DDBE010882
:1000600001BF010825BF010849BF01086DBF010894
:100070006FBF010871BF010873BF010875BF010898
:1000800077BF010879BF01087BBF0108F71F00088F
:10009000F71F0008F71F0008F71F00087DBF0108C1
:1000A000C9BF0108CBBF0108CDBF0108CFBF010800
:1000B000D1BF0108D5BF010801C0010861C0010816
:1000C00063C0010865C0010867C0010869C0010874
:1000D0006DC00108D5C1010805C1010899C2010818
:1000E0005DC3010821C4010823C4010825C4010817
:1000F00029C4010885C4010887C4010889C401080E
:100100008BC401088DC401088FC4010891C4010883
:1001100095C4010869C501086BC501086DC50108D2
:100120006FC5010871C5010873C5010875C50108CF
:1001300000000000000000000000000000000000BF
:1001400000000000000000000000000000000000AF
:10015000000000000000000000000000000000009F
:10016000000000000000000000000000000000008F
:10017000000000000000000000000000000000007F
:10018000000000000000000000000000000000006F
:10019000000000000000000000000000000000005F
:1001A000000000000000000000000000000000004F
:1001B000000000000000000000000000000000003F
:1001C000000000000000000000000000000000002F
:1001D000000000000000000000000000000000001F
:0401E0005FF8E0F1F3
:1001E800032A70B404460D4626D941EA000313F0E9
:1001F800030F13D020782B78984208BF294606D0E1
:100208001EE014F8010F11F8013F984218D1012A95
:1002180002F1FF32F5D1002070BC70470B4604464E
:1002280051F8045B50F8046BAE4204D1043A04461A
:10023800032A0B46F2D81D461046002ADAD1EBE70E
:10024800C01AE9E7032A2DE9F00109D82AB10023E9
:10025800CC5CC45401339342FAD1BDE8F001704735
:100268000B468218014603E02478013301F8014B5C
:1002780011F0030F1C46F7D113F003055DD06E4251
:10028800C5F1040CED009B594FEACC0C08E004348E
:10029800A7593B4607FA0CF748EA070741F8047BD9
:1002A800571A23FA05F8032FF1DC03E014F8013B91
:1002B80001F8013B8A42F9D8CFE753F8404C41F89E
:1002C800404C53F83C4C41F83C4C53F8384C41F8FE
:1002D800384C53F8344C41F8344C53F8304C41F80E
:1002E800304C53F82C4C41F82C4C53F8284C41F81E
:1002F800284C53F8244C41F8244C53F8204C41F82E
:10030800204C53F81C4C41F81C4C53F8184C41F83D
:10031800184C53F8144C41F8144C53F8104C41F84D
:10032800104C53F80C4C41F80C4C53F8084C41F85D
:10033800084C53F8044C41F8044C561A1D460C4618
:10034800403340313F2EB8DC2B460FE053F8101CE9
:1003580044F8101C53F80C1C44F80C1C53F8081CE7
:1003680044F8081C53F8041C44F8041C161B2146C6
:100378001D46103410330F2EE8DC2B4602E02468AB
:1003880041F8044B551A1C46032D03F10403F6DC0F
:1003980090E700BF032AC9B270B408D82AB103464F
:1003A800121803F8011B9342FBD170BC70478218E6
:1003B800044601E004F8011B14F0030FFAD14FF0D2
:1003C800013303FB01F31FE044F8403C44F83C3C94
:1003D80044F8383C44F8343C44F8303C44F82C3C6D
:1003E80044F8283C44F8243C44F8203C44F81C3C9D
:1003F80044F8183C44F8143C44F8103C44F80C3CCD
:1004080044F8083C44F8043C161B254640343F2E6B
:10041800DADC2C4607E044F8103C44F80C3C44F87D
:10042800083C44F8043C161B254610340F2EF2DC19
:1004380001E045F8043B541B032CFADC01E005F805
:10044800011B9542FBD3B0E710F0030F38B5044603
:1004580012D10368A3F1013222EA030313F0803FAB
:100468000AD1031D184653F8042BA2F1013525EAD9
:10047800020212F0803FF5D003782BB1431C1846D6
:1004880013F8012B002AFAD100F076F9204638BD7E
:10049800C9B2F0B4002950D010F0030F10D003787F
:1004A800002B79D0994246D0431C05E013F8012B64
:1004B800002A3FD091423ED013F0030F1846F5D1E1
:1004C800036841EA01270646A3F1013247EA0747D4
:1004D80022EA030212F0803F1DD187EA0303A3F149
:1004E800013222EA030313F0803F14D1043002E002
:1004F80012F0803F0FD1064650F8043BA3F10135B6
:1005080087EA030225EA0303A2F1013413F0803FCE
:1005180024EA0202ECD033783046002B3CD09942D2
:1005280009D0731C01E0914205D0184613F8012B3D
:10053800002AF8D11046F0BC704710F0030F0CD019
:100548000378002BF7D0431C03E013F8012B002A93
:10055800F1D013F0030F1846F7D102680346A2F151
:10056800013121EA020212F0803F0AD10430034629
:1005780050F8042BA2F1013121EA020212F0803F67
:10058800F5D01A781846002AD5D00133184613F842
:10059800012B002AFAD1CEE71846CCE780EA0102FF
:1005A80012F0030F3AD110F0030220F0030021F0FB
:1005B800030150F804CB08BF51F8043B0DD082F07A
:1005C80003024FEAC2026FF07F4323FA02F251F8A6
:1005D800043B4CEA020C43EA020300BFACF10132CF
:1005E8009C4501BF22EA0C0212F0803F50F804CB70
:1005F80051F8043BF2D04FEA0C604FEA1C2C01285A
:1006080028BFB0EB036F08BF1B0AF4D003F0FF0349
:100618004FEA1060A0EB0300704700BF10F0030F13
:100628000AD010F8012B11F8013B012A28BF9A4281
:10063800F4D0A2EB030070474DF8045D4DF8044D6B
:100648004FF0010242EA022242EA024201F0030CA0
:1006580021F0030150F8044B51F8045BBCF1020F80
:1006680026D04BD824F07F4CBCEB152FA4EB02030B
:1006780023EA04030DD113EAC21308BF51F8045B3F
:100688000AD18CEA040CBCEB056F0CD150F8044B72
:10069800E8E74FEA15255CE033F07F4352D10D7847
:1006A8004FEA146C55E04FEA146C05F0FF0550E072
:1006B8004FEA044CA4EB02034FEA1C4C23EA040360
:1006C800BCEB154F17D113EAC21308BF51F8045BEE
:1006D80007D18CEA040CBCEB054F08D150F8044B49
:1006E800E6E71B042ED10D884FEA144C31E04FEA9F
:1006F80005454FEA144C4FEA15452AE004F0FF0C73
:10070800BCEB156FA4EB020323EA04030DD113EA33
:10071800C21308BF51F8045B0AD18CEA040CBCEB85
:10072800052F0AD150F8044BE8E74FEA156510E0A9
:1007380014F0FF0F06D051F8045B4FEA142C25F093
:100748007F4506E04FF000005DF8044B5DF8045B60
:1007580070470CF0FF0205F0FF00012828BF904207
:1007680004BF4FEA1C2C2D0AF3D0A2EB00005DF861
:10077800044B5DF8045B704780EA0102844612F07E
:10078800030F4FD111F0030F32D14DF8044D11F082
:10079800040F51F8043B0BD0A3F101329A4312F035
:1007A800803F04BF4CF8043B51F8043B16D100BF0E
:1007B80051F8044BA3F101329A4312F0803FA4F19F
:1007C80001320BD14CF8043BA24312F0803F04BF26
:1007D80051F8043B4CF8044BEAD023460CF8013B93
:1007E80013F0FF0F4FEA3323F8D15DF8044B70473D
:1007F80011F0010F06D011F8012B0CF8012B002A7B
:1008080008BF704711F0020FBFD031F8022B12F069
:10081800FF0F16BF2CF8022B8CF8002012F47F4F24
:10082800B3D1704711F8012B0CF8012B002AF9D12C
:10083800704700BF20F0030110F00300C0F1000072
:1008480051F8043B00F1040C4FEACC0C6FF00002A5
:100858001CBF22FA0CF213434FF0010C4CEA0C2C8B
:100868004CEA0C4CA3EB0C0222EA030212EACC126B
:1008780004BF51F8043B0430F4D013F0FF0F1FBF3E
:10088800013013F47F4F013013F47F0F18BF01308C
:10089800704700BFF0B4002A46D041EA000313F0C5
:1008A80003032CD1032A07460E4643D904680D6872
:1008B800AC423FD1043A37D0A4F1013525EA04040B
:1008C80014F0803F18BF18462CD1041D0D1D0EE0F2
:1008D80054F8043B55F8041BA3F101308B4220EA7D
:1008E800030027D1043A1FD010F0803F1ED1032AFD
:1008F80027462E46ECD820462946002A1DD00478E3
:10090800013A0D78AC420CD172B18CB1002302E0EF
:1009180093420BD064B1013310F8014FCD5CAC4267
:10092800F6D0601BF0BC70471046FBE70020F9E7E3
:100938002046F7E738463146E1E724782D78F0E796
:1009480041EA000313F0030F0B4670B414BF0024F0
:100958000124032A94BF002404F001040546D4B9F5
:10096800BAB10E782B46013A03F8016B56B1AC1CAC
:100978007AB111F8015F2346013A04F8015C0134A9
:10098800002DF5D12AB19A18002103F8011B9342D2
:10099800FBD170BC7047194653F8044BA4F10136DB
:1009A80026EA040616F0803FDAD1043A45F8044BEB
:1009B800032A1946EFD8D3E701232DE9F0071D468E
:1009C80000264FF0FF37AC1900EB070C8C420DD214
:1009D8001CF805C010F80480E0452ED201252646F3
:1009E800E31BAC198C4200EB070CF1D34FF0010963
:1009F80000264D464FF0FF3C1360AC1900EB0C0885
:100A0800A1420ED918F8058010F804A0C2451AD9D9
:100A180001252646CCEB0409AC19A14200EB0C08D1
:100A2800F0D80CF101000137B8423CBF994638466E
:100A3800C2F80090BDE8F00770470BD00123374695
:100A48001D46F618BFE709D04FF00109B4464D46D8
:100A58004E44D2E79D4205D00135B4E74D4505D057
:100A68000135CAE72B4626460125ACE7A9462646A6
:100A78000125C2E72DE9F04FADF5826D81B014462E
:100A8800074610460DF580628B460C3219461D4606
:100A9800FFF792FF03AE04A901F57E72331F0090A1
:100AA80043F8045F9342FBD14DB1681E0023E25C1A
:100AB800C11A013303AEAB4246F82210F7D1DDF874
:100AC8000C142046009A6118FFF78AFB002877D19A
:100AD8000099814605F1FF380646C1F101020192ED
:100AE8005A46AB4609EB0B0501F1FF3AB81800214D
:100AF800AA1A00F0E5F900284FD1002D00F0C080B7
:100B08007B1903A913F8013C51F82330002B4CD171
:100B1800009B9E4228BF334698450FD903EB090135
:100B2800E05C7A18795C884205D038E012F8011F39
:100B3800E05C884233D101339845F7D8009A964251
:100B480080F0A48007EB090214F80A10534612F843
:100B58000A20914204BF0AEB0901791807D095E0F1
:100B680014F802C011F8010D844503D113465A1E2A
:100B7800B342F5D101369E4200F28D80DDF80C6457
:100B88002A46B144C6EB0B0609EB0B05B818002141
:100B9800AA1A00F095F90028AFD0002071E0019A58
:100BA8000026914499442A46EEE7002EFAD0DDF853
:100BB8000C2493423CBFC2EB0B0306469944F2E770
:100BC800009E4FF000080099AB1BB34238BF334674
:100BD800C1F101026E1E019201F1FF3A5A4689469F
:100BE800AB460133CDF80C3408EB0B05B8180021DF
:100BF800AA1A00F065F90028CFD1002D40D07B1942
:100C080003A913F8013C51F82330002B30D1B1452A
:100C180013D208EB090314F80910FA18FB5C99427F
:100C280018BF4B4627D14B4604E012F8011FE05C81
:100C3800884220D10133B342F7D3BAF1FF3F53467C
:100C48002CD007EB080C14F80A101CF80A20914263
:100C58000CD10AEB0802BA1804E0E05C12F8011D96
:100C6800884203D1013BF8D260460AE0DDF80C3433
:100C780098442A46B8E701992A4688449844B3E735
:100C8800284605B00DF5806DBDE8F08F009B013654
:100C98009E427FF673AF07EB0900F2E707EB080CFB
:100CA8006046EEE72DE9F04F8346037885B00C46A1
:100CB800002B00F0F9800A78A2B106460131012024
:100CC80002E011F8012B8AB1934214BF002000F012
:100CD800010016F8013F0D46002BF2D12B782BB1FD
:100CE8004FF0000B584605B0BDE8F08F0028F9D149
:100CF8000BF101002178FFF7CBFB2D1BA5F10102B9
:100D0800534243EB0203002808BF43F001030746A0
:100D180083B90BEB0508404594BFC0EB08084FF0BA
:100D280001081F2D08D9414622462B46FFF7A2FE8F
:100D38008346D7E78346D5E7294603AA2046FFF727
:100D48003BFE03996118814620464A46FFF748FA58
:100D580000284FD109F1FF33C9F10102064601927B
:100D680082464246C84699460AEB050BB818002148
:100D7800C2EB0B0200F0A4F80028B1D1BBF1000FC0
:100D8800B0D046452CBF334643469D420FD903EBAE
:100D98000A01E05C7A18795C884205D075E012F89F
:100DA800011FE05C884270D101339D42F7D1B04504
:100DB8007DD907EB0A0214F809104B4612F80920EE
:100DC800914202BF09EB0A01AC46791806D06EE0E1
:100DD800A55C11F8010D854203D113465A1EB34292
:100DE800F6D1654601369E4267D8039E5A46B244FC
:100DF800AE1BB9E7C9F10101C9EB0503424600265C
:100E080009F1FF3A88464B4538BF4B4601330393F7
:100E180006EB050BB8180021C2EB0B0200F050F8E6
:100E280000287FF45DAFBBF1000F3FF45BAF4D4589
:100E380012D906EB090314F80910FA18FB5C994259
:100E480008BF4B4605D026E012F8011FE05C884237
:100E580022D101339D42F7D1BAF1FF3F534628D042
:100E680007EB060C14F80A101CF80A20914217D157
:100E78000AEB0602BA1804E0E05C12F8011D884289
:100E88000ED1013BF8D2E3462CE7019A00269244A2
:100E98005A469A4468E74B4646445A46F618B7E716
:100EA800039B5A46F618B3E70D46012016E743465A
:100EB80098E707EB060CE34614E707EB0A0B11E784
:100EC80010F0030F034670B4C9B211D0002A22D023
:100ED80003788B421DD0013A013005E0DAB110F8F1
:100EE800014B013A8C4218D010F0030F0346F5D19C
:100EF800032A14D87AB1187888420ED0541E5D1C83
:100F080003E015F8016B8E4203D0013C2846F8D265
:100F1800002070BC70471046FBE71846F9E741EA25
:100F2800012646EA0646184653F8044B86EA0404A6
:100F3800A4F1013525EA040414F0803F03D1043AF2
:100F48001846032AEFD80346D4E700BF0000000084
:100F5800C1F30A5C0246ACF57E7C2DE9F84FACF192
:100F68000704132C0B4606460F468946804627DCA5
:100F7800002C52DB4FF6FF7CC0F20F0C4CFA04FA3F
:100F88000AEA0105054317D037A3D3E9002300F087
:100F980075F80022002300F0B3FC002856D0002F7B
:100FA80005DD4FF4801353FA04F407EB040929EA2A
:100FB8000A0900264B46324610461946BDE8F88F06
:100FC800332C07DDB4F5806FF6D100F057F80246F0
:100FD8000B46F1E74FF0FF3BACF11B0C2BFA0CFB77
:100FE8001BEA000FE8D020A3D3E9002300F046F85D
:100FF8000022002300F084FC40B3002F0ADD142CEB
:1010080006D00126C4F13404A64016EB080601D325
:1010180007F1010926EA0B0619E013A3D3E9002317
:1010280000F02CF80022002300F06AFC78B1002FB1
:1010380013DB46EA07054FF000094D45C3F6F07982
:101048000CBF2E46002608BFA94600E0B9464B460D
:10105800324610461946BDE8F88F00264FF0004981
:10106800F5E700BFAFF300809C7500883CE4377E4D
:1010780081F0004102E000BF83F0004330B54FEA41
:1010880041044FEA430594EA050F08BF90EA020FAE
:101098001FBF54EA000C55EA020C7FEA645C7FEA41
:1010A800655C00F0E2804FEA5454D4EB5555B8BF64
:1010B8006D420CDD2C4480EA020281EA030382EAD5
:1010C800000083EA010180EA020281EA0303362D67
:1010D80088BF30BD11F0004F4FEA01314FF4801C3A
:1010E8004CEA113102D0404261EB410113F0004F4C
:1010F8004FEA03334CEA133302D0524263EB430303
:1011080094EA050F00F0A780A4F10104D5F1200EA0
:101118000DDB02FA0EFC22FA05F2801841F10001FB
:1011280003FA0EF2801843FA05F359410EE0A5F1CF
:1011380020050EF1200E012A03FA0EFC28BF4CF000
:10114800020C43FA05F3C01851EBE37101F00045B6
:1011580007D54FF0000EDCF1000C7EEB00006EEBC3
:101168000101B1F5801F1BD3B1F5001F0CD349084D
:101178005FEA30004FEA3C0C04F101044FEA4452A4
:1011880012F5800F80F09A80BCF1004F08BF5FEA2B
:10119800500C50F1000041EB045141EA050130BD0B
:1011A8005FEA4C0C404141EB010111F4801FA4F1AE
:1011B8000104E9D191F0000F04BF01460020B1FA03
:1011C80081F308BF2033A3F10B03B3F120020CDA3B
:1011D8000C3208DD02F1140CC2F10C0201FA0CF019
:1011E80021FA02F10CE002F11402D8BFC2F1200C7E
:1011F80001FA02F120FA0CFCDCBF41EA0C01904034
:10120800E41AA2BF01EB0451294330BD6FEA04047C
:101218001F3C1CDA0C340EDC04F11404C4F1200267
:1012280020FA04F001FA02F340EA030021FA04F379
:1012380045EA030130BDC4F10C04C4F1200220FAD0
:1012480002F001FA04F340EA0300294630BD21FA0E
:1012580004F0294630BD94F0000F83F4801306BFD4
:1012680081F480110134013D4EE77FEA645C18BFC8
:101278007FEA655C29D094EA050F08BF90EA020F5F
:1012880005D054EA000C04BF1946104630BD91EA57
:10129800030F1EBF0021002030BD5FEA545C05D15A
:1012A8004000494128BF41F0004130BD14F5800499
:1012B8003CBF01F5801130BD01F0004545F0FE410D
:1012C80041F470014FF0000030BD7FEA645C1ABF42
:1012D800194610467FEA655C1CBF0B46024650EA79
:1012E800013406BF52EA033591EA030F41F40021A5
:1012F80030BD00BF90F0000F04BF0021704730B52B
:101308004FF4806404F132044FF000054FF00001FF
:1013180050E700BF90F0000F04BF0021704730B5C0
:101328004FF4806404F1320410F0004548BF404295
:101338004FF000013EE700BF42004FEAE2014FEAEA
:1013480031014FEA02701FBF12F07F4393F07F4FC5
:1013580081F06051704792F0000F14BF93F07F4FF7
:10136800704730B54FF4607401F0004521F000413A
:1013780020E700BF50EA010208BF704730B54FF0C0
:1013880000050AE050EA010208BF704730B511F0C5
:10139800004502D5404261EB41014FF4806404F1FD
:1013A80032045FEA915C3FF4DCAE4FF003025FEA7F
:1013B800DC0C18BF03325FEADC0C18BF033202EB07
:1013C800DC02C2F1200300FA03FC20FA02F001FA61
:1013D80003FE40EA0E0021FA02F11444C1E600BF00
:1013E80070B54FF0FF0C4CF4E06C1CEA11541DBFB3
:1013F8001CEA135594EA0C0F95EA0C0F00F0DEF87E
:101408002C4481EA030621EA4C5123EA4C5350EA62
:10141800013518BF52EA033541F4801143F48013B3
:1014280038D0A0FB02CE4FF00005E1FB02E506F044
:101438000042E0FB03E54FF00006E1FB03569CF099
:10144800000F18BF4EF0010EA4F1FF04B6F5007F9F
:1014580064F5407404D25FEA4E0E6D4146EB060611
:1014680042EAC62141EA55514FEAC52040EA5E509A
:101478004FEACE2EB4F1FD0C88BFBCF5E06F1ED844
:10148800BEF1004F08BF5FEA500E50F1000041EB7B
:10149800045170BD06F0004646EA010140EA020028
:1014A80081EA0301B4EB5C04C2BFD4EB0C0541EA4A
:1014B800045170BD41F480114FF0000E013C00F35F
:1014C800AB8014F1360FDEBF002001F0004170BD83
:1014D800C4F10004203C35DA0C341BDC04F114049C
:1014E800C4F1200500FA05F320FA04F001FA05F228
:1014F80040EA020001F0004221F0004110EBD370F5
:1015080021FA04F642EB06015EEA430E08BF20EA20
:10151800D37070BDC4F10C04C4F1200500FA04F3C3
:1015280020FA05F001FA04F240EA020001F0004155
:1015380010EBD37041F100015EEA430E08BF20EAC8
:10154800D37070BDC4F1200500FA05F24EEA020E10
:1015580020FA04F301FA05F243EA020321FA04F03F
:1015680001F0004121FA04F220EA020000EBD370F6
:101578005EEA430E08BF20EAD37070BD94F0000FF6
:101588000FD101F00046400041EB010111F4801F2A
:1015980008BF013CF7D041EA060195F0000F18BFDB
:1015A800704703F00046520043EB030313F4801F17
:1015B80008BF013DF7D043EA0603704794EA0C0FD1
:1015C8000CEA135518BF95EA0C0F0CD050EA4106E7
:1015D80018BF52EA4306D1D181EA030101F0004164
:1015E8004FF0000070BD50EA410606BF104619468C
:1015F80052EA430619D094EA0C0F02D150EA013698
:1016080013D195EA0C0F05D152EA03361CBF1046D8
:1016180019460AD181EA030101F0004141F0FE4177
:1016280041F470014FF0000070BD41F0FE4141F4FB
:10163800780170BD70B54FF0FF0C4CF4E06C1CEAFB
:1016480011541DBF1CEA135594EA0C0F95EA0C0FB0
:1016580000F0A7F8A4EB050481EA030E52EA03356B
:101668004FEA013100F088804FEA03334FF080558C
:1016780045EA131343EA12634FEA022245EA1115B9
:1016880045EA10654FEA00260EF000419D4208BF6A
:10169800964244F1FD0404F5407402D25B084FEA17
:1016A8003202B61A65EB03055B084FEA32024FF4C3
:1016B80080104FF4002CB6EB020E75EB030E22BF20
:1016C800B61A754640EA0C005B084FEA3202B6EBE0
:1016D800020E75EB030E22BFB61A754640EA5C008F
:1016E8005B084FEA3202B6EB020E75EB030E22BF1F
:1016F800B61A754640EA9C005B084FEA3202B6EB20
:10170800020E75EB030E22BFB61A754640EADC00DE
:1017180055EA060E18D04FEA051545EA16754FEA40
:1017280006164FEAC30343EA52734FEAC2025FEA5E
:101738001C1CC0D111F4801F0BD141EA00014FF0ED
:1017480000004FF0004CB6E711F4801F04BF0143BE
:101758000020B4F1FD0C88BFBCF5E06F3FF6AFAEDA
:10176800B5EB030C04BFB6EB020C5FEA500C50F16A
:10177800000041EB045170BD0EF0004E4EEA1131ED
:1017880014EB5C04C2BFD4EB0C0541EA045170BDF4
:1017980041F480114FF0000E013C90E645EA060E38
:1017A8008DE60CEA135594EA0C0F08BF95EA0C0F66
:1017B8003FF43BAF94EA0C0F0AD150EA01347FF4AE
:1017C80034AF95EA0C0F7FF425AF104619462CE785
:1017D80095EA0C0F06D152EA03353FF4FDAE1046E8
:1017E800194622E750EA410618BF52EA43067FF439
:1017F800C5AE50EA41047FF40DAF52EA43057FF4C9
:10180800EBAE12E74FF0FF3C06E000BF4FF0010CD3
:1018180002E000BF4FF0010C4DF804CD4FEA410C37
:101828007FEA6C5C4FEA430C18BF7FEA6C5C1BD004
:1018380001B050EA410C0CBF52EA430C91EA030F85
:1018480002BF90EA020F0020704710F1000F91EAE2
:10185800030F58BF994208BF90422CBFD8176FEAB0
:10186800E37040F0010070474FEA410C7FEA6C5C7E
:1018780002D150EA013C07D14FEA430C7FEA6C5C85
:10188800D6D152EA033CD3D05DF8040B704700BFB1
:101898008446104662468C461946634600E000BFFF
:1018A80001B5FFF7B7FF002848BF10F1000F01BDD1
:1018B8004DF808EDFFF7F4FF0CBF012000205DF89C
:1018C80008FB00BF4DF808EDFFF7EAFF34BF012021
:1018D80000205DF808FB00BF4DF808EDFFF7E0FFBA
:1018E80094BF012000205DF808FB00BF4DF808ED0B
:1018F800FFF7CEFF94BF012000205DF808FB00BF72
:101908004DF808EDFFF7C4FF34BF012000205DF853
:1019180008FB00BF4FEA4102B2F1E04324BFB3F530
:10192800001CDCF1FE5C0DD901F0004C4FEAC0024E
:101938004CEA5070B2F1004F40EB830008BF20F032
:101948000100704711F0804F21D113F13872BCBFEC
:1019580001F00040704741F480114FEA5252C2F141
:101968001802C2F1200C10FA0CF320FA02F018BF8A
:1019780040F001004FEAC1234FEAD32303FA0CFCDD
:1019880040EA0C0023FA02F34FEA4303CCE77FEA6C
:10199800625307D150EA01331EBF4FF0FE4040F4B6
:1019A8004000704701F0004040F0FE4040F4000065
:1019B800704700BF80F0004002E000BF81F00041A6
:1019C80042001FBF5FEA410392EA030F7FEA226CDD
:1019D8007FEA236C6AD04FEA1262D2EB1363C1BF6D
:1019E800D218414048404140B8BF5B42192B88BFDC
:1019F800704710F0004F40F4000020F07F4018BFFF
:101A0800404211F0004F41F4000121F07F4118BF1E
:101A1800494292EA030F3FD0A2F1010241FA03FCC6
:101A280010EB0C00C3F1200301FA03F100F00043AE
:101A380002D5494260EB4000B0F5000F13D3B0F176
:101A4800807F06D340084FEA310102F10102FE2AE5
:101A580051D2B1F1004F40EBC25008BF20F0010055
:101A680040EA03007047490040EB000010F4000F03
:101A7800A2F10102EDD1B0FA80FCACF1080CB2EB96
:101A88000C0200FA0CF0AABF00EBC25052421843F5
:101A9800BCBFD0401843704792F0000F81F400019A
:101AA80006BF80F400000132013BB5E74FEA41036D
:101AB8007FEA226C18BF7FEA236C21D092EA030FD9
:101AC80004D092F0000F08BF0846704790EA010F53
:101AD8001CBF0020704712F07F4F04D1400028BF80
:101AE80040F00040704712F100723CBF00F5000062
:101AF800704700F0004343F0FE4040F40000704798
:101B08007FEA226216BF08467FEA23630146420243
:101B180006BF5FEA412390EA010F40F48000704756
:101B28004FF0000304E000BF10F0004348BF4042FC
:101B38005FEA000C08BF704743F0964301464FF038
:101B480000001CE050EA010208BF70474FF0000394
:101B58000AE000BF50EA010208BF704711F00043D5
:101B680002D5404261EB41015FEA010C02BF8446A5
:101B78000146002043F0B64308BFA3F18053A3F504
:101B88000003BCFA8CF2083AA3EBC25310DB01FA4B
:101B980002FC634400FA02FCC2F12002BCF1004FCF
:101BA80020FA02F243EB020008BF20F00100704760
:101BB80002F1200201FA02FCC2F1200250EA4C00B4
:101BC80021FA02F243EB020008BF20EADC707047FA
:101BD8004FF0FF0C1CEAD0521EBF1CEAD15392EA08
:101BE8000C0F93EA0C0F6FD01A4480EA010C4002E4
:101BF80018BF5FEA41211ED04FF0006343EA50103E
:101C080043EA5111A0FB01310CF00040B1F5000F7F
:101C18003EBF490041EAD3715B0040EA010062F12E
:101C28007F02FD2A1DD8B3F1004F40EBC25008BF18
:101C380020F00100704790F0000F0CF0004C08BF36
:101C480049024CEA502040EA51207F3AC2BFD2F103
:101C5800FF0340EAC250704740F400004FF0000311
:101C6800013A5DDC12F1190FDCBF00F0004070474B
:101C7800C2F10002410021FA02F1C2F1200200FA89
:101C880002FC5FEA310040F1000053EA4C0308BF50
:101C980020EADC70704792F0000F00F0004C02BFA1
:101CA800400010F4000F013AF9D040EA0C0093F01C
:101CB800000F01F0004C02BF490011F4000F013B76
:101CC800F9D041EA0C018FE70CEAD15392EA0C0FE4
:101CD80018BF93EA0C0F0AD030F0004C18BF31F04F
:101CE800004CD8D180EA010000F00040704790F025
:101CF800000F17BF90F0004F084691F0000F91F0C9
:101D0800004F14D092EA0C0F01D142020FD193EA8E
:101D18000C0F03D14B0218BF084608D180EA010016
:101D280000F0004040F0FE4040F40000704740F0F2
:101D3800FE4040F4400070474FF0FF0C1CEAD052C0
:101D48001EBF1CEAD15392EA0C0F93EA0C0F69D01C
:101D5800A2EB030280EA010C49024FEA402037D087
:101D68004FF0805343EA111143EA10130CF000407E
:101D78008B4238BF5B0042F17D024FF4000C8B426E
:101D880024BF5B1A40EA0C00B3EB510F24BFA3EB4E
:101D9800510340EA5C00B3EB910F24BFA3EB91031E
:101DA80040EA9C00B3EBD10F24BFA3EBD10340EA78
:101DB800DC001B0118BF5FEA1C1CE0D1FD2A3FF6BE
:101DC80050AF8B4240EBC25008BF20F00100704773
:101DD8000CF0004C4CEA50207F32C2BFD2F1FF0316
:101DE80040EAC250704740F400004FF00003013A47
:101DF80037E792F0000F00F0004C02BF400010F4EB
:101E0800000F013AF9D040EA0C0093F0000F01F0FE
:101E1800004C02BF490011F4000F013BF9D041EA20
:101E28000C0195E70CEAD15392EA0C0F08D1420253
:101E38007FF47DAF93EA0C0F7FF470AF084676E726
:101E480093EA0C0F04D14B023FF44CAF08466EE7FF
:101E580030F0004C18BF31F0004CCAD130F00042CD
:101E68007FF45CAF31F000437FF43CAF5FE700BF25
:101E78004FF0FF3C06E000BF4FF0010C02E000BF4E
:101E88004FF0010C4DF804CD4FEA40024FEA4103F0
:101E98007FEA226C18BF7FEA236C11D001B052EAA6
:101EA800530C18BF90EA010F58BFB2EB030088BF6C
:101EB800C81738BF6FEAE17018BF40F001007047DB
:101EC8007FEA226C02D15FEA402C05D17FEA236CBD
:101ED800E4D15FEA412CE1D05DF8040B704700BF04
:101EE800844608466146FFE70FB5FFF7C9FF00289B
:101EF80048BF10F1000F0FBD4DF808EDFFF7F4FFD4
:101F08000CBF012000205DF808FB00BF4DF808ED6C
:101F1800FFF7EAFF34BF012000205DF808FB00BF8F
:101F28004DF808EDFFF7E0FF94BF012000205DF8B1
:101F380008FB00BF4DF808EDFFF7D2FF94BF012062
:101F480000205DF808FB00BF4DF808EDFFF7C8FF5B
:101F580034BF012000205DF808FB00BF42000ED20C
:101F6800B2F1FE4F0BD34FF09E03B3EB126209D4CC
:101F78004FEA002343F0004323FA02F070474FF082
:101F88000000704712F1610F01D1420202D14FF0F7
:101F9800FF3070474FF00000704700BF00F026F890
:101FA8000C4880F30888002103E00B4B5B58435032
:101FB80004310A480A4B42189A42F6D3094A02E009
:101FC800002342F8043B084B9A42F9D313F044FF2C
:101FD8007047000000C00020A8BE020800000020D2
:101FE800180E0020180E00200C3B00207047FEE75A
:101FF80010B586B0002301244FF46022114801A9CE
:1020080001938DF80930039204938DF808408DF8F8
:1020180014401CF0FBF90B4821461CF01DFA094836
:102028001CF024FA07481CF026FA0028FAD10548C3
:102038001CF025FA03481CF027FA0028FAD106B04C
:1020480010BD00BF00240140014610B50D48012213
:1020580003231CF027FA0B4801211CF019FA7F20F2
:102068001DF056F8074802211CF066FA0028F6D041
:10207800044802211CF066FA0248BDE810401CF032
:1020880058BA00BF002401400C4A0C2303FB01236B
:1020980010B59C880CB9588010BD5B8803F11304F7
:1020A800844204DA142B07D9133B834204DC0C2343
:1020B80003FB012102238B8010BD00BF5C200020A0
:1020C8000A4B10B500241C7021464FF48072084852
:1020D800FEF760F9074B43F6DE301C70064B1C70A8
:1020E8000DF09AF9054B187010BD00BFD8100020EC
:1020F800E0110020F7120020E3120020E512002072
:10210800074B1978013101F01F011970054B1A7836
:102118008A4203D1013202F01F021A70704700BFD1
:10212800E3120020F712002010B50A4B0A4A03EB0D
:10213800C0000A4B1978036802EBC10442F8313039
:102148004368002163600822FEF724F9BDE81040C7
:10215800FFF7D6BFDC100020E0110020E3120020BA
:102168002DE9F3479846474B1746DA78054602F0BB
:102178002002D2B20E46BDF82890002A7AD1B8F1D2
:10218800000F0AD19B7803F04003DBB2C3B900F01B
:102198007F0000F56E50633009E0B8F1010F09D1F6
:1021A8009B7803F04003DBB2BBB949F2D8400DF08D
:1021B80033F9C4B2002C5FD0B8F1000F09D100E0A8
:1021C800012405F07F0149000DF1060001F5715168
:1021D8000CE0B8F1010F0CD100E04446E90101F52B
:1021E8000A41D8310DF1060001EB460102220DF03B
:1021F80024F9BDF9063013B9B8F1000F3ED0B9F192
:10220800000F06D1204B93F800A0FFF779FF1F4B72
:1022180008E01F4B93F800A00AF1010202F01F0228
:102228001A701C4BB8F1000F12D1BDF8061040F619
:10223800B8326DB212EA250538BF4FF47A756D18B9
:1022480003EBCA0223F83A509470D670177109E06C
:10225800B8F1010F06D1BDF8061003EBCA0223F846
:102268003A10947003EBCA0383F80580A3F806902C
:10227800012004E0002002E0204600E04046BDE8DE
:10228800FC8700BF302A0020E3120020E011002064
:10229800D7100020DC10002001228240094B0A4997
:1022A8001B78D2B2097808E0084800EBC3008078B0
:1022B800024205D1013303F01F038B42F4D1FF23FF
:1022C80018467047F7120020E3120020E0110020A2
:1022D800F0B500EB800101F56E51314F042285B055
:1022E800304836310DF0A9F82F4C3B7804EBC30287
:1022F80056791EBB2B4D31222A7107326A7134F987
:10230800331001A8343A05F063FE3B7802A804EBC9
:10231800C3031979022205F05BFE3B780DF10A0030
:1023280004EBC304E178032205F052FEA81D01A9BD
:102338000922FEF705FB2E740F250CE0012E0AD1A9
:10234800184A322111710531517134F8333008259A
:10235800190AD1719371002314481A4612E010F833
:10236800011FA1F13004E4B2092C04D8E318302984
:10237800DBB203D004E037395B1800E00A33DBB284
:102388000132D2B2AA42EAD10F21B3FBF1F108011E
:10239800411A5B1A0348C3F10F03835405B0F0BD1B
:1023A800DD110020E6120020E0110020E5120020D7
:1023B8002DE9F3415F4B04461B7843B15E4B1B7814
:1023C80003F02403042B02D1002900F0AF805B4BFB
:1023D8005B4F1B78002B00F093805A4821461BF076
:1023E800BBF98046002840F08B803B1993F8803079
:1023F8002D2B01D0532B2DD1534E3578F5B10DF03F
:1024080017FB611C034630B1337893201E330093C9
:102418000122002302E0009001229320FFF7A0FE92
:102428000DF006FB014628B1337813201E330093C4
:10243800002101E0009013200A465EE0611C0122A1
:1024480093202B460095FFF78BFE00951320294615
:102458002A4652E0542B05D10090611C9420012299
:1024680043464BE0462B384D11D12E7866B10DF01E
:10247800DFFA611C034620B12B789A201E330093A3
:1024880014E000909A2018E000969A202CE02E780C
:1024980026B30DF0CDFA0346611C04F11C0043B1CC
:1024A8002B7860F07F001E330093C0B201224346B0
:1024B80004E060F07F000093C0B20122FFF750FEF5
:1024C8000DF0B6FA21B2024628B12B7803201E334C
:1024D8000093002211E0009003200EE004F11C009C
:1024E80060F07F000096C0B2611C01223346FFF7FE
:1024F80037FE00960320214632460123FFF730FEBF
:10250800104821463F191BF011F997F88030542BD9
:102518000CD8532B03D22D2B01D0462B06D10B48B8
:10252800214602B0BDE8F0411BF00BB902B0BDE88E
:10253800F08100BFDA100020DC140020E412002033
:10254800881E0020EE14002046150020E614002006
:1025580037B5114B04461B780D4693B10F482146F9
:102568001BF0FAF8034660B9012D04F1010103D10B
:1025780000902A46812002E0009001229820FFF76F
:10258800EFFD214605481BF0D1F80548214603B068
:10259800BDE830401BF0D5B8E4120020EE1400204E
:1025A80003130020024B1A7842F001021A70704798
:1025B8003916002008B50C4B1A780C4B03EBC203F4
:1025C800597921B101290CBF0921002100E010210E
:1025D80040221346064805F01FFB064B1A7842F0C6
:1025E80002021A7008BD00BFDD110020E0110020B2
:1025F800E612002039160020034B1A7802F0F80280
:102608006FF3C3021A70704739160020024B1A780C
:1026180042F004021A70704739160020024B1A78EB
:1026280042F008021A7070473916002038B5114B6D
:102638001C7814F0010502D1FFF7B4FF05E004F09F
:102648000405EDB21DB9FFF7E1FF284638BD04F0D7
:102658000805EDB215B9FFF7E1FFF6E704F002044B
:10266800E4B21CB9FFF7A6FF204638BDFFF7C4FF48
:10267800012038BD39160020014B1878704700BF7B
:10268800D810002030B50F4B85B01B780546BBB974
:102698000D4C2278024112F0010F11D0FF22019354
:1026A8000121431C009202933C200B46FC3A0CF09B
:1026B80027FF012313FA05F5237823EA050525707A
:1026C80005B030BDE5120020E11200202DE9F843E5
:1026D800134A00231370134A1678134A1178904648
:1026E800B14219D0114D2A78072A88BF2B7095F866
:1026F80000902C780D4F2046FFF7CEFDFF280CD117
:102708000134E4B2072C3C7001D900233B702B78CC
:102718004B45EED188F80060FF242046BDE8F883D9
:10272800D8100020F7120020E3120020DE1100204C
:102738000121814010B5C943C9B20023094A9A183A
:102748009478083301EA0404B3F5807F9470F5D1D6
:10275800FFF798FF43F6DE300CF05EFE024B187070
:1027680010BD00BFE0110020E51200202DE9F04166
:102778008B4E054633788B4C13B12378834204D0B3
:1027880043F6DE300CF048FE30702570864C237816
:10279800072B00F2E680DFE813F008002000330082
:1027A80051005A0070008B00B500804B1E221A7031
:1027B8002846FFF771FD7E4BFF28187000F0D58082
:1027C8001AF020FB7B4B002093F8702042F00102A6
:1027D80083F87020784B187065E0744B1B78002BD9
:1027E80000F0C3801AF05AFC012840F00D812378CC
:1027F800142201332370714B01381A70BDE8F0813F
:102808006A4B1B78002B00F0B0806C4E307808B90A
:1028180001234AE01AF042FC022804D01AF03EFCD8
:10282800032840F0F1801AF0EDFA237804220133EE
:1028380023701D233370624B1A70E5E05B4B1E2238
:102848001A702846FFF744FD237801332370574B4D
:102858001B78002B00F08980584B1D78002D40F024
:10286800D3801020FFF7E2FE002800F0D180237803
:10287800284601332370BDE8F0814C4B1B78002BB0
:1028880073D005F033FA002800F0C2804B4B7D224C
:102898001A70494B00201870464B93F8702042F08C
:1028A800010283F87020237801332370BDE8F0819A
:1028B8003E4B1B78002B58D01AF0F0FB01283F4FF5
:1028C80003D01AF0EBFB03280DD1012212FA05F50B
:1028D8003C4B1A7822EA05051D7064233B70237867
:1028E8000133237090E03878002840F08D80344A16
:1028F800032323701378013BDBB21370002B34D011
:10290800BDE8F0812B4B2D4F93F86A3013B13B781B
:10291800002B79D100233B700133AB40244A2A486D
:102928001178904600EBC10090F802E02EEA03030C
:1029380083703BB9254B1A788A4203D1013202F0E1
:102948001F021A702846FFF7A7FC1D4B0422FF2818
:1029580088F800001A703FD0032323701A333B70A5
:1029680052E000202070BDE8F081FFF745FE00230B
:1029780023701AF047FA3378013BDBB2337033B176
:10298800134B9B7803F04003DBB2002B3FD0284663
:10299800FFF7CEFE0F4B1A7801321A7031E000BFF4
:1029A800E5120020DB100020D8100020E2120020E1
:1029B800DD110020FE2D0020D9100020D6100020A7
:1029C800E0120020E1120020E0110020F7120020A0
:1029D800302A0020DE1100200E4B9A7802F04002C7
:1029E800D2B21AB11A6842F400021A60FFF704FE64
:1029F8001AF008FA0023237043F6DE300CF00CFDC1
:102A08003070FF20BDE8F0810020BDE8F081FF2094
:102A1800BDE8F081302A0020044B1A780AB1013A47
:102A28001A701B780BB9FFF783BE7047E5120020B8
:102A3800044A054B10781B7803EA501000F0010097
:102A4800704700BF302A0020B5140020044B054A07
:102A58001B781078C3F3400303EA1010704700BFD7
:102A6800B5140020302A0020034B044A1B78D07884
:102A7800C3F3800318407047B5140020302A0020A3
:102A8800044B054A1B78D078C3F3C00303EA50000F
:102A9800704700BFB5140020302A0020044B054AB7
:102AA8001B78D078C3F3001303EA9000704700BF87
:102AB800B5140020302A0020044B1878044BDB782A
:102AC8005B005BB2DB1103EAD0107047B51400203D
:102AD800302A00202DE9F041154E0024B04620E0B0
:102AE8002046294617F0BAFA90B1F35DFF2B0FD0B4
:102AF8004FF4A07363430A2202FB053318F803302E
:102B0800DB0905D00B4B1878C0F30010BDE8F08145
:102B180001350A37202DE3D10134022C06F5A076C1
:102B280002D000273D46DBE70020BDE8F08100BF6A
:102B38004A2F0020B514002008B516F0D5FE034B27
:102B48001B7800EA931000F0010008BDB5140020BE
:102B5800044B054A1B78D078C3F3401303EAD0002E
:102B6800704700BFB5140020302A00202DE9F84F27
:102B7800FFF75EFF8146FFF769FF8246FFF774FFA4
:102B88008346FFF77DFF8046FFF788FF0446FFF77F
:102B9800A1FF0546FFF7DCFF0746FFF7CDFF064616
:102BA800FFF78AFF4FEA8B0343EA4A0343EA090324
:102BB80043EAC80343EA471343EA861345EA040491
:102BC80043EAC013E0B243EA0010BDE8F88F000002
:102BD800044B987800F00F00A0F10203584240EB34
:102BE8000300704754130020044B987800F00F003E
:102BF800A0F10102504240EB02007047541300203C
:102C0800044B987800F00F00A0F10301484240EB14
:102C18000100704754130020054B987800F00F000E
:102C2800A0F1060CDCF1000040EB0C00704700BF7F
:102C380054130020514AF0B513781446012B29D0BB
:102C480003D3022B40F098805EE04D484D4B04784A
:102C580019786FF3C304047001F0F80158786FF322
:102C6800C301197000F08001C9B2002900F0848006
:102C7800012111709C78062204F00F045443024687
:102C88004148005D60F306025A701A7861F3020247
:102C98001A70F0BD3B494D780B4625F07F0000289F
:102CA80038D00A7802F00802D2B222B9344A117830
:102CB80041F0080111709A7802F00F02012A04D13C
:102CC8002F4A117841F00101117015F07F0F53D18F
:102CD80019789E7801F00700062206F00F0602FB1D
:102CE8000606294F5D78BE5D013066F3060500F0E3
:102CF80007005D7090FBF2F502FB150262F302011A
:102D0800197002232370F0BD1E494D780B4625F03B
:102D18007F0028B98B7860F303038B701070F0BDC7
:102D2800174A11786FF3C3011170997801F00F01F8
:102D3800012903D111786FF30001117015F07F0F8D
:102D48001AD119789E7801F00700062206F00F06BE
:102D580002FB06060C4F5D78BE5D013066F3060582
:102D680000F007005D7090FBF2F502FB150262F3BC
:102D78000201197001232370F0BD00BFA3130020C6
:102D88000213002054130020B8F1010808B543F6D7
:102D9800ED200CF041FB014B187008BD0113002019
:102DA800014B1870704700BFBE140020024B1A5C1C
:102DB8006FF303021A547047FD13002070B50C46D8
:102DC800C10001F5CC411248683108220CF035FBEE
:102DD80000250F482946EEB21AF0BEFC98B10D4BFB
:102DE8002278EB5C1A420ED13046FFF7DFFF294606
:102DF80009481AF0A6FCF608074B06F5CA40A830A1
:102E0800995D0CF0FFFA0135402DE2D170BD00BF8D
:102E1800C0140020B41300205713002038B546F220
:102E2800F05540242046FFF7C1FFA5F5CA43094ADB
:102E3800B03BD15C11F0100F06D06FF30411D154E0
:102E4800284600210CF0DEFA0134E4B20135B82C32
:102E5800E8D138BDFD1300207FB5924B05461B789D
:102E6800002B00F01681904E325C541C04F00F04C5
:102E780064F303023F2832542AD8002C00F00E8154
:102E880001339C4240F00781D3B26FF303033354FC
:102E9800864BC4081B1993F8902100F0070352FAD7
:102EA80003F313F0010F40F0F880294680481AF028
:102EB8003DFC7F4B04F5CA40195DA83001240CF095
:102EC800A1FA2D19022300930194029518209CE081
:102ED800002C00F0E38001339C4240F0DC80335C3E
:102EE80001216FF30303335400F5CA40B0300CF0EE
:102EF80089FA735D43F010037355A5F14003DBB203
:102F0800072B07D804220092013302320192029360
:102F18001920AAE0A5F14803DBB2072B07D8042241
:102F2800009201330332019202931A2061E0A5F165
:102F38005003DBB2062B07D8042200920133033278
:102F4800019202931B2054E0A5F15703DBB2032B37
:102F580007D8042200920133033201920293212000
:102F680047E0A5F15B03DBB2012B07D804220092EE
:102F78000133023201920293222076E05D2D06D1C0
:102F8800042300930193043B02935D207BE05E2DB4
:102F980007D10423009301330193053B029328468C
:102FA80071E0A5F15F03DBB21F2B09D80422009260
:102FB800013392180192029333200121053A64E00B
:102FC80005F16103DBB2072B07D804220092013315
:102FD8000332019202935F200BE005F15903DBB243
:102FE800012B09D804220092013303320192029383
:102FF80060200121043A48E0AA2D0CD10423009353
:103008000124043B019402936120214603222346B4
:103018000CF076FA42E0A92D07D104230093023B75
:103028000193023B029362202DE0AC2D08D10423CA
:1030380000930322043B019202936320012124E0C0
:10304800AB2D06D104230093043B01930293642023
:1030580019E005F15303DBB2032B09D804220092CF
:10306800013302320192029368200121033A0CE0F5
:103078004F35EDB2062D10D80423009301350233E5
:10308800019302956A20012103220B460CF038FABD
:1030980003E01C4602E0002400E00124204604B0BE
:1030A80070BD00BF00000020FD130020881E002016
:1030B80057130020024B185CC0F30010704700BF84
:1030C800FD130020F8B508220E4600210746FDF73B
:1030D80061F946F2686500243378234113F0010F43
:1030E80008D02946064808220CF0A7F938460449B2
:1030F8001AF0DFFA01340835082CEDD1F8BD00BF0D
:10310800CA140020024846F2A85108220CF095B9CA
:103118005713002070B5044600F56A5044300CF08F
:103128007BF90B4D06462B7813F0010F02D1CC200A
:103138001BF000F92B8843F001032B80054B1E552B
:10314800054B13F8242042F0010203F8242070BD37
:10315800DC1400203413002013130020024B185CE9
:10316800084100F001007047B413002070B505460F
:103178000024094BE0B2E618E35C4BB12946FFF79F
:10318800EDFF28B100233370044821461AF0D9FA1C
:103198000134402CEDD170BDFE14002044130020F2
:1031A80038B5054600242846E1B2FFF7D7FF10B12D
:1031B800044BE35C23B90134082CF4D1002038BD5A
:1031C800012038BD3413002038B505460CF030FC1A
:1031D800A0B100242846E1B2FFF7C0FF40B1084B78
:1031E80013F8243013F0010F02D0064BE35C23B12F
:1031F8000134082CEED1002038BD012038BD00BFB5
:103208001313002034130020F8B511480021402280
:10321800FDF7C0F846F26865002401270D482946E5
:103228000822A7400CF009F9FFB2002609483146E8
:103238001AF092FA20B1064BF25C47EA0202F25405
:103248000136402EF2D101340835082CE5D1F8BDFD
:10325800B4130020CA1400202DE9FF41002634468B
:10326800B0461A4B1B78234113F00102184B23D0A8
:10327800184F1D5D17F82430A84538BFA84613F02D
:10328800010F1AD0CDB965F3000307F8243023B233
:103298000122F71902935B2029462B4600920195DB
:1032A8000CF02EF97B78B878F9781843621C2B4615
:1032B8000095FEF755FF00E01A5501340436082C36
:1032C800CFD1054B83F80080BDE8FF8101130020B2
:1032D80034130020131300200013002010B50C4BEA
:1032E8001B78A3B10B4B1B788BB100240A482146ED
:1032F8001AF032FA40B1094821461AF02DFA18B9E5
:1033080020460121FFF754F80134402CEED110BDBE
:10331800E4120020DA100020E6140020D21B00205E
:103328002DE9F043364D374A2B8800266FF3861374
:103338006FF3C4032B80344B344F85B016701E7066
:103348009146984617F8013B5BB32A78D20052B2EF
:1033580043EAA2122B88402E62F3C40343F04003D1
:103368002B801ED000243046E1B2FFF7F7FEA8B14B
:1033780017F8013C13F0010F06D00122A24099F87A
:1033880000100A4389F8002013F0020F06D0012329
:10339800A34098F80020134388F800300134082C23
:1033A800E1D10136F6B2412ECCD12B7803F040049E
:1033B800E4B20CBB03F02403042B12D1FFF78EFFF9
:1033C800FF230093402021460122234601940294C2
:1033D8000CF096F880202146012223460094FEF73F
:1033E800BFFE2B8800226FF345136FF382036FF340
:1033F800C4032B80064B1A7005B0BDE8F08300BFEC
:10340800DC1400203C2C00206C2C002062130020CF
:10341800BF14002010B50024054821461AF09CF975
:1034280008B9044BE0540134402CF5D110BD00BF5D
:10343800B61400206213002070B516460D46317888
:1034480004469DF81020002925D0002B23D012B166
:1034580011491AF023F90121204609F031FE2046CE
:103468002946324609F004FEACB1082246F2A851BA
:103478000A480BF0E2FF214608481AF01AF90749F2
:10348800082246F2A8500BF0D2FF05480349BDE8D0
:1034980070401AF02FB970BD20200020F8120020CB
:1034A8005713002030B5064B04781D7824EA05042C
:1034B8000C7001781B7823EA0103137030BD00BF3C
:1034C8000113002038B50A4D002415F8013F2D2BB3
:1034D80009D0532B07D0542B05D0462B03D00548D1
:1034E80021461AF02EF90134402CEED138BD00BF28
:1034F800071F0020E614002010B50D481AF0C6F882
:1035080000240C4821461AF027F968B10A4BE31841
:1035180093F88030462B03D0542B01D02D2B03D1A8
:10352800034821461AF002F90134402CE9D110BDB4
:10353800A4130020E6140020881E0020094A0A4B24
:10354800117831B1997801F00F01814201D0002141
:1035580011709A7860F303029A705A7842F08002E8
:103568005A707047A3130020541300207FB55F4B97
:10357800154604461A780E4600235D4911F82310B3
:1035880011F0010F03D00121994022EA0102013311
:10359800082BF2D1574B1A70002C6FD014F0010F82
:1035A8000AD0FF2301210093FF3B0193029352208D
:1035B8000A460B460BF0A4FF14F0020F0AD0FF23B3
:1035C80001210093FF3B0193029353200A460B46C7
:1035D8000BF096FF14F0040F0AD0FF23012100938B
:1035E800FF3B0193029354200A460B460BF088FFD9
:1035F80014F0080F0AD0FF2301210093FF3B019329
:10360800029355200A460B460BF07AFF14F0100F70
:103618000AD0FF2301210093FF3B01930293562018
:103628000A460B460BF06CFF14F0200F0AD0FF235C
:1036380001210093FF3B0193029357200A460B4652
:103648000BF05EFF14F0400F0AD0FF230121009316
:10365800FF3B0193029358200A460B460BF050FF9C
:1036680014F0800F0AD0FF2301210093FF3B019340
:10367800029359200A460B460BF042FFCEB10024B4
:10368800284621461AF068F860B1FF230093FF3BF3
:103698000193631C1BB2012102935A200A460B4670
:1036A8000BF02EFF2146284601341AF04AF8402C28
:1036B800E6D110481049114AFFF7F4FE104B0022DA
:1036C8001A700132009206320192F83202920A49C7
:1036D8000A4A084809F07EFC0A4B3C2251201A701D
:1036E80004B0BDE870400CF089BA00BF0113002097
:1036F80013130020A41600200E1700200217002024
:10370800691600203313002010B5FFF72FFA04467E
:10371800074819F0F4FFD0F1010138BF002104B9BE
:1037280029B1034A2046BDE81040FFF71FBF10BD6E
:10373800F5130020054B03EBD00393F8903100F00C
:10374800070053FA00F000F001007047881E0020BF
:1037580010B50C4B04461B7813F001030FD0FFF78C
:103768001FFD68B10CF064F918B92046FFF7E2FFB5
:1037780030B10548214619F0D9FF012010BD18467F
:1037880010BD00BFDC140020F5130020024B187890
:10379800003818BF012070473313002010B5034CC0
:1037A80004EB830358709970DA7010BD131300206E
:1037B80010B5002409480021001908220834FCF734
:1037C800E9FDB4F5807FF5D1054A00231370054A59
:1037D800002199520233AA2BF9D110BDDC10002028
:1037E800D7100020821700207FB5444B04461B7871
:1037F8000E46AA2B75D04248214619F0ADFF054662
:1038080000286ED12046FFF7A3FF00286AD13D4863
:10381800214619F0A1FF50B93B48214619F09CFFF9
:10382800054620B92046FFF717FB00285AD1374B29
:103838001B7823B9364B1B7813F0010F09D1354B90
:10384800DB7803F02003DBB21BB9334B032283F888
:103858004020012E05D82B48214619F07DFF40B1A4
:103868003FE0022E07D12848214619F075FF10B114
:1038780037E0244800E02448214619F057FF27483C
:10388800214619F05EFF022E12D1012564194A2043
:10389800294603222B460096019502940BF030FE30
:1038A8000023182021462A460093FEF759FC19E008
:1038B800012E09D102230093631C02930196122062
:1038C80031460322334609E07EB9012102230093E1
:1038D800631802930191112003220B460BF010FE8E
:1038E80003E00025284604B070BD012000232118FC
:1038F800024600930125FEF733FCF3E7BE140020CF
:1039080057130020031300203E1500200113002048
:103918007E170020302A002062130020EE140020B9
:103928002DE9FF4704460D466148214619F014FF6A
:103938008046002840F0B88021465D4819F0F6FE20
:103948005C48214619F0FDFE5B4E0DBB012708F1CE
:103958000208E31902934246032039463B46CDF854
:10396800008001970BF0CCFD327862B10CF060F862
:10397800024630B1337840461E33009321462A462A
:1039880004E0009000E00092404621463B461CE0DF
:10399800012D1FD1631C022202930E2029462B46BB
:1039A800009201950BF0ACFD32788AB10CF040F82A
:1039B800024630B133780D201E330093214642462B
:1039C80002E000900D2021462B46FEF7C9FB50E08F
:1039D8000092F7E7022D0AD10121631802931420FF
:1039E8002A464346009501910BF08AFD41E0032DDC
:1039F8003FD101272A464FF0020904EB070A4D2060
:103A080039463B46CDF800900197CDF808A00BF059
:103A180077FD3578EDB10CF00BF8024630B133780C
:103A280048461E3300932146424602E00090214654
:103A380048463B46FEF794FB0BF0FAFF611C034631
:103A480020B133781A201E3300931FE000901A200B
:103A580020E021462A463B4648460095FEF780FB73
:103A68001A2051463A462B460095FEF779FB384610
:103A78001BE033789BB10BF0DBFF0346611C04F1BC
:103A88001C0033B10C4B1B781E330093012200231A
:103A980001E000930122FEF763FB012005E000939B
:103AA80004F11C00611CF5E7002004B0BDE8F087B4
:103AB800E6140020EE14002046150020064B1B18C3
:103AC80093F84001492804D0452814BF0320022058
:103AD80070470120704700BF881E00202DE9F04183
:103AE800244F00243C702448214619F035FEE5B2E5
:103AF800224B002837D01E5D3B789E4200D303B985
:103B08003E70002E30D131461C484022FCF742FC62
:103B18001B4B1C4803EBD50393F8888104F007037B
:103B280048FA03F8214608F0010819F015FE68B9AB
:103B3800B8F1000F02D02846022101E0284631469C
:103B4800FFF7EEFE28460CF059F80DE0B8F1000F2B
:103B58000AD12846FFF7B2FF0B4BDB7803F02003AE
:103B6800DBB20BB9094B18550134402CBBD1BDE869
:103B7800F08100BF4615002044130020FE140020E9
:103B8800881E0020E6140020302A0020621300203E
:103B98002DE9F04F914B89B01B7813F0010F06D037
:103BA8008F4B1A786FF386121A7001F09FBA8D49FD
:103BB8008D4A0B7810788D4D984218BF8C49137038
:103BC80018BF0B706B7803F00803DBB24BB143F6F8
:103BD800CF200BF021FC864B18702B886FF3CB237A
:103BE8002B80844B1B78AA2B08D18349AA3B0B70E6
:103BF8002B8843F080032B8000F0AFBE6A787B4BA4
:103C080002F01002D2B27D4CA2B11A886FF30C32C6
:103C18001A807B4B1B7823B97A4B1B7813F0010F62
:103C280008D1E37803F02003DBB21BB9764B0322FB
:103C380083F840202368754F6FF3186323603A7840
:103C480002F00202D2B232B96B494A781AB16B4A11
:103C580043F080731360E67816F0010648D05D20C3
:103C6800FFF728FA00285AD16B78DFF8808103F033
:103C78000203DBB22BBB5D30FFF7EEF8064600BB54
:103C8800B8F80030012143F40073A8F80030042389
:103C980003220093019302900B460D200BF030FC99
:103CA80045200BF0ABFF3146012233460D2000962C
:103CB800FEF756FA09203146324601230096FEF7F0
:103CC8004FFA6B7803F00203DBB243B34C4B1B781B
:103CD80023B94C4B1B7813F0010F20D1E37803F084
:103CE8002003DBB2DBB9484B032283F8402016E0FF
:103CF8006B7803F00203DBB26BB131463246012325
:103D08000A200096FEF72CFA8D2031460122334610
:103D18000096FEF725FA2B886FF349232B8023683A
:103D2800354A6FF35963236093787BB1D37823B90D
:103D38003B7813F00C0F05D108E03B7803F00C0337
:103D4800042B03D0236843F000732360E17801F06B
:103D58000201C9B200295BD05E20FFF7ABF9002849
:103D680065D16B78214F03F00403DBB2EBB95E3009
:103D7800FFF772F80646C0B93B88012143F4806317
:103D88003B800423009301330322019302900B46E6
:103D980017200BF0B5FB45200BF030FF0D20314606
:103DA800012233460096FEF7DBF96B7803F0040333
:103DB800DBB2002B3BD0124B1B7823B9114B1B787D
:103DC80013F0010F33D1E37803F02003DBB273BBA8
:103DD8000D4B032283F8402029E000BFA5160020E0
:103DE800E82C0020C8140020C9140020DC1400208E
:103DF80047150020BE140020180E0020302A00208D
:103E0800011300207E17002062130020861E002068
:103E18006B7803F00403DBB22BB18D2001220B4633
:103E28000091FEF79DF92B886FF38A232B80236876
:103E3800DFF8D0B26FF3DF7323605F2306930026A9
:103E4800D94696E03046394616F008F9002871D070
:103E58001BF80A30FF2B6DD04FF4A0727243A8F103
:103E68005E03DBB207930A2303FB072219F802E07B
:103E780009EB02035FEADE1E50D02268404642F09A
:103E8800004222600593FFF715F9059B00285CD1D5
:103E98001A7912F0040F24D14046FEF7DDFF059B86
:103EA8008446F0B91A79322042F004021A7107994F
:103EB800042300930291DB180121032201930B468E
:103EC800CDF814C00BF01CFB4A200BF097FEDDF870
:103ED80014C00C20079901226346CDF800C0FEF7F4
:103EE8003FF94FF4A07373430A2202FB07334B4494
:103EF8001B7913F0040F28D07D4B1B7823B97D4B19
:103F08001B7813F0010F20D1E37803F02003DBB214
:103F1800DBB9794B032283F8402016E01B7913F0B4
:103F2800040F07D08C20079901227346CDF800E0D2
:103F3800FEF716F94FF4A07373430A2202FB073306
:103F48004B441A796FF382021A71013708F101089C
:103F5800202F5FFA88F80AF10A0A7FF473AF069AED
:103F6800013602F12003DBB2022E0BF5A07B06938B
:103F780005D04FF0000ADDF81880574662E723683D
:103F88005E4923F080636FF39E7323600B79002BE7
:103F980000F05184DFF870A1DFF870B14FF09F088E
:103FA80000271AF8011F3E460137002950D0236820
:103FB800A8F15F0943F080635FFA89F923604846F6
:103FC800FFF778F8002859D14D4A122303FB06233E
:103FD800997811F0200F21D148460593FEF73CFF50
:103FE800059B8146D0B99A78012142F020029A7047
:103FF80004230093023301933BB2032202930F2060
:104008000B460BF07DFA45200BF0F8FD0D204946D4
:1040180001224B46CDF80090FEF7A2F8384912234A
:1040280003FB06139B7813F0200F27D0304B1B7827
:1040380023B9304B1B7813F0010F1FD1E37803F03D
:104048002003DBB2D3B92C4B032283F8402015E0C0
:104058002B4B122202FB06329278994612F0200F5F
:1040680005D08D2001220B460091FEF779F8122326
:1040780003FB06939A786FF345129A701BF8011F99
:10408800002945D02368404643F080432360FFF76A
:1040980011F8002852D11A4B4FF0120909FB0639C2
:1040A80099F8023013F0400F48D14046FEF7D4FE8D
:1040B8000646002842D199F80230012143F0400316
:1040C80089F8023004230093033301933BB203229F
:1040D80002934B200B460BF013FA50200BF08EFD89
:1040E80019203146012233460096FEF739F825E0BB
:1040F800011300207E17002062130020180E0020F4
:10410800A72B00204A2F0020982B00206C2B002082
:10411800A64B122202FB06329278994612F0400F03
:1041280005D0992001220B460091FEF719F81223B9
:1041380003FB0696B3786FF38613B37008F1010892
:10414800082F5FFA88F87FF42CAF994BDFF874B228
:1041580006934FF05008083F1BF8011F3E460137F1
:10416800002952D0236808F1610A43F080635FFA9E
:104178008AFA23605046FEF79DFF00285CD1330180
:10418800DFF844929B1B19F8032012F0400F23D14B
:1041980050460593FEF760FE059B8246E0B919F884
:1041A8000320012142F0400209F803200423009370
:1041B800023301933BB20322029369200B460BF0B2
:1041C8009FF945200BF01AFD0D2051460122534658
:1041D800CDF800A0FDF7C4FF33019B1B19F803308D
:1041E80013F0400F28D0734B1B7823B9724B1B7800
:1041F80013F0010F20D1E37803F02003DBB2DBB921
:104208006E4B032283F8402016E03301DFF8B891A3
:104218009B1B19F8033013F0400F05D08D200122A5
:104228000B460091FDF79CFF33019B1B19F80320F7
:104238006FF3861209F80320069A12F8011F0692F6
:10424800002935D02368404643F080432360FEF7B9
:1042580031FF002843D1DFF870A14FEA0619C6EBF9
:1042680009091AF8093013F0200F38D14046FEF733
:10427800F3FD064698BB1AF80930012143F02003E4
:104288000AF8093004230093033301933BB2032255
:10429800029310200B460BF033F950200BF0AEFCC4
:1042A80019203146012233460096FDF759FF16E0E2
:1042B8003301DFF814919B1B19F8033013F0200F1A
:1042C80005D0992001220B460091FDF749FF3301E3
:1042D8009E1B19F806306FF3451309F8063008F1EC
:1042E8000108072F5FFA88F87FF436AF344ADFF801
:1042F800DCB006924FF05708073F1BF8011F3E46F7
:104308000137002966D0236808F1560A43F0806314
:104318005FFA8AFA23605046FEF7CCFE002870D177
:104328003301DFF8AC909B1B19F8032012F0400F03
:1043380023D150460593FEF78FFD059B8246E0B9D1
:1043480019F80320012142F0400209F80320042350
:104358000093023301933BB20322029367200B467A
:104368000BF0CEF845200BF049FC0D2051460122F8
:104378005346CDF800A0FDF7F3FE33019B1B19F857
:10438800033013F0400F3CD00A4B1B7823B90A4B7B
:104398001B7813F0010F34D1E37803F02003DBB26C
:1043A8007BBB064B032283F840202AE0A72B002082
:1043B800332A0020011300207E17002062130020FA
:1043C8007B2A0020532B0020EB2A00206F2A002094
:1043D800982A00203301DFF864939B1B19F80330F7
:1043E80013F0400F05D08D2001220B460091FDF7F8
:1043F800B7FE33019B1B19F803206FF3861209F8E7
:104408000320069A12F8011F0692002935D0236866
:10441800404643F080432360FEF74CFE002843D11A
:10442800DFF818A34FEA0619C6EB09091AF809308C
:1044380013F0200F38D14046FEF70EFD064698BB14
:104448001AF80930012143F020030AF8093004233F
:104458000093033301933BB2032202931F200B46C0
:104468000BF04EF850200BF0C9FB19203146012201
:1044780033460096FDF774FE16E03301DFF8BC9270
:104488009B1B19F8033013F0200F05D09920012247
:104498000B460091FDF764FE33019E1B19F80630A8
:1044A8006FF3451309F8063008F10108042F5FFA85
:1044B80088F87FF422AF4FF000094FF0A70AC846EA
:1044C8004E46954B08F10108F15C00294ED023684F
:1044D800AAF14C0B43F080635FFA8BFB23605846CC
:1044E800FEF7E8FD002854D1162373438B4FFA5C7E
:1044F80012F0200F22D158460593FEF7ADFC059B1C
:104508008346D8B9FA5C012142F02002FA54042308
:104518000093023301930FFA88F3032202932020B9
:104528000B460AF0EDFF45200BF068FB0D205946BD
:1045380001225B46CDF800B0FDF712FE1623734347
:10454800FB5C13F0200F24D0754B1B7823B9754BF7
:104558001B7813F0010F1CD1E37803F02003DBB2C2
:10456800BBB9714B032283F8402012E01623734332
:104578006A4FFB5C13F0200F05D08D2001220B46FB
:104588000091FDF7EDFD16237343FA5C6FF34512B6
:10459800FA54664BF15C002936D02368504643F044
:1045A80080432360FEF786FD002842D15B4B4FF025
:1045B800160B0BFB063B9BF8013013F0200F38D18C
:1045C8005046FEF749FC0746002832D19BF80130D7
:1045D800012143F020038BF80130042300930333B7
:1045E80001930FFA88F3032202934C200B460AF03A
:1045F80087FF50200BF002FB1920394601223B4669
:104608000097FDF7ADFD14E0444F162303FB067336
:104618005B7813F0200F05D0992001220B460091FA
:10462800FDF79EFD162303FB06777B786FF3451392
:104638007B703F4B1B78002B00F094803D4B374F2D
:10464800F35C1622002B7BD002FB06F3FA5C07EB27
:104658000901C2F3801BBBF1000F1BD142F04002DD
:10466800FA54782204234A800093DB18012101932D
:104678000FFA88F3032202932E200B460AF040FF1C
:1046880046200BF0BBFACDF800B0092041460122C4
:104698005B4665E0B1F9021029BB5FEAD21B22D163
:1046A80043F6DE2005930AF0B7FE059BD8B1FA5C05
:1046B800012142F08002FA5404230093DB1801938D
:1046C8000FFA88F3032202932F200B460AF018FFF3
:1046D80047200BF093FA0920414601225B46CDF8AA
:1046E80000B0FDF73DFD16237343FB5CDB0939D0B1
:1046F8000B4B1B7823B90B4B1B7813F0010F31D1EF
:104708000D4BDB7803F02003DBB25BBB064B0322C7
:1047180083F8402026E000BF6A2B0020442A0020AE
:10472800011300207E170020621300205C2B00205C
:104738008C2A0020812A0020302A0020982A002074
:104748007243B95C11F0400F0CD063F3861163F328
:10475800C711B9544F447B808920009341460122F8
:10476800FDF7FEFC01360AF1010A022E09F11609CD
:104778005FFA8AFA7FF4A5AEDFF8D8A34827023E8D
:104788001AF8011FB0460136002937D02368384689
:1047980043F080432360FEF78DFC002847D14FF09B
:1047A8001C0909FB08F9DFF8A0B31BF8093013F05E
:1047B800200F3CD13846FEF74FFB8046002836D103
:1047C8001BF80930012143F020030BF809300423BA
:1047D80000930333019333B20322029313200B4651
:1047E8000AF08EFE50200BF009FA192041460122EA
:1047F8004346CDF80080FDF7B3FC18E01C2303FB0B
:1048080008F3DFF8449319F8033013F0200F05D0AC
:10481800992001220B460091FDF7A2FC1C2303FB03
:1048280008F819F808306FF3451309F8083001370C
:10483800082EFFB2A4D1A37803F00803DBB2002B43
:1048480040F08B8048F68E24A4F50A478E3FA9488D
:10485800394618F081FF28B9A748394618F07CFF77
:10486800002874D0A548394618F076FF00286ED184
:104878003946A24818F05AFF20460AF0CDFDA04E4E
:10488800C0B23070002862D00138C0B2307009F070
:104898003BFF00285BD130789A4E00F56A506E30A5
:1048A8000AF0BAFD984BC0B214F80380307000EAE1
:1048B800080839468F4818F04FFFDFF89CA2DFF848
:1048C8004C9238B18C48394618F046FF10B99AF81E
:1048D800003014E08848394618F03EFF38B1854862
:1048E800394618F039FF10B99AF8003004E09AF800
:1048F800003018EA030F02D023EA080801E048EA6A
:1049080003088248824989F80080824AFEF7CAFD76
:104918007F4881490FF09CFB68B10BF089F850B9CA
:104928007D4808F00FFC30B901237B487B49784A61
:104938000093FEF781FD0023009301330193337840
:10494800724802937249734A744B08F043FB01346E
:1049580048F6CE239C427FF477AF714E73786FF39D
:10496800C71373702B7803F08002D2B2002A00F0CC
:1049780011816C490C78002C40F00C8103F0240361
:10498800042B12D1FEF7AAFCFF23009340202146F6
:1049980001222346019402940AF0B2FD80202146A8
:1049A800012223460094FDF7DBFB2B8800246FF3DC
:1049B800C7136FF3820364F3451364F3410364F38D
:1049C8000003594A64F3492364F38A2314702B8043
:1049D800564B1A7842F0C0021A705A7864F3C30230
:1049E8005A70FEF76FFD524818F050FE514818F003
:1049F8004DFE514818F04AFE504821464122FBF727
:104A0800C9FC4F4B122202FB04339A78013402F09E
:104A1800BF026FF34512082C9A70F2D100231A01D5
:104A28004849D21A885C013300F0DF006FF3861022
:104A3800072B8854F3D1444B1A786FF345121A7038
:104A48001A7F6FF345121A7793F838206FF34512DF
:104A580083F8382093F854206FF3451283F85420D4
:104A680093F870206FF3451283F8702093F88C2028
:104A78006FF3451283F88C2093F8A8206FF3451242
:104A880083F8A82093F8C4206FF3451283F8C42054
:104A98002E4B1A7802F0DF026FF386121A70DA7B57
:104AA80002F0DF026FF38612DA739A7F02F0DF02F8
:104AB8006FF386129A7793F82D2002F0DF026FF3D6
:104AC800861283F82D20224B5A786FF345125A70BC
:104AD8001A7802F07F026FF345121A70DA7D6FF3CD
:104AE8004512DA759A7D02F07F026FF345129A75C6
:104AF800002345E06C1E0020741E00207C1E002050
:104B0800F4130020CE160020BA94FF1FA41600202C
:104B18000E170020021700200B1300206916002032
:104B280054130020180E0020BF140020E82C002089
:104B38003E150020031300204413002062130020B8
:104B4800A72B0020EB2A0020042D0020982A002003
:104B5800442A0020E22A0020011300204FF4A0710B
:104B680059430A2000FB021175480132411808799F
:104B7800202A6FF382000871F0D10133022B01D093
:104B88000022EBE708226F480021FBF703FC6E4B7D
:104B980000221A706D4F3878002843D12A786C4B60
:104BA80002F00202D2B2B2B16A4A517860F3C3018C
:104BB80051701A88CA3042F080021A8019F0BAFB84
:104BC800C62019F0B7FB19F003FC0BF0A3F8FEF7A9
:104BD80025F9FEF7EDFD604A2B8811786FF3410344
:104BE8006FF300016FF3000311705C48002140224D
:104BF8002B80FBF7CFFB5A4818F048FD594818F0AE
:104C080045FD594818F042FD584818F043FD082260
:104C18004C480021FBF7BEFB4B4A00231370544A53
:104C2800137067E02C7804F00203DBB293B914F038
:104C380001040FD14A4818F029FD3B78E0B223411E
:104C480013F0010F03D0FEF765FA0AF0E7FE01340E
:104C5800082CF2D12B783E4C13F0010F22D0FEF72E
:104C680053FD238843F002032380FEF7F5FA364B01
:104C78001F78A7B9CA2019F05DFBCD2019F05AFB9F
:104C880023883C4867F300032380334B1A7842F0AB
:104C980001021A7018F0FAFCFEF7C0F802E00120D1
:104CA800FEF74CFC2B7803F00202D2B212B3304A62
:104CB80012782AB113F0010F02D10220FEF73EFC50
:104CC800FEF70CFF2C49274818F0FEFC254926481A
:104CD80018F0E4FCFEF710FC2249284818F0DEFC26
:104CE8002749264818F0E5FCFEF794FB1F481D49A4
:104CF80018F000FD2348204918F0D0FC224A137808
:104D08000BB9FEF70DFB737803F08003DBB2002BC1
:104D180042D12B7803F02403042B06D143F6EC2070
:104D28000AF07AFB08B1062034E0FEF72FFD08B13F
:104D380005202FE00BF0C2F840B303202AE000BFA3
:104D48004A2F0020341300200013002001130020F4
:104D5800DC140020E82C002002130020FE140020A0
:104D6800CD230020B614002044130020F6140020A0
:104D780046150020F513002057130020E6140020E4
:104D8800A41300203C130020180E002001F03EF868
:104D980010B10420FEF7D2FB684B1B781BB1737867
:104DA8006FF3C713737066490B7813B1654B1B78A3
:104DB8000BB32B78644E03F04403402B1BD1002423
:104DC80021460122234620460094FDF7C9F9FF2316
:104DD80000933F20214602222346019402940AF0C0
:104DE8008FFB338843F6CE2043F0040333800AF068
:104DF80013FB564B1870524A554E13789BB1514BC2
:104E0800197881B92A78504B02F04002D2B252B1D7
:104E18001A8861F382021A80337823B943F6CE20C8
:104E28000AF0FAFA30702A78474902F00400C0B252
:104E3800484B002873D002F02000C0B2434C68B140
:104E48001A7842F0C0021A702378002B6BD10A88B6
:104E580063F3820263F345120A8064E0D20052B21F
:104E680019789211D2B241F0C00112F0010F1970F5
:104E780003D0C9B260F3C711197012F0020F03D042
:104E88001A786FF386121A701B78324A03F04003BF
:104E9800DBB21BB9537843F00803537043F6CD20B7
:104EA8000AF0BAFAC0B20128307002D1284B0222A7
:104EB8001A702478002C36D1FEF710FA2146012208
:104EC800234680200094FDF74BF9FF23012200932D
:104ED800402021462346019402940AF011FB2B88B6
:104EE80043F6CD2043F020032B800AF095FA174BA8
:104EF8001870194B1C70134B1A780AB1013A1A70C2
:104F0800197881B90E4A13786BB1FF2300934120B9
:104F180002220B46019102910AF0F2FA03E01A7894
:104F280042F0C0021A700AF079FF0C4818F0E7FB4B
:104F38000B4BB8B91A7860F3820216E0623400208D
:104F4800C814002047150020DC140020BF140020DE
:104F580061130020E82C0020180E0020AC1300205C
:104F6800021300201A7842F004021A706A78614825
:104F780012F001011A780CBF61F3410242F00202FB
:104F88001A705D4918F0B6FB5C495A4818F091FB55
:104F980058485B4918F08DFB3378012B40F0A68008
:104FA8002B8800246FF349236FF38A232B80554BFA
:104FB80021461C7041225448FBF7ECF9534818F07D
:104FC80065FBFEF77FFA4D4818F060FB4C4818F077
:104FD8005DFB4F4B122202FB04339A78013402F036
:104FE800BF026FF34512082C9A70F2D100231A0100
:104FF8004849D21A885C013300F0DF006FF386104D
:10500800072B8854F3D1444B1A786FF345121A7062
:105018001A7F6FF345121A7793F838206FF3451209
:1050280083F8382093F854206FF3451283F85420FE
:1050380093F870206FF3451283F8702093F88C2052
:105048006FF3451283F88C2093F8A8206FF345126C
:1050580083F8A82093F8C4206FF3451283F8C4207E
:105068002E4B1A7802F0DF026FF386121A70DA7B81
:1050780002F0DF026FF38612DA739A7F02F0DF0222
:105088006FF386129A7793F82D2002F0DF026FF300
:10509800861283F82D20224B5A786FF345125A70E6
:1050A8001A7802F07F026FF345121A70DA7D6FF3F7
:1050B8004512DA759A7D02F07F026FF345129A75F0
:1050C800002311E04FF4A07159430A2000FB02119C
:1050D8001448013241180879202A6FF382000871B8
:1050E800F0D10133022B01D00022EBE709B0BDE873
:1050F800F08F00BF2C270020E614002003130020A7
:105108003E15002061130020621300204413002084
:10511800A72B0020EB2A0020042D0020982A00202D
:10512800442A00204A2F00202DE9FF4104460D465D
:105138000AF09EFE9D4B1A1992F880709C4A984678
:105148001278AA2A0AD1A7F14F03DAB20B2A00F281
:10515800AE81984A5BB29A4040F1A981964B0C22E5
:1051680002FB04335A7A0833AA42C0F0A081FF2A0E
:1051780000F09D81FF229A7008EBD40393F88851C0
:1051880004F007031D41502F05F0010500F02881A8
:1051980014D8462F00F0F18009D8412F00F08F80F5
:1051A800452F00F01D812D2F40F07F8130E0482FE2
:1051B80000F0BD804F2F40F078810DE0542F5BD078
:1051C80005D8522F7BD0532F40F06F8118E0A7F1FC
:1051D8005903012B00F269817848214618F0BCFA7E
:1051E8000646002840F063815A2F01D174480AE12D
:1051F800592F03D07248214618F098FA714802E1F5
:105208007148214618F0A8FA0646002800F0568191
:105218006E48214618F0A0FA002840F0488121463F
:105228006A4818F083FA6A48214618F08AFA012673
:1052380002224DB1A4191420314600230092019690
:1052480002940AF05DF939E101340A20294633460F
:105258000092019602940AF053F9214632462B46F1
:1052680013200095FCF77CFF122029462A46334676
:105278000095FCF775FF21E15448214618F06CFAB7
:105288000546002840F0138101260222A7193E2076
:10529800314633460092019602970AF031F93946B1
:1052A80032462B4614200095FCF75AFF2146474802
:1052B80018F03CFA2146464818F043FAFEE0424806
:1052C800214618F049FA0646002800F0F7804148C0
:1052D800214618F041FA002840F0E9803B48214671
:1052E80018F03AFA064628B92046FDF7B5FD002819
:1052F80040F0E480002D40F09F802046FEF728FA19
:10530800002840F0D6802046FEF7D8FB324BDB78E9
:1053180003F02003DBB20BB9304B1855412F00F0D6
:105328009980522F40F0C1802046012194E02948FD
:10533800214618F011FA002840F0B9802348214688
:1053480018F00AFA28B92046FDF786FD002840F033
:10535800AE80002D70D12046FEF7FAF9002840F003
:10536800A8801D4BDB7803F02003DBB2002B71D142
:105378001A4B032283F840206CE01648214618F0A7
:10538800EBF9002840F093801048214618F0E4F922
:10539800064628B92046FDF75FFD002840F08E80BC
:1053A800002D49D12046032156E000BF881E002069
:1053B800BE140020000030805C2000207C1E0020ED
:1053C8006C1E0020741E0020B6140020E614002075
:1053D800EE14002057130020302A0020621300200A
:1053E8003848214618F0B8F90646002866D03648ED
:1053F800214618F0B1F90646002858D12046FDF795
:10540800E3FE20B13148214618F090F956E0502FBC
:1054180028D12F4B1B782BBB2046FDF7C1FE08BBBC
:105428002C48214618F098F9064620B92046FDF781
:1054380013FD002842D115B1204602210CE0204678
:10544800FEF73CFB244BDB7803F02003DBB20BB9FF
:10545800224B185520460021FEF762FA061E18BF97
:1054680001262BE02046FDF79BFE0546F8B91C48AF
:10547800214618F071F90646D8B92046FDF7ECFC2C
:105488000746D8B91648214618F050F9154A135D51
:105498008BB911494E7806F02006F6B26EB908EBC2
:1054A800040393F80031135508E0012606E00026AE
:1054B80004E02E4602E03E4600E01E46304604B0B8
:1054C800BDE8F081B614002057130020F513002022
:1054D80046150020E6140020302A00206213002020
:1054E80044130020FE140020032210B50549064885
:1054F800FBF726FA054806490222BDE81040FBF7EB
:105508001FBA00BF8E1C00200202002007020020E4
:105518008C1C002070B5804C237813F0010F0AD042
:105528000AF08EFA38B100207C4902F02BFD7C4B42
:105538007C48197849E07C4D2B78002B4AD00AF03A
:1055480085FA002846D0794B1B7873B9784B5B787D
:1055580013F0010F09D00AF06BFA30B9237803F081
:105568002403042B01D10330B6E0724C207870B1CB
:105578000020714902F006FD217801226F4802F0EF
:1055880027FD00201021621C07F0AAF902E06C49EF
:1055980002F0F8FC6B4C644807F0F0F92378002B14
:1055A80000F00A810AF04CFA002800F005816649EB
:1055B80066481022FBF7C4F964485B21FAF768FFD4
:1055C800002800F0F980217801308322BDE870407E
:1055D80002F0FEBC5E4C237803F00503012B5DD17D
:1055E80000205C4902F0CEFC202110225A48FAF72C
:1055F800D1FE601D59490322FBF74CF940BBE01C62
:1056080057490222FBF746F930B95648FBF712F919
:105618005449024650480BE0E01C53490222FBF76C
:1056280039F940B95148FBF705F9504902464A484B
:10563800FBF786F90EE0E01C4D490222FBF72AF938
:1056480030B94C48FBF7F6F84A4902464248EFE7BA
:10565800FFF74AFF6278303AD3B2092B00F2AC80E8
:105668003B4B9B78303BDBB2092B00F2A5800A212B
:1056780001FB0231C9B2002900F09E80334BFF22A2
:105688000C291A7740F2988010295A7740F29480B2
:1056980013299A7740F29080DA7770BD234E3378D9
:1056A800F3B9234B5B7813F0010F19D00AF0C0F956
:1056B800B0B9314818F023F868B1304C304B226843
:1056C80002EA03033BB914F00FF920B9E37803F0B9
:1056D8004003DBB223B10020BDE8704008F00EBCE7
:1056E800337863B90AF0A4F948B1264B1B7803F064
:1056F8000603042B03D02B780BB90120ECE7FEF747
:1057080045F810B10020204952E0204B1C78002CAD
:1057180040D01F494CE000BFDC140020D96A0208C1
:1057280000130020FE01002001130020CC160020E9
:105738007E17002089160020B048020803020020C6
:105748006E480208461500208F480208F201002022
:10575800891C0020B74D0208020200209CBC0208E8
:10576800A0BC02081A4E0208A3BC0208F94D0208A0
:10577800A6BC0208D84D0208AC130020302A00202D
:105788003000000F02130020DD5A02081D0E002011
:10579800D148020802F09AFB02F08CFB17F0B0FA2D
:1057A800064BDB7803F02003DBB22BB1044920461B
:1057B800BDE8704002F0E6BB70BD00BF302A002093
:1057C800C9470208054B1B78D8019B015BB2DB1166
:1057D80040B243EAE070C0B2704700BFDC1400205A
:1057E80070B50E4686B041000122054601F5E97103
:1057F80005A809F022FE0021012E8DF815104FF0A2
:10580800FF0205F1010305D10092019102930920DD
:10581800FB3A04E00092019102931E2004220B46F9
:1058280009F06EFE05A83F49FAF7B8FE50B105A881
:105838003D49FAF7B3FE28B105A83C49FAF7AEFE90
:1058480000286BD105A83949FAF7A8FE384B044659
:10585800C0B95A78214642F010025A70FF2302223A
:1058680000930190FE3B02903D2009F049FE4D2037
:105878000AF0C4F91220691C012223460094FCF79F
:105888006FFC03E05A786FF304125A700024294B16
:10589800E35C552B07D12846214611F08EFF10B145
:1058A800204611F079FF0134112CF0D1002E32D1AD
:1058B80021482249224AFDF7F5FD204821490EF0EA
:1058C800C7FBC0B10AF0B4F8A8B91E4807F03AFC03
:1058D80088B905A81349FAF761FE012320B9009396
:1058E80018481949154A04E016481749134A0093FD
:1058F8003346FDF7A1FD154B10491D700023009399
:1059080005330193124B0E4A1B780B4802930E4B3A
:1059180007F060FB02E00F4B00221A7005A806B0E2
:1059280070BD00BFD7BC0208A9BC020894BE02081B
:10593800E82C00203D2C0020A41600200E17002083
:10594800021700200B13002069160020E42D002008
:10595800CE1600203313002007B54100012201A80C
:1059680001F5E97109F069FD002301A804498DF8E2
:105978000530FAF713FED0F1010038BF00200EBD44
:10598800D7BC020807B54100012201A801F5E97159
:1059980009F053FD002301A804498DF80530FAF7F2
:1059A800FDFDD0F1010038BF00200EBD66BE020823
:1059B80070B5134B04461B1893F8805089B11148F1
:1059C800214617F0B3FEA5F15903DBB2012B0CD920
:1059D8004F2D0AD0542D08D021460B4817F0A6FEAB
:1059E80007E00848214617F0ACFE0748214617F0A3
:1059F800A8FE04480549BDE8704017F04FBE00BF37
:105A0800881E0020AC1300204C130020F614002040
:105A1800024B1878C0F38000704700BF02130020C3
:105A2800024B1A8860F308221A807047DC140020A1
:105A3800034B5878C00140B2C011C0B2704700BFD4
:105A4800DC140020014B1878704700BF01130020B8
:105A580030B5457800230021C218917055FA03F13A
:105A680011F0010F08D0064959188C7C017804EA16
:105A78000101A14208BF91700133042BEBD130BD65
:105A88008916002046F65221042209F0D6BC0000EF
:105A980070B5104C0546102220460021FAF77AFC12
:105AA800002004F8010C2A78103414F8011FC3B23E
:105AB80091420BD152B10849013301F8013B11223F
:105AC80046F6A243BDE8704002F09AB901300428B6
:105AD800EBD170BD8A160020891600202DE9F3410C
:105AE8002D4C0722E37848F6242702FB0030C0B289
:105AF80000F50A40453009F08FFC257964795FFA92
:105B080080F8002648FA06F313F0010F3AD0394618
:105B1800042201A809F091FC9DF804009DF80530C5
:105B28009DF806109DF8072000282BD0002929D0C1
:105B3800002B27D0002A25D0934204D19C4221D1A2
:105B480085421FD30FE09A4210D99C421AD394423F
:105B580018D89C4201D994421AD39C4201D185425B
:105B680016D294420ED18D420CD811E09C4201D13C
:105B780085420DD2944201D18D4209D99C4207D861
:105B8800944205D301360437082EBBD1002000E02B
:105B98000120BDE8FC8100BFD031002010B50446CB
:105BA800C00800F50A407D3009F036FC04F007040F
:105BB800C0B2204100F0010010BD70B5C50805F560
:105BC8000A457D35044628460E4609F025FC04F0B2
:105BD8000704C0B2012126B9A14040EA0101C9B2B7
:105BE80002E0A14020EA01012846BDE8704009F022
:105BF80009BC0000F0B57C4B95B0DE78082200EBBC
:105C0800C606F6B2F10001F5EC4104A8AC3109F082
:105C180014FC764B764C1A78002304A9C95C312908
:105C280005D13039994041EA0202D2B205E0302963
:105C380003D12F39994022EA01020133082BECD114
:105C480022706B486B496C4AFDF72CFC694B1B783A
:105C580013B9694B1B78F3B1664868490EF0F8F937
:105C680068B109F0E5FE50B9644807F06BFA30B93D
:105C78000123624862495F4A0093FDF7DDFB002378
:105C8800009302330193FD330293594859495A4A04
:105C98005B4B07F09FF906EB0611002501F5F04173
:105CA800257004A86C31112209F0C7FB2C462F4639
:105CB800544B0135E35C542B36D104AB1B5D312BBF
:105CC80003D1204611F070FC38B104AB1B5D302BBA
:105CD8002AD1204611F068FC30B34FB9FF23009356
:105CE8003420394604223B460197029709F008FC04
:105CF80004AF385D2146303811F064FC3B5D012764
:105D0800312B4FF0030305D100932BB20197029377
:105D1800352004E000932BB201970293362000212E
:105D280004220B4609F0ECFB0134112CC0D1B1015F
:105D380001F5F84104A82431402209F07EFB113C0A
:105D480004AD274615F8013BE6B20134302B03D1E8
:105D58003046FFF723FF38B115F8013C312B2CD121
:105D68003046FFF71BFF40B34FB9FF2300933420A1
:105D7800394604223B460197029709F0C1FB15F802
:105D8800011C30463039C9B2FFF717FF15F8013C3E
:105D98000021302B4FF0FF0305D1009323B201916E
:105DA8000293372004E0009323B201910293382034
:105DB80004220B4609F0A4FB0127402CC2D1124D46
:105DC8006B7803F00403DBB263B1403C2046FFF775
:105DD800E5FE38B90134E4B2402CF7D16B7860F3B2
:105DE80082036B7015B0F0BDD03100200113002084
:105DF800A41600200E170020021700200B13002005
:105E0800691600203D2C0020E82C0020014B187852
:105E1800704700BF1D0E00202DE9F04F4A4B0022AD
:105E28001A704A4A85B01678002E40F08A80484B8E
:105E38004FF4B468DA78997808FB02F24FF03C081E
:105E480008FB01285A78434F90441FFA88F8BA464D
:105E580065E03AF815303C24DAB2544304EB1324D5
:105E68004C44A4B2042CEEB207D842F25A739845B7
:105E780003D904F51C546034A4B2444511D948F63A
:105E8800442009F0C9FAC8EB0403834209DC324B09
:105E98001A787B1993F87030934302D02A4901236A
:105EA8000B702B4AD378B3422BD142F26073B4FB08
:105EB800F3F203FB12439BB243451CD1274B9B785B
:105EC80013F0090F3DD1264B5B7803F02003DBB2BA
:105ED800002B36D1234B1A781BEA020F11D10199F6
:105EE800009841EA02021A70FFF7F8FD48B90098D5
:105EF800FFF780FE05E01B4B02991A7801EA0202BF
:105F08001A70013509F5B469072D1FFA89F9A0D16E
:105F1800039E07370136082E0AF10E0A11D04FF0FA
:105F2800010B0BFA06FB5FFA8BF301936FEA0B0385
:105F3800F2B2DBB24FF00009009202934D4603968D
:105F480087E705B0BDE8F08F1D0E00204915002039
:105F5800D03100204A15002001130020302A0020EB
:105F6800F62C00204815002073B50C4601EBC00143
:105F7800C9B2C90001F5EC41054608226846AC31B2
:105F880009F05BFA104B002003EBC402121B5219F4
:105F980082F870001DF80020312A0AD101218140C1
:105FA80003EBC402121B521992F87060314382F855
:105FB800701001300828EDD169463122302317F0DE
:105FC800D3FBC0B27CBD00BF4A15002000B501EB71
:105FD800C001C9B2890191B001F5F84124314022CC
:105FE800684609F02AFA402069463122302317F022
:105FF800BBFBC0B211B000BD7FB501EBC001C9B297
:1060080001EB011101F5F0416C31112201A809F0F1
:1060180014FA112001A93122302317F0A5FBC0B2D0
:1060280007B000BD2DE9F843002634462BE0214691
:106038002846FFF799FF214681462846FFF7C6FF05
:10604800214640EA09092846FFF7D6FF5FFA89F991
:1060580049EA000010F0FF0F05D0404639460222F9
:1060680009F0EBF903E04FF0FF33A8F800300135F1
:10607800EDB20237072D08F10208D8D10134E4B295
:106088000E3E082C07D0054BC6F5EC47C6EB0308B7
:106098003C370025CBE7BDE8F88300BF4A15002050
:1060A80010B518F0C9FB4FF4803018F0E5FB18F074
:1060B800FDFC0128044628D1102018F0DFFA022040
:1060C80018F0D0FA002018F017FC002018F028FC6F
:1060D8004FF4806018F01AFC4FF4404018F02AFC86
:1060E8004FF480304FF4E01118F0E2FB204618F02E
:1060F800EBFB392018F0C6FC0028FAD0022018F073
:10610800E9FB18F0F1FB0828FBD17C20012118F0ED
:1061180083FC46F60120012118F07EFC0C48012181
:1061280018F086FC0B48012118F082FC042001219C
:1061380018F07EFC7E2018F0A5FC38B118F0CCFCD5
:10614800054B04211A7861F344021A7010BD00BF90
:1061580003400600000808184534002010B50C4616
:10616800014620B110220C48FAF7EAFB04E00A487D
:1061780020211022FAF70EF934B1084821461022DE
:10618800BDE81040FAF7DCBB044820211022BDE826
:106198001040FAF7FFB800BFF20100200202002009
:1061A80010B5FF2B1446029A03D0421802F8013C9E
:1061B80008E06FF07F439A4204D01314437013121F
:1061C8008370C27015F07CFD02E07F2018F0A0FFFC
:1061D80015F062FD0028F8D1ACB10B4890F82010FA
:1061E800163001F00F0115F06BFD02E07F2018F06A
:1061F8008FFF15F051FD0028F8D1044B93F8693052
:1062080013F0010FE9D110BD4C0C002060330020C1
:1062180010B50A4B002203EBC003013B10460849A6
:1062280051184C7813F8011F8C4205D10130C0B2C7
:106238000C320828F3D1F73010BD00BFE2F1010895
:106248005C20002070B50D4C05460E464FF4807258
:1062580000212046FAF79EF82A46314604F5807058
:10626800F9F7F0FF642004F8025C16F0A7FF00239A
:1062780084F8F131024B64221A6070BDC8340020E2
:10628800941C002010B5054C002120464FF4807264
:10629800FAF780F8002384F8F13110BDC8340020E3
:1062A800164B2DE9F0415D8A07462846FBF738FC76
:1062B8001349FBF741FD134B134E1860D723B5FB69
:1062C800F3F5EDB2822229460446F01901F080FE6A
:1062D8002846FBF729FC01462046FBF76FFB0B49D4
:1062E800FBF776FCFBF73AFE0337BE19C1B28122F1
:1062F8003046BDE8F04101F06BBE00BF9823002096
:1063080000005743F4150020F2010020000020414E
:1063180070B54B4D2868FBF70FF845A3D3E9002368
:10632800FAF7AAFEFBF7F6FAFBF706F842A3D3E959
:106338000023FBF755F83EA3D3E90023FBF77AF9CE
:10634800FBF7E8FAFAF7F8FFFAF702FEFBF7E2FACA
:106358003C4906462860FBF7E3FD20B13046FBF7D1
:10636800FDFDC4B25EE030463649FBF7EDFD50B1A5
:1063780030463549FBF7D4FD28B13046FBF7EEFD32
:10638800C0B2441C4EE030462F49FBF7DDFD50B14A
:1063980030462E49FBF7C4FD28B13046FBF7DEFD39
:1063A800C0B2841C3EE030462849FBF7CDFD50B111
:1063B80030462749FBF7B4FD28B13046FBF7CEFD40
:1063C800C0B2C41C2EE030462149FBF7BDFD50B1D8
:1063D80030462049FBF7A4FD28B13046FBF7BEFD47
:1063E800C0B2041D1EE030461A49FBF7ADFD50B19E
:1063F80030461949FBF794FD28B13046FBF7AEFD4E
:10640800C0B2441D0EE030461349FBF79DFD48B16C
:1064180030461249FBF784FD20B13046FBF79EFD5C
:10642800C0B2841D0A202146BDE8704008F0EABFCA
:10643800736891ED7CFF7F400000000080842E414E
:10644800F8150020000010410000F041000048420B
:1064580000008E420000B8420000E0420000F24214
:106468002DE9F04F9DB015F0C1FB092016F0D2FFC1
:1064780016F028FE4FF4614017F008F8092017F0CD
:1064880085F80022A3484FF4804118F05CF9A2482F
:10649800002118F025FDA14904224B78DFF8A0E27D
:1064A8006FF300034B709E4B9E4C1A705A709A7093
:1064B800DA701A715A719A71DA719B4B033A1A7031
:1064C8009A4B00201F328EF8000020705A700590F9
:1064D8000546069006467F2018F01AFE23780E2BF4
:1064E80001F2B281DFE813F00F004F009500E000E1
:1064F8007902DE0330048504E806DA07ED0756085A
:10650800AF08CE087E098A4E8A48317801F00F011B
:10651800013149014118FFF721FE337813F00F03C9
:1065280008D1854A92F80123012A41F08D81834AD6
:10653800138024E0012B03D17F4B93F819330BE030
:10654800022B04D17C4B93F80D33032B05E0032B6E
:1065580006D1794B93F80D33012B41F075810EE08C
:10656800774901220A7077484FF4007118F0EBF868
:10657800754BC8221A6033786FF30303BFE333788F
:106588005A1C01F05DB8704B1A6822B96D484FF477
:10659800007118F0D8F8DFF898816C4898F8001066
:1065A80001F00F01013149014118FFF7D7FD36B15C
:1065B80098F800305A1C62F3030388F800305F4BE8
:1065C80000221A8098F8001001F00F02022A03D165
:1065D8001A7842F010020AE0042A03D11A7842F02D
:1065E800040204E0052A05D11A7842F040021A7024
:1065F80001F02AB9062A04D14D4B6FF30301197033
:106608007EE301F00F01012212FA01F1198001F075
:106618001BB9474E4E48317801F00F01013149014D
:106628004118FFF79BFD96F8008008F00F08B8F1B5
:10663800070F27DC18F0010F464B02D000205880C6
:1066480002E04FF0FF3159804FEA6809062209F14C
:10665800010902FB09394FF0FF32A9F80220404630
:10666800FFF7D6FDFF2806D03B4B03EB400058232D
:10667800437401F0E9B80023A9F8023008F10108D1
:1066880001F088B80021102213A8F9F783FE0FA89B
:1066980000211022F9F77EFE237801332370337826
:1066A8006FF3030301F079B8DFF884A09AF800804B
:1066B80018F00F0840F03F81284E337803F040036C
:1066C800DBB2F3B926486FF07F43817A0122009349
:1066D80001F00F01FF23FFF763FD224B93F86920B8
:1066E80012F0400F08D093F86C3013F0040F03D069
:1066F800337843F0400333707378142262F3C7038E
:106708007370737813F0F80F30D0174800F1200138
:10671800A5E300BF00180140002C0140BA23002067
:10672800881E0020FE1500201B0E0020A72B00202D
:10673800FD15002022F201085C200020E82C002032
:10674800C41C0020000C0140941C0020C2F2010867
:10675800A2F301086E2C0020F20100201D2A00205F
:106768004C0C002060330020C2F40108BC4B1B789D
:1067780003F04003DBB2002B00F0D980DFF804837C
:10678800DFF8049398F8003013F00C0B30D1B54EB5
:106798006FF07F4396F82B1006F12100009301F06B
:1067A8000F0101220523FFF7FBFC96F84C104FF46C
:1067B800860A06F1420001F00F010122FF23CDF8FD
:1067C80000A0FFF7EDFC96F84110FF2306F1370013
:1067D80001F00F015A46CDF800A0FFF7E1FC0423B1
:1067E80089F8003098F8003043F0080301F02AB81F
:1067F80003F00803DBB2002B39D099F800A0BAF1F6
:10680800000F03D0984800F1400138E0954E6FF032
:106818007F4B717D06F10B0001F00F010122FF2370
:10682800CDF800B0FFF7BCFC96F82B1006F121005C
:1068380001F00F0101220723CDF800B0FFF7B0FCEB
:1068480096F836104FF48603009306F12C00FF23C8
:1068580001F00F015246FFF7A3FC98F800306AF3E5
:10686800C303DBB243F0040388F800305AE099F818
:1068780000C0BCF1000F08D07B4800F16001FFF7B1
:106888006DFC99F80020303208E2764E6FF07F40B8
:10689800717DFF23009001F00F0106F10B0001222A
:1068A800CDF80CC0FFF77CFC9AF80030DFF8C4B1D3
:1068B80003F0100A5FFA8AFADDF80CC0BAF1000F8B
:1068C8000CD098F800206CF3820288F800205A1C3B
:1068D80062F303038BF8003000F0B6BF96F82B1074
:1068E8006FF07F42009206F1210001F00F010122B2
:1068F8000C23FFF755FC96F836104FF486030093E7
:106908005246FF2306F12C0001F00F01FFF748FC67
:106918009BF8003083F01002C2F3001262F30413F4
:106928008BF80030042389F8003000F08DBF4E4802
:1069380000F1800193E2B8F1010F3CD14A4800F11F
:10694800A001FFF70BFC002E00F07E879AF80030BC
:10695800444E5A1C62F303038AF8003096F82B1051
:106968006FF07F4906F1210042460F2301F00F0125
:10697800CDF80090FFF714FC96F82B1006F12100D3
:1069880042460E2301F00F01CDF80090FFF708FCF6
:1069980096F82B1006F12100424601F00F010F2353
:1069A800CDF80090FFF7FCFB30488021424617F0F5
:1069B800CAFE00F049BF2C4800F1C001FFF7CEFB2A
:1069C800002E00F041872A4B96221A609AF8003070
:1069D8006FF303038AF8003092E1264E317811F004
:1069E8000F0A16D1244800F12001FFF7B7FB204B0E
:1069F8001B68002B40F0288713A8F9F71BFF4022DB
:106A08001346014613A801F007F93378012200F074
:106A180017BEBAF1010F39D112486FF07F4390F8D1
:106A2800201000220093163001F00F01FF23FFF71A
:106A3800B7FB01F05BF9002800F0068733780222E3
:106A480062F3030333700D4B1A7842F080021A7018
:106A58000B4B5A7842F002025A7000F0F5BE00BFA4
:106A68001D2A00204C0C0020C2F40108001001402F
:106A7800941C0020FD150020A2F50108222A002000
:106A8800702E0020843900200B3B002001F00F01FC
:106A980001F10E0303F00F03012B44D89B48490171
:106AA8004118FFF75BFB9A486FF07F4390F820107E
:106AB80000221630009301F00F01FF23FFF770FB4F
:106AC80016F0B8F9337803F00F03022B13D112F044
:106AD800DFFE002800F0B8868E4B1A7842F040029C
:106AE8006FF304121A705A786FF345125A7033789C
:106AF800032200F0A5BD12F0B5FE78B112F060FFD8
:106B080012F02CFE844B00201A7858816FF3C712BC
:106B18001A703378042262F3030333707F4B1A78B8
:106B28006FF3000263E5BAF1040F4DD1DFF8DC9191
:106B38004901DFF8108249444846FFF70FFB98F8EF
:106B48000010774B01F00402D2B27AB941F0040187
:106B58006F4883F800A088F8001090F836104FF4BA
:106B6800860300932C3001F00F01ECE293F800A0AB
:106B7800BAF1000F40F0688665486FF07F45417DA7
:106B880001220B3001F00F01FF230095FFF708FBEE
:106B980064480122817AFF2301F00F010095FFF775
:106BA800FFFA98F8003005226AF3820388F800306B
:106BB8003378484662F30303337009F1A001FFF705
:106BC800CDFA554600F040BEDFF84481FF2398F81F
:106BD800201000226FF07F4908F1160001F00F0124
:106BE800CDF80090FFF7DCFA2BB2072B18D13378D9
:106BF80008F121006FF30303337023780122013376
:106C0800237098F82B100E2301F00F01CDF8009097
:106C1800FFF7C6FA44488021002217F094FD0025AA
:106C2800424E96F86B3013F0040F00F00D8698F87A
:106C380057106FF07F43002200933D48FF2301F077
:106C48000F01FFF7ADFA96F86B303A4A03F00F03DD
:106C5800012B137003D1002D08BF01250CE0022B76
:106C680004D12BB2012B08BF032505E0032B03D168
:106C78002BB2032B08BF0725ABB213F0010F02D0CC
:106C88002D4A3121517713F0020F02D02A4A3221BE
:106C9800917713F0040F00F0D7853322264BDA776B
:106CA80000F0D2BD1948254E00F1C001FFF756FA91
:106CB80096F80090DFF85C8019F00F090CD112F0FB
:106CC80067FC98F8003069F3000388F800303378DF
:106CD8005A1C62F30303337012F0ECFC98F800308E
:106CE80013F0010F00F0B08500221548802117F03D
:106CF8002AFD0A4B00225A70337862F3030333707B
:106D080023780133237000F09FBD00BFA2F501086E
:106D18004C0C0020702E0020222A0020EC2D002090
:106D28000B3B0020010000200010014060330020D0
:106D3800990C00201C2A0020F2010020FD150020DB
:106D480000180140843900208548864E00F1E00192
:106D5800FFF704FA0FA8F9F76DFD0FA9024682485C
:106D6800F9F7EEFD00218148B18090F8C5106FF069
:106D78007F4300220093BB30FF2301F00F01FFF790
:106D88000FFA7B4A92F86B1092F86C30327843EA2B
:106D9800012312F0010FB38010D0A3F1EB0292B2DD
:106DA8000A2A04D9A3F5E6739BB2282B02D8F388E4
:106DB8000133F38033786FF3000333707378002B5B
:106DC80040F04285674AD2887AB16A4A1BA811788E
:106DD80063F30301117022788DF86F30013222704D
:106DE80028228DF86C2017F0CDFC0022F28000F0EC
:106DF8002BBD614EDFF8A8A1337803F00408B8F181
:106E0800000F15D109A841461522F9F7C3FA5B4BC3
:106E1800CAF800801B684546CDF8273033684746D6
:106E280043F004033360564B83F8F98100F00CBD3E
:106E380003F08003DBB2002B67D1DAF800100029D9
:106E480040F002854F48FFF789F94F484FF48051C9
:106E580017F06FFC012806D04A4800F1A001FFF79F
:106E68007DF900F0F1BC464991F8F921002A43D098
:106E780008314648013AF9F763FD444B03F1100124
:106E880013F8012B0D2A01D00A2A02D1202203F877
:106E9800012C8B42F4D13E4B4FF03C0808FB0738DD
:106EA80008F11E084046F9F7C5FC41460246394834
:106EB800F9F7F0FCD8B9022F03D1336843F0100377
:106EC80004E0032F03D1336843F040033360327882
:106ED80053005BB203EAC263DB173268DBB263F3C9
:106EE800C71232601BB1FFF7CDF900F0ADBC013716
:106EF800FFB2042F08BF0227254B3C2606FB0736A6
:106F08003046F9F797FC314626E0DAF80080B8F108
:106F1800000F40F09984737803F02002D2B2002A5F
:106F280040D11D4B09A81A889B781C498DF826303A
:106F3800ADF82420F9F788FA114B1B7A302B07D1CA
:106F4800FFF7A0F9336843F40053336000F07CBCCA
:106F580009A8F9F76FFC09A9FFF774F900F074BCE8
:106F6800A2F50108EC2D0020060200204C0C0020A0
:106F780060330020FD150020981C0020ABBC0208DF
:106F8800C0340020A2F601080008014002020020D7
:106F98000C000020C8340020B0BC0208B4BC0208B1
:106FA800941C002003F04003DBB2002B40F08980E2
:106FB800B14800F16001FFF7D1F8B048F9F73AFCA1
:106FC8008046AE49AE484246F9F764FC002873D1C2
:106FD800AC4B43441B7A302B6ED1FFF753F933681F
:106FE800DFF8D09243F48043336099F82B106FF0A8
:106FF8007F43009309F12100082301F00F010122CA
:10700800FFF7CEF86423CAF800307F2018F080F824
:10701800DAF80030002BF8D1984699F88E10D6335C
:10702800994E89F886304B3B6FF07F4A89F8873054
:10703800964801F00F0142467433CDF800A0FFF7DF
:10704800AFF896F8B91106F5D670033001F00F01C4
:107058004246FF23CDF800A0FFF7A2F896F8C41126
:1070680006F5DD7001F00F014246FF23CDF800A0C0
:10707800FFF796F896F8CF1106F5E270013001F0A7
:107088000F014246FF23CDF800A0FFF789F896F8D4
:10709800DA1106F5E87001F00F014246FF23CDF83A
:1070A80000A0FFF77DF899F899107948CDF800A06D
:1070B80001F00F01424646E07648F9F7BBFB7549F7
:1070C8004AE796F802B0DFF8EC910BF0020B5FFA92
:1070D8008BFBBBF1000F3AD199F82010FF236FF01A
:1070E8007F4809F1160001F00F015A46CDF80080DB
:1070F800FFF756F8684B93F86B3003F00803DBB2E0
:10710800002B00F0A18399F82B10012209F121002E
:1071180001F00F010323CDF80080FFF741F8336831
:10712800554843F4003300F180013360FFF716F847
:1071380055485A4690F8E51100F5EC70CDF80080F6
:10714800033001F00F01FF23FFF72AF87CE3CAF8A8
:10715800008099F820106FF07F4300934246FF2388
:1071680009F1160001F00F01FFF71AF82AB241F2EF
:1071780011139A421DD1434B1B7A302B13D1FFF7C1
:1071880081F83368454668F3514368F38E3368F3F2
:107198004D333360414B1A7868F303021A70237831
:1071A8000133237050E33E48F9F744FB3C49FFF7AD
:1071B80049F8394E96F86B3013F0040F00F0448309
:1071C80025B9384820211022F9F7E4F87F2017F074
:1071D8009FFF99F857106FF07F43002200933248C1
:1071E800FF2301F00F01FEF7DBFF96F86B202F4B12
:1071F80002F00F020D2A1A7005D125B92C4A412137
:1072080091754FF480551A78062A08D12AB2B2F53A
:10721800805F04D1264A3621D1754FF488551A78F3
:10722800082A08D12AB2B2F5885F04D1204A382149
:10723800117641F210151B780B2B09D12AB241F2B5
:1072480010139A4204D11A4B2A225A7641F2111588
:107258000D486FF07F4390F8F0110022009300F57D
:10726800F370FF2301F00F01FEF79AFF96F86B30D9
:1072780013F0010FAAD0E7E2A2F601081A010020D4
:10728800C8340020C034002001000020D00C0020A9
:10729800DB0C0020FC00002060330020FD150020DE
:1072A8003801002002020020990C00201C2A00202E
:1072B800F20100204C0C0020A34B1A7842B30022A4
:1072C8001A700F20FAF7C0FE06460A20FAF7BCFE2D
:1072D8009E4B9F4958824A7812F0010F18D06436A5
:1072E800301A58839B4B1A78642A01D19B321A7042
:1072F8001B78984EFF2B0BD00A21B3FBF1F1964B6C
:1073080023311980954817F0EBFD3378013333703A
:10731800DFF8648298F8003013F00F0612D18E4B14
:1073280023228B481A804378232143F001034370BA
:107338008A4817F0D5FD8A4800F12001FEF70EFFB4
:1073480004967AE2012E68D1804B5A8BA2F169012A
:1073580089B2112908D8049911F0010F04D141F01C
:107368000101C9B204910592049A12F0020F0DD1DD
:107378005B8A7C4A1380A3F5AE630B3B9BB2D72B89
:1073880004D8049840F00203DBB204931B20FEF7F4
:1073980087FF0599744B0AB2632A05DD642192FBC5
:1073A800F1F230321A7401E0092A0CDD059A11B2A3
:1073B800642291FBF2F002FB10120A2012B292FB37
:1073C800F0F230325A74059802B2642092FBF0F160
:1073D80000FB11210A2209B291FBF2F002FB101204
:1073E80030329A745B4B1B78FF2B08D158495B48A5
:1073F8004B786FF300034B70002117F071FD049A6E
:10740800032A40F021825248002143786FF3000399
:107418004370524817F064FD0FE2022E03D1534B1C
:10742800C8221A6009E2032E16D1504B1B68002BA4
:1074380040F00A824A4800F14001FEF78FFE1B2007
:10744800FEF72EFF414B5B8AA3F51E630F3B9BB2F1
:10745800542B00F2F981F0E1042E0CD13B4B988AB1
:107468000CF0ECF9002840F0EF813D4800F1600194
:10747800FEF774FEE1E1052E07D1344B988A0CF033
:10748800DDF9032840F0E081D7E1062E40F0D581F0
:1074980022786FF3030301322270D3E1344800F1FC
:1074A8002001FEF75BFE334B1B78002B00F0CC81EC
:1074B800237801332370304B1A786FF30302FFF7F8
:1074C80096B82D4EDFF8A480337813F00F021AD146
:1074D8002A4800F12001FEF741FE2948F9F7AAF9E8
:1074E800274902462748F8F7ADFE2548F9F7A2F9DB
:1074F800254BA3F8160233785A1C62F30303337042
:1075080016F06EF891E0012A16D1D8F80030002B59
:1075180040F09A8116F090F8012840F095811B48B8
:10752800F9F788F9194902461948F9F7B3F9002813
:1075380040F08A8111486FE0D8F80020002A40F016
:1075480083810B217BE000BF1E0E002098230020C2
:10755800BA2300200C160020480C0020002C014003
:1075680062F7010800160020F2010020941C002098
:10757800E2F70108FC150020FD15002022F801089B
:10758800740100200B2800202437002092010020DD
:1075980025370020864E337813F00F080CD1854824
:1075A8004146FEF7DBFD33785A1C62F30303337060
:1075B800814BA3F8028047E1B8F1010F18D17F4849
:1075C800042117F0B6F8002800F03E81794800F150
:1075D8002001FEF7C3FD33784FF0FF315A1C62F3E8
:1075E80003033370764B64221A60734B59802BE186
:1075F800B8F1020FDFF8C8811BD1D8F80030002B92
:1076080040F022816D48042117F093F8002840F0DB
:107618001B81694B5880674800F14001FEF79EFDC9
:1076280033785A1C62F3030333706423C8F80030BC
:107638000AE1D8F80020002A40F006810C212170C8
:1076480062F30303A9E05F4910234FF40052CB70A3
:107658000D3B8B700A805C4817F01CF80A22002149
:107668005A48F8F797FE802016F078FF2378013300
:1076780023704F4B1A786FF303021A70504BC822CD
:107688001A60E1E05248DFF844A100F12001FEF75A
:1076980065FD9AF80030002B00F0D6804D48DAF8E6
:1076A8000020434E0260BAF8042082809AF806202F
:1076B8008271317811F00F0159D1DFF80481D8F8BF
:1076C8000010002940F0C0809AF80410A2F5A652D4
:1076D8004FF0640B103A0BFB01229AF805004FF0AB
:1076E8000A0909FB00200393FAF71AFA3A49FAF74C
:1076F80023FB02469AF80200039BA0F5A650103817
:107708000BFB030B9AF80100344B09FB00B018601F
:107718000392FAF705FA039A01461046FAF750F968
:107728002F4B1860F9F708FE1DA3D3E90023824602
:107738008B46FAF7DBF8002800F086805046594659
:1077480019A3D3E90023FAF7C7F800287CD0FEF77D
:10775800DFFD337848465A1C62F303033370C823AD
:10776800C8F8003007F058FEC0B207906CE0012955
:107778006AD10D300799832200F02AFC104BD3F808
:107788000080B8F1000F5FD1404616F0E7FE23787D
:1077980001332370337868F30303337054E000BF78
:1077A800736891ED7CFF7F400AD7A3703D0080404D
:1077B800FD15002082F801086E2C0020000C014005
:1077C800941C0020B623002000100140141600204D
:1077D800E2F801080202002000007A441016002096
:1077E800F81500208448854E00F12001FEF7B6FC0C
:1077F800F37913F0010F27D0DFF8488298F800904A
:1078080019F00F0920D17E4B0A22597818781039BF
:1078180002FB0011B1701979D878103902FB0011F8
:107828007170D9799B79103902FB0312327013F009
:1078380047FBF37969F30003F37198F800305A1C99
:1078480062F3030388F80030DFF8FC9199F80060D0
:1078580016F001063EF43FAE6A4B01221A7014F08E
:107868009BFF2378092B01D00D2B28D101206649D5
:107878000EF05AFC654B664A5B7803F01F03D35C35
:10788800644A522B137002D1634B01221A70634B66
:10789800634A03F1200153F8040B8B4242F8040BAE
:1078A800F9D1002117A80EF05BFC17A80D2115F0DF
:1078B80033FE5C4B1A78013202F003021A7099F811
:1078C800006006F00206F6B2002E00F08B800CF085
:1078D80011FA0FF001FE06980322431C93FBF2F203
:1078E80002EB42029B1ADBB20693002B79D1DFF838
:1078F800488198F84960C246002E4DD0022E03D127
:1079080098F80130312B49D023780E2B13D14648F3
:1079180046490522F8F7BEFF8246002840D1B21F2B
:1079280037484349F9F70CF8344B5646DA7942F0B0
:107938000102DA7135E00D2B03D13E483A4907229E
:1079480027E0032B22D13C4B002713F8012F2C2AC8
:1079580003D00137FFB2B742F7D113A832493A46EC
:10796800F8F7EEFF7B1C07E00AEB03025278303A87
:10797800D2B2092A03D80133DBB2B342F4D30AEBFB
:107988000701FA430FA80231D21802E0264909A8D4
:10799800721EF8F7D5FF03E0069E02E0012600E01C
:1079A80000261E4B204A03F1100153F8040B8B42AA
:1079B80042F8040BF9D1214B214A03F1100153F885
:1079C800040B8B4242F8040BF9D1402388F811309C
:1079D8001C3B88F82230023B88F84B3015F094FBAA
:1079E80000E0002699F8003003F0F5036FF3000378
:1079F80089F80030FEF76FBD22F90108D031002068
:107A0800021600201E0E0020C1360020C0360020BD
:107A18008C280208DC2A0020FC150020F201002036
:107A2800792B00203B2A00206F340020B7BC0208C5
:107A380074340020141600206E3400200202002046
:107A480080340020FD15002048340020AFF300806A
:107A5800084B187800F00400C0B250B11A6822F040
:107A680004026FF341021A60034B00221A70034BA1
:107A780018787047302A0020381600202016002079
:107A8800084B1B7813F0010F0AD1074B1B783BB149
:107A9800064B1B6823B9064A136843F002031360B8
:107AA800704700BF39160020381600203416002011
:107AB800302A0020064B00211970064B06481A6828
:107AC80022F0020261F382021A601222F8F762BC05
:107AD80038160020302A00202016002038B5094C1E
:107AE800094922780546F8F7ADFB23780021E954C7
:107AF800064B1A6822F0040261F341021A602078EA
:107B080038BD00BF3816002020160020302A00207B
:107B18000D4B1B7813F0010F14D10C490C4A0818AF
:107B2800137810F8010C0B49112BC85401D80133F4
:107B38001370094B4FF496721A60084A136843F0A1
:107B480004031360704700BF3916002062F901086A
:107B5800381600202016002034160020302A002075
:107B680070B5294C002384F8293084F8283014F89B
:107B7800103094F82A2003F00F0363F3030284F80B
:107B88002A202A2604EB4000417873431F4D61F3F5
:107B9800071284F82A20628CE95A1D48E28417F0FB
:107BA8009DF994F82A301A4803F00F0306FB035393
:107BB8005988013989B217F095F901210A46144804
:107BC80017F05CF90121124817F049F994F82A30A6
:107BD80010481B097343E95A17F080F994F82A30C2
:107BE8000C481B0906FB03556988013989B217F04F
:107BF80077F901210A46074817F040F9054801219D
:107C0800BDE8704017F02BB93A1600206EF901084C
:107C1800000800400034014030B5164C94F82B5051
:107C2800A38445F00105002384F82B50628484F86E
:107C3800211084F8203019E0C55CA5F13002D2B2D9
:107C4800092A08D9A5F14102D2B2052A9ABFA5F19D
:107C58003702D2B22A46084D013305EB420292F8A8
:107C6800515192F85021257062700234DAB28A427A
:107C7800E2D330BD3A1600206EF90108124B10B558
:107C88009A8C0024DA8483F8294083F82840224615
:107C980001210E4817F0F2F864210C4817F01EF97C
:107CA80032210A4817F01EF901212246084817F028
:107CB800E5F86421064817F011F905483221BDE8B6
:107CC800104017F00DB900BF3A1600200008004018
:107CD8000034014010B500212C220348F8F75AFB64
:107CE800BDE81040FFF7CABF3A16002070B5204C17
:107CF8002378042B37D8DFE803F0030D152A30006A
:107D08001C4B012093F82B3013F0010F2ED020705C
:107D1800013870BD174B93F82000FFF721FF0223AD
:107D2800237020E0134DEE8CEEB9FFF7A7FF95F80E
:107D3800203095F821200133DBB29A4285F82030B3
:107D480001D8042300E003232370304670BD094B9B
:107D5800D88C50B90123237070BDFFF7BBFF0023F7
:107D68002370012070BD002070BD002070BD00BFD1
:107D7800661600203A160020202102480A46F8F725
:107D880009BB00BFF201002038B5044608460D467D
:107D9800F8F750FD98B10319202B094BC8BFC4F15F
:107DA80020001C19002308E014F8012BE02A14BF56
:107DB800EA5C202204F8012C01338342F4DB38BD4D
:107DC800F20100200D4B46F612221B689B68934275
:107DD8000FD043F6EE2293420BD0122B09D0B3F505
:107DE800E97F08D046F6B6201B1A584240EB03003C
:107DF8007047012070470120704700BFA01600207F
:107E0800F0B51F4687B006460C46084600211546C1
:107E1800F8F7C0FA244B07B19F80B3F9041005A8FE
:107E280001EB8601042207F008FB002605AB9B5DE9
:107E3800013BDBB2B92B34D81D2B4FEA031208D80B
:107E4800D31803F514416846EE31112207F0F5FA0C
:107E58000BE01649D3185B186A4603F11007186837
:107E680059680833BB4203C2F9D12046F8F7E2FC4F
:107E7800C7B26846F8F7DEFC3818A84203D8E019FC
:107E88006946F8F779FC6846F8F7D4FC7B1C1B18A0
:107E9800AB4203D8E0190649F8F7D6FA0136042EA2
:107EA800C4D107B0F0BD00BF10170020FF9E020824
:107EB800CBBC020810B5044C002120466C22F8F710
:107EC80069FA0123A37010BD10170020044B00228B
:107ED8005A701A709A7842F001029A70704700BF7F
:107EE800101700202DE9F843244C8046A3780D464E
:107EF80013F0010F3FD06FF30003A37015F0DCF807
:107F08006378002B37D123780BB90A336370A378D1
:107F18001B4F6FF30003A37015F0CEF8217807EB21
:107F280008066118073130462A46F8F709FD304639
:107F3800F8F780FCC6B2AE42DFF840900FD80CD2FA
:107F4800002306EB080089F8003038180A3320218E
:107F5800AA1B89F80130F8F71DFAAE420BD1217837
:107F6800064B6418227A1AB101311970BDE8F883FA
:107F78001A700A225A70BDE8F88300BF1017002053
:107F8800F2010020054B1A780AB100221A701B78FA
:107F980045F6551202FB0311FFF7F6BE86160020C0
:107FA800F8B505460C460818002107F02BFA013CE5
:107FB800E4B26719384607F02FFAC6B2202E03D864
:107FC8003846002107F01EFA0CB1202EEFD9F8BD73
:107FD80002F00F03032B22F07F0230B5D2B20CD986
:107FE8004FF47A7491FBF4F42025E4B2057002B1E1
:107FF80014B13034047000220130B1F57A7F05DB0A
:108008004FF47A7491FBF4F504FB1511022B0BD98C
:10801800642491FBF4F42025E4B2057002B114B194
:108028003034047000220130632904DD642491FB9C
:10803800F4F504FB1511012B0AD90A2391FBF3F37C
:108048002024DBB2047002B10BB13033037001306D
:10805800092904DD0A2391FBF3F203FB12113031E5
:10806800017030BD13B5104B01461B689A899C7B83
:1080780012F0100214BF0220012034B10B4C9B7C7B
:108088002478634303FB001109B23AB10DF10600ED
:10809800022207F0D2F9BDF8060002E0084607F010
:1080A800BBF900B21CBD00BFA0160020C1160020FD
:1080B80010B50F4B1B689A899C7B12F0100214BFF5
:1080C8000221012134B10B4C9B7C2478634303FBD0
:1080D800010000B22AB108490222BDE8104007F0A9
:1080E800A6B9054B1968BDE8104007F08BB900BF69
:1080F800A0160020C1160020D81600203038C0B2C3
:10810800092894BFFF20002070470000044B1A780C
:108118006FF300021A70034B00221A70704700BFF9
:10812800011700208316002070B58B4CFFF7EEFF77
:108138002578264605F0F005202D6BD107F078FC50
:10814800002867D1854B1B783BB92378C3F303120A
:10815800013262F30713237070BD814B1B7803F063
:108168008003DBB2002B51D07E48F8F763FBC4B222
:10817800C4B17D4E7D4930462A46F8F7E1FB0A2C0A
:108188000BD8224630467749F8F7DAFB30192946EA
:10819800C4F10A02F8F7FEF804E0304671490A22F1
:1081A800F8F7CEFB704C042204F10C00A521F8F777
:1081B800F1F86F4B1A7852B1FF23012A237306D9BD
:1081C800022A637303D0032AA37318BFE373694CAD
:1081D80094F8A33013B96848684902E0664804F186
:1081E800A3010622F8F7ACFB654B1B78452B40F042
:1081F8006281237813F00C0F40F05D81022243F076
:10820800100362F301035B4A137070BD56485D4961
:108218002A4645E1347804F0F004102C3FD107F0E9
:1082280007FC00283BD1202257494F48F8F788FB24
:108238004D4855492246F8F783FB544B1B7813F0F9
:10824800010F06D05248F8F7F5FA5149024651484D
:1082580005E05148F8F7EEFA4F4902464D48F8F75D
:108268006FFB3E4B1B781BB94C484D49102217E158
:108278004A484C491022F8F763FB394B1B7803F046
:108288008003DBB22BB14248F8F7D4FA02464648DD
:108298004FE04148F8F7CEFA0246434842E03378C7
:1082A80003F0F003302B46D107F0C2FB002842D17F
:1082B8002D4C20223D492046F8F742FBA5210522F6
:1082C80004F10B00F8F766F8394B1B78042B02D938
:1082D800FF23E37300E002D1FF23A37301E0032B24
:1082E80002D1FF23637301E0022B02D1FF23237322
:1082F80000E00BB1FF23E3722E4B5B7813F0600FA5
:1083080005D03F23E37223736373A373E3732A4B8C
:108318001B7803F02003DBB233B11F48F8F78AFA61
:10832800024626481C49BBE01948F8F783FA02467A
:1083380022481749B4E0337813F0F00344D12022DF
:108348001F490948F8F7FCFA1E4B07481988832289
:10835800BDE87040FFF73CBE01170020C41C002098
:10836800981C00209C1C0020F2010020D06D0208FF
:10837800911D0020CC1C00200C0200203B4E02085E
:10838800681600208E6D0208309B0208702E0020AF
:108398009B9C0208FF010020BC9C020802020020EE
:1083A800DCA00208519B02080F020020E04E0208E0
:1083B800871E0020C0230020302A00200D02002044
:1083C8007D4E020880160020502B1ED107F030FB8E
:1083D800D8B9394920223948F8F7B2FA3848F8F7B5
:1083E80029FA374902463748F8F7AAFA3648F8F71B
:1083F80021FA354902463548F8F7A2FA3448F8F721
:1084080019FA3349024633484AE0337803F0F00357
:10841800102B06D107F00CFB18B128482E49202252
:108428003EE0337803F0F002402A3DD123482B493F
:10843800203AF8F785FA2A4B1B781BB3294B1C788E
:1084480034B92948F8F7F6F92749024627481FE0C2
:10845800022C06D12648F8F7EDF9254902462348AB
:1084680016E02448F8F7E6F9224902461F48F8F7CB
:1084780067FA012C0ED12048F8F7DCF91E490246AC
:108488001E480DE01E48F8F7D5F91D490246174861
:10849800F8F756FA1B48F8F7CDF91A490246174873
:1084A800BDE87040F8F74CBA174A6FF3071313701A
:1084B800164B00221A6070BD5C4E0208F2010020C3
:1084C8005C470208F6010020664702080602002001
:1084D800614702080D020020BF4E0208729B020885
:1084E8001B2A002029270020BC9C0208FB01002031
:1084F800D59B02089B9C0208939B02080B02002054
:10850800DD9C0208B49B020801170020A016002079
:10851800204B70B5F022204D1A702B7813F0010F04
:108528000BD01E4C207810F0010006D11C49FFF733
:1085380029FD237843F0010323701A4E3378532B17
:108548000ED1164C237813F0010F07D000201649DE
:10855800FFF718FD23786FF300032370FFF7D6FDAC
:108568003378232B14D10D4B1B7813F0010F0FD147
:10857800FFF7CCFD2B780D4A43F006032B701378D8
:10858800013BDBB213700A4A52F82320094B1A60E8
:1085980070BD00BF0D17002001170020A516002090
:1085A8000992020868160020E8910208EF160020D8
:1085B800F0160020A01600202DE9F0415D4BF022B6
:1085C8005D4D1A702A7802F01003DBB2002B2DD112
:1085D8005A4963F347120B601C462A70584A9A5C42
:1085E8002D2A01D00134E4B20133112BF6D1554EB6
:1085F8003A213046F7F74CFF38B1801BC0B2013042
:10860800301821460222FFF7E3FC4F4B1B78452B1D
:1086180040F08D800024204601340EF0B5FF112C67
:10862800F9D12B7843F010032B703AE0474C2378AC
:1086380013F0010F16D1414EFFF73CFC414F316852
:10864800384601310222FFF7C3FC2D23BB70307876
:1086580046F63E433E496522FFF7D2FB237843F0B6
:108668000103237003200D21FFF73CFC2D78324EC7
:1086780015F0E00545D110203649FFF783FC324B51
:108688001B78442B11D12D4A136801331121B3FBF8
:10869800F1F101EB01115B1A2949C95C2D29F4D0CC
:1086A8001360BDE8F041FFF731BD532B0DD132788F
:1086B8004E3B63F347123270204A2749126806205E
:1086C80000FB02125380BDE8F081232B2FD11B4BF6
:1086D8001D60337803F0EF0365F347133370FFF73A
:1086E80015FD23781D4A43F0060323701378013BD8
:1086F800DBB213701A4A52F823201A4B1A60BDE8ED
:10870800F081104C10201849FFF73CFC04F11000D0
:108718002821F7F7BDFE50B1001B3178C0B20130F7
:10872800201849098022BDE8F041FFF751BCBDE897
:10873800F08100BF0D170020A5160020D8160020D4
:108748003D2C0020F20100206816002001170020AF
:1087580017170020859102086E2C0020EF160020C4
:10876800F0160020A0160020A6910208434B2DE920
:10877800F041F022424E1A703378424D43F0010323
:1087880033702B68404C9B7C33B9404B1B7803F00B
:108798004003DBB22BB10DE0012B0BD111F0BCF87B
:1087A80040B907F0B7FA236800206FF355532360E8
:1087B800374943E0A778DFF8D08007F02003DFB21D
:1087C800B7B907F0A7FA2968324B897C1A78384676
:1087D80061F301021A70D8F800302D4943F40013F0
:1087E800C8F80030FFF7CEFB2B4B802283F84320DC
:1087F8000AF0D4FB804678B12B689B7C012B08D10A
:10880800264B5B7803F01003DBB213B10020244938
:1088180014E00020234911E00AF0F0FB074610B1EC
:10882800404621490AE00AF031FC10B138461F4998
:1088380004E0194B93F8433013B91D49FFF7A2FB25
:108848001C4B1B78232B16D1FFF760FC337843F0C1
:108858000603337007F05EFA23686FF355532360FD
:1088680009F00EFC144A1378013BDBB21370134A6B
:1088780052F823302B60BDE8F08100BF0D170020AF
:1088880001170020A0160020302A0020981C002084
:108898002A920208762E0020351A0020702E002019
:1088A8006C9202084B920208AE9202088D9202085E
:1088B800CF92020868160020EF160020F01600205C
:1088C800614B2DE9F341F022604E1A703378604D08
:1088D80043F0010333702B685E4C9B7C8BB95E4B75
:1088E8001B7803F04003DBB283B15C4B1B7803F0C9
:1088F8000403DBB2ABB1A37803F04003DBB22BB1C6
:108908000FE0012B0DD111F007F850B9F9F7D8FB9A
:108918002368002023F480036FF3D7532360504962
:1089280064E0A778DFF82C8107F04003DFB22FBBA3
:10893800F9F7C6FB29684B4B897C1A78384661F3EE
:1089480001021A70D8F80030454943F4800367F3F0
:10895800D753C8F80030FFF715FB2B68198A21B9DF
:108968000091082001220B4606E00BB2012B05D12D
:1089780000970E2039463A46F9F7F2FB0AF00EFB4B
:10898800074678B12B689B7C012B08D1364B5B7866
:1089980003F01003DBB213B10020344926E00020B5
:1089A800334923E0F9F778FCFF2809D1A07800F0D3
:1089B8008000C0B210B138462E4917E02E4915E0A4
:1089C8000AF01CFB804660B1F9F756FEC0B20228D7
:1089D80002D83846294909E0062809D838462849DE
:1089E80004E00AF053FB18B126494046FFF7CAFADB
:1089F800254B1B78232B23D1FFF788FB337843F0D3
:108A080006033370F9F75CFB2368204A23F48003DC
:108A18006FF3D75323601378013BDBB213701C4A02
:108A280052F823302B600F4B1B7813F0030F02D141
:108A38000AF08AFA20B102B0BDE8F04109F020BB83
:108A480002B0BDE8F08100BF0D170020011700201B
:108A5800A0160020302A0020981C0020CC1C0020E2
:108A68002A920208762E0020702E00206C920208AE
:108A78004B9202083293020853930208F0920208BC
:108A8800119302088D92020868160020EF16002044
:108A9800F016002010B5FFF739FB124B2522DA77C4
:108AA800114B124C1B6816219A7C01FB024251782B
:108AB80001F00F000F2814D00A2803DD0A2060F304
:108AC800030151709B7C162202FB034463780A2140
:108AD80003F00F03594306486D32BDE81040FFF715
:108AE80077BA10BDF2010020A0160020442A002009
:108AF8000E0200202DE9F74F984BDFF8B0A2F022C4
:108B08001A70DAF80030D0469C6847F27803E11A08
:108B18004C4244EB0104DA3A6243914B9D5C9F1846
:108B2800C5F30005EEB29946002E29D130468D498D
:108B3800FFF728FA8C4B1B78232B40F035857B7880
:108B480066F304137B70FFF7E1FA884B1A7842F05A
:108B580006021A70864A1378013BDBB21370854A05
:108B680052F82330CAF80030834B1D70834B1D70B8
:108B7800834B1D70834B1E60834B1D7000F014BD2A
:108B8800824E814D337893B1814A4FF4A0711378A6
:108B980003F01F005B0959430A2303FB00137D49B7
:108BA800CB18DB78002B40F06682137084E06E4BA4
:108BB8001B78532B40F0FC8095F80080B8F1000F2B
:108BC8002ED14046214611F084FC5FFA80FABAF1B2
:108BD800000F25D07B7868F304137B706E4F3A78CA
:108BE8001AB9204611F08CFB13E0531E6B49002B79
:108BF800184603EA0101B8BF02F11E00401100291E
:108C080003DA013961F01F01013111F0C5FB0023BE
:108C18003B7011F0F1FC85F800A00022594BE2E00E
:108C28002B78002B00F0278256490A680F460B2A3A
:108C380001D10C2316E00C2A11D1013B6101544AE1
:108C480059181170554903EA0101002903DA01395D
:108C580061F01F010131204611F09EFB1CE0092A3A
:108C680002D10A230B60D0E10A2A27D14B49013BE4
:108C780003EA0101002903DA013961F01F0101311A
:108C8800204611F0CBFB2B786201D318DBB2404AA7
:108C9800591E1170404A13704FF00008C7F8008041
:108CA800FFF734FA162303FB04935A7842F01002B4
:108CB8005A7085F8008014233370DCE1043A042AE2
:108CC8003FD83749D2B20878364F60B300200870D1
:108CD800397841B13448401810F8010C032802D003
:108CE800002840F0C881013B0A2058434FF4A07E79
:108CF8000EFB0400DFF89CE07044801841716001AD
:108D08001B18D8B200EB800000F5E840FC30801852
:108D180006F078FB387818B1013811F0D5FCAAE1D3
:108D28000BF094F8A7E101200870013B0A214B439E
:108D38004FF4A07101FB04331649CB189A185379E4
:108D48000AE00F4F3B7823B901223A700A4A1370A0
:108D580091E1FFF7DBF900233B708CE10D17002050
:108D6800442A0020485C02086816002001170020E9
:108D7800EF160020F016002088160020AE160020FE
:108D8800C1160020D8160020CB1600207E16002021
:108D9800C21600204A2F00207D1700201F000080E7
:108DA800D71600207C170020881E0020A01600205F
:108DB800432B1AD1964A1278002A40F043812B7827
:108DC800002B00F05881934B1A78002A40F0538109
:108DD800914B19680C2903D00A2903D02A7014E191
:108DE8000B2200E009221A600FE1232B7ED1884A6A
:108DF8001278002A40F026812978DFF818A2002985
:108E080035D09AF8003053B184490F2B0A70844941
:108E18000A7000F2308101338AF800302BE17E4A73
:108E28001368082B1ED84FF4A077674301394FF019
:108E38000A0E0EFB01717B4F181F7918C978062797
:108E4800013907FB0101784800EB810151F8040F53
:108E58000133002840F0D880032B40F2D580082B3E
:108E6800F4D9D1E0092B40F006810233CCE07B78BD
:108E78006E4E61F304137B7032781AB9204611F0F4
:108E88003FFA13E0531E6A49002B184603EA010112
:108E9800B8BF02F11E004011002903DA013961F060
:108EA8001F01013111F078FA0023337011F0A4FB8F
:108EB8000AF0CCFFFFF72AF95E4B1A7842F0060257
:108EC8001A705D4A1378013BDBB213705B4A52F8A3
:108ED8002330524AC8F8003000231370504A8AF8E9
:108EE800003013704C4A2B7013605DE32A2B3CD181
:108EF800474A1278002A40F0A58046490B784BB1C2
:108F08004648012B02704648027040F2B480013B8B
:108F18000B70B0E02878002800F0AD803E4A136856
:108F2800002B00F0A880092B1AD84FF4A0716143D8
:108F380001384FF00A0E0EFB00103A491F1F08189F
:108F4800C1780620013900FB0171374800EB810127
:108F580051F8040D013B002856D1032BF8D853E0F3
:108F68000B2B40F08880023B4EE0442B1AD1284A54
:108F78001278002A66D1274B1B78002B7BD12878E2
:108F8800431EDBB21E2B76D8214611F0A2FAC0B2DE
:108F9800002870D0204A13680C2B6CD00A2B6AD09A
:108FA80028701BE0552B4DD1194A1278002A49D157
:108FB800184B1B78002B5ED1287801285BD9023822
:108FC800214611F097FAC0B2002854D0124A13680B
:108FD8000C2B50D00A2B4ED019490870043B042B97
:108FE80013D84FF4A071614301380A2707FB00101A
:108FF8000C490818C1780620013900FB01330A49D9
:1090080051F823300BB904331360FFF77FF832E0CF
:10901800D7160020C1160020D81600208816002078
:10902800AE1600204A2F0020400D00207D1700209A
:109038001F00008001170020EF160020F016002006
:10904800CB160020303BDBB2092B14D89B4A1268A0
:10905800043A042A0FD89A4A117861B9994A1278C1
:109068004AB1994A0A27107807FB0033DBB2402B34
:10907800137088BF11702F78DFF8B082002F5FD18E
:1090880098F8000010F0010012D114B920468F4959
:1090980000E08F49FEF776FF98F8003043F6DF20AE
:1090A80043F0010388F8003006F0B6F9894B1870D0
:1090B800337813B98848894901E0874888490A22E2
:1090C800F7F73EFC204611F0F3F9864D01460222DF
:1090D80005F11900FEF77CFF834B1B7803F0800332
:1090E800DBB22BB3814B1B88EB81337803BB804BFE
:1090F80018781A4618B9204611F0CEF818E07D4BBA
:10910800411E01EA0303002B03DA013B63F01F034E
:1091180001334FF4A07161430A2505FB0313764917
:10912800CB18DB7813B911F095F901E0002313701F
:10913800162303FB0494637843F01003637033E24F
:109148004FF4A0736343013F0A2202FB07336A4EC0
:10915800F31893F803B06301FF1898F80030FFB2D2
:1091680013F0010F45D1FEF7A5FE07EB071101F536
:10917800E0417C311022614806F05FF9604B5948A4
:1091880011229A7144230370173BC370791C013074
:109198000F3AFEF71DFF494B1B6813B910205949B8
:1091A8001FE0012B02D1102057491AE0022B02D1EF
:1091B8001020564915E0092B02D11020544910E01F
:1091C8000A2B02D1102053490BE00B2B02D110209F
:1091D800514906E00C2B02D11020504901E05049BA
:1091E8001620FEF7CFFE98F8003043F0010388F808
:1091F8000030334B1A789846002A00F0EA8007EBD3
:10920800071707F5E0477C3710223648394606F03D
:1092180014F900229146334B995C9A4641B109F101
:1092280001095FFA89F90132B9F1100FF3D106E0AB
:1092380003EB09002021C2F11002F7F7ABF898F808
:10924800000048450BD90138C01906F0E5F830B9D7
:109258001B4B202118780138C01906F0D3F8DFF825
:10926800D09099F8003018460193FEF747FF4A4618
:10927800019BDFF8C09018B9432B40F0848001E0CF
:10928800432B04D1002389F80030202172E0DFF855
:10929800A8E024499EF800C023489C454ED10B788D
:1092A800ACF1300C0133DBB24FF00A0E0B700EFB41
:1092B8000C33C35C002B53D10B7051E0D81600203F
:1092C800C1160020D71600207C170020AB5C0208CE
:1092D8002F5D02085B2B0020F8010020715D020859
:1092E800925D0208F2010020302A0020CABC020860
:1092F8007D1700201F0000804A2F0020171700202C
:10930800101700209A5E0208795E0208BB5E020808
:10931800605F0208815F0208A25F0208C35F02085B
:10932800E45F0208AE160020E0FA010801170020E9
:109338006816002088160020851600208EF8003058
:1093480099F800304FF0000C81F800C043B198F84C
:1093580000300F2B04D803F1010E954B83F800E081
:10936800402389F8003013780978303B0A2202FB41
:109378000313C15C98F8000001380AF80010381887
:1093880006F040F80EE08B4B1B7803F08003DBB24D
:1093980043B199F800302BB998F80030FF225344B4
:1093A80003F8012C99F8003013B1834A013B13707C
:1093B80099F80030012B10D198F800300F2B02D803
:1093C8007B4A013313707D4A002389F800301370FB
:1093D80003E004200C21FEF785FD794B1F681FBBB5
:1093E8004FF4A07254432B780A22013B02FB03443A
:1093F800361975782D090F2D00F0D680714CA521EE
:1094080004F11C00063AF6F7C5FFFF232377002D69
:1094180000F0CA80012D637700F0C680022DA37783
:1094280000F0C280E377BFE0012F18D14FF4A0729B
:1094380054432B780A21013B01FB03443619737806
:1094480003F00F030F2B00F0AF80092B04DC01336E
:109458005D485943BD3AA2E05B4859436AE0022F90
:1094680038D10BF1FF3B5FFA8BFBBBF1070F98BFBD
:10947800564BDFF850819CBF5B4493F8647008F149
:109488001B0088BF002720210522F6F783FF2878D4
:10949800C7EB08080138002318E04FF4A0726243B4
:1094A8000A2101FB0022B25C08EB07011A4112F005
:1094B800010FC7F1000202D08A18DB2101E08A18E7
:1094C800A52182F82010013308F10108DAB2BA4266
:1094D800E3D369E0032F2FD14FF4A07254432B78C4
:1094E8000A25013B05FB0343F218F35C13F0400F18
:1094F80002D01020364906E093785A1ED2B2FD2ACF
:1095080006D93449102003B0BDE8F04FFEF73ABD44
:10951800FE2B02D110203049F5E710202F49FEF725
:1095280031FD2F4B2F481B78013B05FB03442E4D83
:109538002C19A178832232E0043F042F34D8062264
:10954800FFB20BF1FF3B02FB0B7B284B284853F87B
:109558002B100A31F7F7F4F9264B1B7893B1154B0A
:109568001B7803F08003DBB23BB1234820210222A1
:1095780003B0BDE8F04FF6F70DBF204B1E48197831
:1095880082220CE02B780A22013B53434FF4A0724D
:1095980002FB04343619F71917487979BE3A03B033
:1095A800BDE8F04FFEF714BD03B0BDE8F08F00BF73
:1095B800C1160020302A002088160020AE16002090
:1095C800D8160020F20100200D020020E0FA010860
:1095D8001E5F0208DC5E0208FD5E02083F5F0208AB
:1095E800CB1600200F0200204A2F0020400D00203B
:1095F80002020020D7160020100200207C1700204D
:109608002DE9F0474C4C4D4F2378F02243F00103ED
:1096180023704B4BDFF85C911A703B68494A9E688F
:1096280047F27803F01A464246EB000616217143CA
:10963800555C5318C5F300055FFA85F89246B8F1F2
:10964800000F23D140464049FEF79CFC99F80030B2
:10965800232B6FD1FEF75AFD23783C4A43F00603CB
:1096680023701378013BDBB21370394A52F8233068
:109678003B60384B1D70384B1D70384B1D70384B94
:10968800C3F80080374B1D70BDE8F08799F80020BB
:10969800232A23D15A786FF304125A7010F0ACFFC2
:1096A8000AF0D4FBFEF732FD2378284A43F006037C
:1096B80023701378013BDBB21370254A52F823302C
:1096C800244A3B6000231370234A1370234A137003
:1096D800234A1360234A1370BDE8F087532A0DD13B
:1096E8005A78C2F300144CB942F010025A7021465D
:1096F8003046013410F050FE202CF8D1304610F0DE
:10970800D7FE162303FB06A67378C1B213F0100F19
:109718000AD0202902D10020134901E01349002072
:10972800BDE8F047FEF72EBC11480222BDE8F0471D
:10973800FEF74EBCBDE8F08701170020A0160020F8
:109748000D170020442A0020485C0208EF1600206C
:10975800F016002088160020AE160020C116002042
:10976800D8160020CB160020219502084295020841
:109778000B020020681600202DE9F0412D4E2E4FD7
:10978800307800F5E0405A3005F046FE3B78C4B228
:1097980013F0010F26D0294D2B78552B0AD1EC2C2C
:1097A80001D0013CE4B23078214600F5E0405A305F
:1097B80005F028FE2B78442B0DD1A4F11403DBB25D
:1097C800D72B01D90134E4B23078214600F5E040C6
:1097D8005A3005F017FE2B78532B03D1FEF796FC71
:1097E8000AF034FB164B1B7803F08003DBB253B14D
:1097F8003B7813F0010F06D0124820210422BDE85F
:10980800F041F6F7C7BD14F0800F0F4805D12B23A0
:109818000A2103746143113006E02D230374373B9A
:109828005C43113004F520610322BDE8F041FEF7E6
:10983800CFBB00BFC116002001170020681600200A
:10984800302A002002020020F20100201FB5204B20
:1098580020491A781AB1087840F001000870097890
:109868001C4C11F0010F31D01B490978532901D044
:109878000AB103E082B901221A700DE023290BD145
:10988800002018701549FEF77DFBFEF73FFC237892
:1098980043F00603237019E01B78012B16D1202111
:1098A8000A460F48F6F776FD0E4B68461B681022ED
:1098B800996805F0C2FD002409491DF8040001EB70
:1098C8004401013413F063FF102CF5D11FBD00BF14
:1098D800C1160020011700206816002018980208F9
:1098E800F2010020A0160020034B1B78532B01D156
:1098F800FEF70CBC704700BF68160020084BFF2815
:109908001A68936807D1917B41B10649927C09781E
:1099180001FB023302E0927C02FB003318467047D9
:10992800A0160020C11600204328F8B504460D46AD
:10993800174608D1114B0A261A7891FBF6F66FF3F1
:10994800C3021A7000E00E462046FEF7D7FB90B11E
:109958000A4B303C1A780A2602F00801C9B20029DD
:1099680018BF002506FB05466FF3C30236B21A700E
:10997800BE42A8BF3E4630B2F8BD00BF0117002066
:10998800634B2DE9F3411A689846157C977C614C26
:109998002DB1614821780222FEF71AFB00E02570FC
:1099A800FF01237807F50A47D83707EB43075B4ED3
:1099B8000BB90DB10FE015B901A8394601E001A8AE
:1099C800B91E022205F039FD9DF80430F3759DF8A3
:1099D8000530337605E006F117003F210222F6F73D
:1099E800D9FC5B23B375023373764D4B1B7813F0A8
:1099F800010F61D04B4B1B78A3F13002D2B2092A78
:109A080035D822780AB9002D40D1474A1178144632
:109A18009942464A01D000211170DFF814E10DF196
:109A2800080C9EF800E0A3F13000E644DFF80CC112
:109A3800117800EB8000604400EB010C0131C9B2E1
:109A480040189CF86CC090F86C000EF804CC1170AB
:109A580008B1032901D90021117023700DB93846C6
:109A680000E0B81E01A9022205F0E1FC17E0232B53
:109A780004D12F4B1A7892B9013205E02A2B05D16F
:109A88002B4B1A785AB1013A1A7008E0532B06D1B9
:109A9800284A533B1370264A1370FFF725FF264BBD
:109AA8001B7803F08003DBB2002B2FD0204B1B78F0
:109AB800F6182023F37529E045B31A4B1878A0F15E
:109AC8003003DBB2092B10D81A4A137803B9237074
:109AD800013303F001031370D8F800302178B3F98B
:109AE8001020FFF721FF207005E0432803D1114B18
:109AF8001B7803B92370104B1B7803F08003DBB28B
:109B080023B1054820210222F6F744FCBDE8FC8178
:109B1800A0160020AF16002000020020F20100204D
:109B2800011700206816002085160020AE160020B8
:109B380082160020CB160020302A0020E0FA010807
:109B4800F7B5364E364D3378364C6FF341033370E4
:109B580013F018F9FFF7C8FE02238DF807302B78A9
:109B68008BB1314AD17941F00101D1712F4A207866
:109B780002EBC303D3F8A07093F8A5203978FFF758
:109B8800D3FE38700DE0337813F0010F06D0237838
:109B9800303BDBB2062B9CBF234AD37003238DF8DE
:109BA8000730337813F0010F12D0214B1B7803F0E4
:109BB8008003DBB263B129781C4B1E4803EBC10359
:109BC80093F8A4309DF80720C0182021F6F7E2FB8F
:109BD8002378232B09D1184A2B781268927C013AF2
:109BE800934202DA0E4A0133137023782A2B04D1E8
:109BF8002B7813B10A4A013B13702378532B0AD1EF
:109C080011F05EF90021084B2970DA7961F300023E
:109C1800DA71FFF769FE00232370FEBD01170020EB
:109C2800CB16002068160020D0310020E0FA010889
:109C3800302A0020F2010020A01600202DE9F14F63
:109C4800914E924C3378924D232BDFF888820BD1BA
:109C58002368B3F90800FEF705FA286098F8003081
:109C680043F0080388F800303378532B40F0E28043
:109C7800236848F685229B68934202D12A68854B5F
:109C880005E04AF21422934203D12A68824B1A70E3
:109C98000EE043F6DD2293420AD1804B29681A78F8
:109CA80061F300021A7005F0C3FE08B105F0DEFE8C
:109CB800236843F6E0229B68934206D1774B2968D4
:109CC8001A7861F3C7121A7019E043F6EA22934230
:109CD80006D1724B29685A7861F300025A700EE077
:109CE80043F6E72293420AD129686D4B19B11A68E5
:109CF80042F0005202E01A6861F35D721A6023684C
:109D080043F6DA229B68934202D12A68654B05E044
:109D180043F6E822934203D12A68634B1A7008E09D
:109D280048F68E22934204D12B6813B9584B01226E
:109D38001A602368986848F6CF23984202D12A68A7
:109D48005A4B05E048F6D023984203D12A68584B6D
:109D58001A7016E048F6CE23984203D12A68554B6C
:109D68001A7015E048F6D123984203D12A68524B5D
:109D78001A701BE048F6D223984202D12A684F4B4A
:109D88001AE048F6D423984202D12A684C4B13E0D3
:109D980048F6D523984202D12A684A4B0CE043F68C
:109DA800E233984202D12A68474B05E049F2DC4386
:109DB800984202D12A68454B1A7000B2FEF778F92A
:109DC80023689A6843F698139A4231D12968DFF8D4
:109DD8000CB1DFF8BCA00BEBC1031B793C4FC3F3FC
:109DE8004113012BDFF8F8901EDD387800F5665036
:109DF800203005F007FB3B78DAF8001009EB030286
:109E080011720BEBC1021279C2F34112032A0BD172
:109E18001E4A126890681030C01805F0F3FA3B78B3
:109E2800DAF800204B441A743B782A6809F80320B2
:109E3800FFF75AFD98F80030264F13F0010F00F095
:109E4800B1802368114F9A6843F698139A4267D1F4
:109E58003378442B4ED12F7844E01F4B01371B78C1
:109E6800FFB233B109EBC7031B79C3F34113012BCD
:109E780040DC05F0DDFD28B109EBC7031B7913F0C1
:109E8800100F2FD02F6035E068160020A016002094
:109E9800D8160020C41C00201B2A00207E17002092
:109EA800302A00205E3400208C2A0020722E0020E8
:109EB800422F0020452F0020432F0020742E002021
:109EC800EB2D002038180020DA100020491500205A
:109ED800C1160020011700203E0D002008040020B4
:109EE800881E0020914B03EBC7021279994612F0A5
:109EF800080FB2D03378552B5ED12E780DE0013E95
:109F0800F6B205F095FD30B1884B03EBC6031B791B
:109F180013F0100F01D02E604EE0002EEFD14BE071
:109F280005F086FD00282CD03B6843F6C4219A68CA
:109F38008A4203D046F6AA718A4204D13078B5F92C
:109F480000102D2219E0A2F56A516139052903D9BB
:109F580043F6E9218A4201D1012307E043F6E021D3
:109F68008A4202D00A318A4202D100232B6023E0C0
:109F78003078B5F90010B3F91020FFF7D5FC286048
:109F88001AE03B686A4A99688A18012AF0D8327838
:109F98002F2A11D9B3F9103030339A420CDC303AF9
:109FA8002A6009E02368B3F90800FEF75BF8286027
:109FB8003B7843F008033B70FFF796FC216843F6B3
:109FC800D2228B6893420BD12B6813B959485A494E
:109FD80001E0584859490222F6F7B2FC0226D2E0BD
:109FE800534A9A18012A17D82B6813B95448554967
:109FF80008E0012B02D15248534903E0022B05D156
:10A008004F4852491022F6F79BFCBBE0032B40F067
:10A01800B9804B484E49F5E748F6D32293424D4F55
:10A028000DD129680A22B1FBF2F302FB1312303278
:10A03800FA7730332E22BA777B770326A3E043F6EC
:10A04800981293425ED12E68384D102255F836107A
:10A0580007F1100005EBC605F6F772FC2D7905F03F
:10A068000705012D02DC781D3B4910E0022D0AD1BD
:10A078003A490B22781DF6F763FC394BB81D19785D
:10A088002A4601313BE0032D09D13649781D0B22C0
:10A09800F6F756FC324BB81D197801312EE0042D25
:10A0A80002D1781D304903E0052D10D12F49781DC4
:10A0B8002B4D0B22F6F744FC2978B81D01310222FA
:10A0C800FDF786FF297807F10A00093116E0062D09
:10A0D80058D1234D26490B222648F6F731FC29781A
:10A0E800254801310222FDF773FF297823480931F9
:10A0F8000222FDF76DFF2978214811310222FDF770
:10A1080067FF3FE0B1F91060092E04DD632ECCBF74
:10A118000326022600E00126C6F120003818296827
:10A1280046F08002FDF754FF2DE000BF0804002030
:10A138003175FFFF10020020B0FB0108B2FB0108D7
:10A1480002020020F69B0208179C0208389C0208AD
:10A15800599C0208F2010020A39D0208FE9C0208F7
:10A16800C1160020829D0208409D02081F9D02081A
:10A17800619D0208F7010020F8010020FC01002081
:10A1880000020020102698F8003013F0010F0BD0C1
:10A19800264B1B7803F08003DBB22BB12448202127
:10A1A800801B3246F6F7F6F8224EB37803F0020326
:10A1B800DBB2002B36D0FDF705FE1F4D034628B94C
:10A1C8002878F11D6522FDF71BFE08E0B279297891
:10A1D800B388F01D01FB023109B205F02EF923689E
:10A1E80046F6AA729B6893420FD006DC43F6C42257
:10A1F80093420AD043F6784205E046F6EA72934263
:10A2080003D048F68E2293420CD105200B21FDF78E
:10A2180069FE297809480131022201B0BDE8F04FF2
:10A22800FDF7D6BE01B0BDE8F08F00BF302A002090
:10A238001202002010170020C1160020F301002090
:10A24800F0B5114B1F78114B303F1E680DE0D6F862
:10A2580014C01CF803C00133644501D112E0002387
:10A26800DAB28242F3D301350D70094B062209494F
:10A2780002FB07330D785B1993F8D440002CEED11C
:10A288000C70F9321046F0BD68160020A0160020A8
:10A29800E0FA0108AE1600202DE9F74F934C9448D8
:10A2A800226890F800909368977C99B207FB091789
:10A2B80047F2AC65AB42BFB280460BD18D490878F6
:10A2C800497800F00700C1F3420101EBC00107EB38
:10A2D800C10725E047F66C0083420CD18549087810
:10A2E8004D7800F0070088214843C5F342057739C7
:10A2F80001FB05010DE047F6244083420BD17D495F
:10A308000878497800F00700C1F3420101EBC00169
:10A3180089017F1804E0B3F5E97F08BF01EB49071D
:10A32800754E764D317811F0010F52D146F6B26272
:10A33800934204D046F6B242934240F04381704AB9
:10A3480012782A2A3CD16F4A92F800A00AF1010A31
:10A358000AF0010A82F800A0BAF1000F1BD046F6F5
:10A36800B242934208D1684B46F63E329A809A78B8
:10A3780042F002029A7025E1202110226348F6F784
:10A3880009F84FEA49139944614B002009EB03018E
:10A39800FDF7F8FD16E1FDF78DFD236850469A6834
:10A3A80046F6B2439A420CBF5A495B49FDF7EAFDAB
:10A3B80098F80010594801310222FDF709FE01E121
:10A3C800552A02D0442A40F0FD804E4B00221A70D4
:10A3D800F8E05069F6F72EFA494B834693F800A047
:10A3E8009946BAF1450F02D14D4B00221A705046DA
:10A3F800FDF784FE00284ED04A4B5FFA8BFB1A7893
:10A4080052450ED15846FFF71BFFFF2804D1584686
:10A41800FFF716FFFF283ED0434B1A7801321A7017
:10A4280015E0DFF804A100228AF8002058460193BD
:10A43800FFF706FFFF28019B04D09AF8002001329D
:10A448008AF8002099F80020FF281A7023D0216884
:10A45800364A4B6910601B5C886846F6B2618842D0
:10A468001360924610D1562B01D0542B0CD198F87A
:10A478000030123BDBB2022B06D82B7838B2C0185A
:10A4880004F0CAFFCAF800002B7838B2C018DAF80E
:10A49800001004F0B7FF99F80030552B17D1236846
:10A4A800997C0F2913D92A7808398A42134B01DA83
:10A4B800083200E000221A70134B9B7803F0020365
:10A4C800DBB20BB1FDF702FD174B00221A7099F8A9
:10A4D8000030442B39D123689A7C0F2A35D9297842
:10A4E800064B072924D90839197023E0A016002043
:10A4F800C1160020C616002001170020CB16002028
:10A50800681600200C17002010170020F201002008
:10A51800A1840208B2820208F4820208F301002032
:10A528008216002085160020AE160020D8160020BE
:10A53800083A1A70874B9B7803F00203DBB20BB121
:10A54800FDF7C4FC844B00221A7099F80030432BA5
:10A558000CD1236838B25B691978804B19602B7865
:10A56800C01804F04FFF7C4B00221A7099F8003095
:10A57800232B13D122682B78927C013A93420DDA6F
:10A58800774A01331370744B00221A70714B9B7811
:10A5980003F00203DBB20BB1FDF798FC99F8003029
:10A5A8002A2B0FD12B786BB16D4A013B13706A4B84
:10A5B80000221A70674B9B7803F00203DBB20BB1E1
:10A5C800FDF784FCFFF790F9664A2B7811789246DC
:10A5D800994288BF137012780F32934202DD614AA4
:10A5E8000F3B137023684FF0000B93F81290B9F1EA
:10A5F8000F0F9ABFC9F120095FFA89F94FF01009C6
:10A608009AF8003038B2C018584404F005FF564B89
:10A6180003F8090009F101095FFA89F9B9F11F0F77
:10A6280005D822680BF1010B927C9345E8DB327860
:10A6380012F0010F16D022684C49927C09780F2A33
:10A6480001F0800198BFC2F11002C9B294BFD2B222
:10A65800002239B129789AF8000010319A18091A9D
:10A668005F2353542368986849F2DA43984209D122
:10A678003F4B1B78532B05D104F0CEFE3D4B187091
:10A6880004F0BAFFDFF8CC9099F802304F4603F097
:10A698000203DBB2002B4DD0FDF794FB034690B9C3
:10A6A800226847F6244192688A420CD046F6B241A5
:10A6B8008A4214BF287898F8000009F1070165223A
:10A6C800FDF79EFB10E02368BA799B682A48B3F52A
:10A6D800E97F0CBF98F800102978BB8801FB02318C
:10A6E800BA7909B204F0A9FE23689A7C102A13D813
:10A6F8009B6847F2AC6293420BD1337813F0010F99
:10A7080001D0102013E0202107221C48F5F742FE53
:10A7180010E0B3F5E97F02D105200B2108E046F6E9
:10A72800B242934202D10020102101E0002007210B
:10A73800FDF7D8FB23689B7C102B08D92978104893
:10A748000131022203B0BDE8F04FFDF741BC03B070
:10A75800BDE8F08F10170020AE160020D816002094
:10A76800CB160020C3160020F2010020302A00205A
:10A778006816002087160020171700200202002004
:10A78800F30100202DE9F74F864C874F2368874E49
:10A7980099689B7C3A78B3F1010848BF03F1060831
:10A7A8004FEAE808337808F1010812F0010F03FBBB
:10A7B80008187F4D00F0AD807E4B1A789946432AE1
:10A7C8004DD128780FFA88FA0AEBD00004F024FE5D
:10A7D8002268794B916846F2A2529142186001D1E1
:10A7E8002A783AB12A78012102F0070211FA02F216
:10A7F80050401860287819780AEBD00004F002FE5F
:10A80800236847F24A029B68934209D1684B1A7839
:10A818006A4B03EBD203684A126883F8A0211EE052
:10A8280046F65222934205D13178002001310AF0D0
:10A838008FFB14E046F2686A4FF0000B23689B68B0
:10A84800534504D101200BEB00010AF081FB0AF10A
:10A85800080A46F2A8639A450BF1010BEED199F864
:10A868000030232B10D122682B78927C013A934236
:10A878000ADA4F4A01331370514B9B7803F00203F5
:10A88800DBB20BB1FDF722FB99F800302A2B0CD173
:10A898002B7853B1464A013B1370494B9B7803F020
:10A8A8000203DBB20BB1FDF711FB99F80030552B11
:10A8B80014D12368997C0F2910D92A7808398A423B
:10A8C8003B4B01DA083200E000221A703C4B9B78BF
:10A8D80003F00203DBB20BB1FDF7F8FA99F8003088
:10A8E800442B7ED123689A7C0F2A7AD92978304B59
:10A8F800072902D90839197001E0083A1A70304B53
:10A908009B7803F00203DBB2002B6AD0FDF7DEFA76
:10A9180067E048F6452399420DD1264B1B78A3F1F1
:10A928003101C9B2072906D842F006023A70072257
:10A938005343573B337023689A6843F6E3339A428C
:10A948004FD11C4B1B782A2B44D11E4B93F80090F7
:10A9580009F1010909F0010983F80090B9F1000F24
:10A9680013D033781B2B08D9154B46F63E329A8004
:10A978009A7842F002029A7033E05A011249D318C9
:10A988000020C918FDF7FEFA2BE0FDF793FA4846B8
:10A998000E49FDF7F7FA31780D4801310222FDF72B
:10A9A80017FB1EE0A016002001170020C11600208A
:10A9B800CB16002068160020D8160020881E00201C
:10A9C80010170020CD160020A08802085E88020813
:10A9D800F3010020552B01D0442B02D17D4B0022DE
:10A9E8001A70FEF781FF7C4A2B78117893469942BA
:10A9F80088BF137012780F32934202DD764A0F3BFC
:10AA0800137023684FF0000A93F81290B9F10F0FF2
:10AA18009ABFC9F120095FFA89F94FF010099BF82C
:10AA280000004FFA8AF318180FFA88F202EBE000D8
:10AA3800019304F0F1FC9BF80020019B5FFA80FC75
:10AA48009B1803F0070316E04CFA03F0634901333F
:10AA580000F0010000280CBFA520DB20DBB201F8C4
:10AA680009000AF1010A09F10109082B5FFA8AFABB
:10AA78005FFA89F903D0B9F1200FE5D109E0B9F1FE
:10AA8800200F06D023684FFA8AF19B7C89189942D7
:10AA9800C5DB3B7813F0010F15D0236850499B7C28
:10AAA80009780F2B01F0800198BFC3F11003C9B2D8
:10AAB80094BFDBB2002331B1297810318A1A474993
:10AAC800CB185F219954DFF8248198F80230474663
:10AAD80003F00203DBB2002B63D0FDF773F90346E2
:10AAE80000BB226846F6522192688A4206D0243179
:10AAF8008A4203D043F6E5118A4204D130783949B5
:10AB08006522002309E043F6E3318A4208D1307810
:10AB18001C38C0B208F107016522FDF771F918E089
:10AB28002878F7E7236846F612229B68934203D0F9
:10AB380043F6EE22934202D1BA79317801E0BA792C
:10AB48002978BB88274801FB0231BA7909B204F099
:10AB580074FC23689A7C102A02D905200B211EE078
:10AB68009B6846F6122293420ED006DC43F6E512A5
:10AB7800934209D043F6EE2204E046F6522293426D
:10AB880002D02432934201D1102007E043F6E33289
:10AB9800934202D10020102101E000200721FDF797
:10ABA800A1F9236846F6B6219A688A420FD046F67C
:10ABB80070118A420BD09B7C102B08D929780A483F
:10ABC8000131022203B0BDE8F04FFDF701BA03B02E
:10ABD800BDE8F08FCD160020C3160020F20100203A
:10ABE800302A002017170020F3010020101700203A
:10ABF8002DE9F04F714E89B033689C689F7C122C08
:10AC080001D00B2C0DD16E4A1778303F122CFFB2B1
:10AC180009D19B7B3BB96B4BD879FEF76FFE054694
:10AC280015E0013FFFB2FF20FEF768FE4AF2481325
:10AC38009C4205460BD14AF2152004F0EDFBC0B248
:10AC4800069020B15F4B9B790BB1FDF75FFA336833
:10AC58009A68122A17D19B7BC3B1594B187831389F
:10AC6800401904F0D9FB574B5FFA80FA9B7973B10E
:10AC7800AAF13003DBB2092B09D8534B1B7833B93F
:10AC8800FDF744FA03E04FF0000A00E09A464F4C03
:10AC9800DFF84C812178DFF84C9111F0010100F0C8
:10ACA8006B8198F80030DFF840B100218BF8001074
:10ACB800184605910493FDF721FADFF830B105999C
:10ACC800049B002800F0B5804148DFF824E10170BA
:10ACD8009EF800003F4A984213603B4940F08A8042
:10ACE80033689B8903F00F03032B21D1A0F1300CAB
:10ACF8000A2000FB0CF0384BDFF8E0C093F800E0C6
:10AD08000390704407900EF1010E1CF80000DDF866
:10AD18000CC05FFA8EFE106083F800E00CEB0E00AA
:10AD2800DFF8B8E01EF80000002870D118706EE057
:10AD3800082B2CD1A0F1300C27480CEB8C0E037893
:10AD48000793264B9E44079B734493F86CE0079344
:10AD5800224BBEF1000F01D180F800E090F800E02E
:10AD68000CEB8C0C634403EB0E0C0EF1010E5FFA36
:10AD78008EFE73449CF86CC093F86C30C2F800C027
:10AD880080F800E0002B42D1134803703FE0072B06
:10AD98000ED130280ED1DFF840E09EF8003003B124
:10ADA8000538013303F0010310608EF800302EE0FF
:10ADB800062B2CD10B78013328E000BFA016002009
:10ADC80087160020CE160020CB1600200117002081
:10ADD80063340020D8160020AE160020E0FA0108DF
:10ADE80068160020B0160020831600208816002060
:10ADF8008516002099488EF800309BF800304FF0F7
:10AE0800010C80F800C013B10B7863440B70402329
:10AE18008BF800300B78BB4202D3914B781E187028
:10AE280008781168281804F0EDFA237843F0040331
:10AE3800237098F80030232B1ED1894B7A1E18787E
:10AE4800904219DA0130C0B218702818049304F03F
:10AE5800E3FA049B20B918782021281804F0D2FAC4
:10AE6800804B40221A7023787C4A43F004032370F5
:10AE780000238BF80030137098F800302A2B10D17B
:10AE8800774B1A786AB1013A1A70764B40221A70D9
:10AE98002378724A43F00403237000238BF80030B0
:10AEA800137098F80030432B1ED16D4B1878B842B8
:10AEB80005D228182021049304F0A4FA049B9BF8D7
:10AEC800002032B91B787A1E934202DA644A0133B1
:10AED80013702378634A43F004032370002313702C
:10AEE8005E4A8BF8003013709BF8003013B15E4A4D
:10AEF800013B13709BF80030012B0ED1584B1A7888
:10AF0800BA4201D201321A70544A002313702278CF
:10AF180042F0040222708BF80030237803F0040218
:10AF2800D2B2002A3BD0514A6FF38203137000213A
:10AF380011224F48F5F72EFA4E4A494B11781B78E3
:10AF4800994288BF137011780F318B4202DD49494D
:10AF58000F3B0B704848137801781022C91849191B
:10AF6800434804F06AFA4248F5F764FCC2B20F2A73
:10AF780015D809EB02000DE011224846F5F70AFA48
:10AF880010222946484604F058FA4846F5F752FC7C
:10AF9800024648442021C2F11002F5F7FBF998F85F
:10AFA8000030532B20D133689A684AF248139A42EA
:10AFB80008D1284604F030FA20B14AF215200121C0
:10AFC80004F020FA28463946FCF7EAFF264A00230F
:10AFD8001370294A01201370264A01461370009302
:10AFE8000246034609F0E0FFFEF77EFC204B234AA9
:10AFF80003F1100153F8040B8B4242F8040BF9D10A
:10B0080033689A68122A50D19B7B002B4DD0AAF145
:10B01800300A5FFA8AFABAF1090F46D8237813F092
:10B028000107174B08D09A7932B10D4A1178154AA1
:10B038001278313A914238DA9B792BB9104BDA7988
:10B04800114B1B789A4230D00E4B054A187811786C
:10B05800054A30381278002325E000BFAE160020DC
:10B06800CB1600206334002088160020011700202A
:10B07800B0160020C316002083160020020200200C
:10B08800CE16002087160020C116002017B199425D
:10B0980000D132B9DFF8F4C04FF02A089C448CF88C
:10B0A80010800133DBB28342F0DB326893680B2BEC
:10B0B80001D0122B0AD1334B991D13F8010B20280C
:10B0C80002D10D3003F8010C8B42F6D192684AF296
:10B0D80048139A4210D12C4B9B796BB1069B5BB1FC
:10B0E8000027781904F098F918B1284B2A22DB199F
:10B0F8001A740137102FF4D1237813F0010F0ED0F2
:10B10800234B1B7803F08003DBB243B1214B224A67
:10B118001B78127810339B1A1C4A5F21D1541F4C9C
:10B12800A37803F00203DBB2002B28D0FCF74AFE19
:10B138001B49034628B908786522E11DFCF760FE23
:10B1480012E03068B4F90430A27984680978122CC6
:10B1580001FB023105D1807B18B90B49C97902FB83
:10B168000131104804F069F933689B68122B06D145
:10B178000820014609B0BDE8F04FFCF7B3BE09B09E
:10B18800BDE8F08F02020020CE160020F201002058
:10B19800302A0020CB160020C316002010170020EC
:10B1A800C11600201717002024282DE9F041144665
:10B1B80009D15C4B5C481978801801310222FCF7F0
:10B1C80007FF0234AAE0E72809D1564B56481978F8
:10B1D800801801310322FCF7FBFE03349EE0A3280C
:10B1E8002AD1504D2B783F2B15D810464F49FCF7E4
:10B1F800C9FE4E48F5F71EFB2A2124184A48E4B236
:10B20800F5F746F9002800F08A80297802220131F2
:10B21800FCF7DEFE83E05901C918454D01F552518E
:10B22800393110466918FCF7ADFE05F572505830F3
:10B23800F5F700FB241871E0F22821D1394F3A4D77
:10B248003978072605EB0208B1FBF6F140460131D3
:10B258000222FCF7BDFE39782D23B1FBF6F688F8FB
:10B268000230F3009E1B8B1B324FDBB207EB8303CC
:10B278001988E21CA9529B78A818837006344DE0FF
:10B2880025280BD12C4B46F63E329A8045229A71DE
:10B298009A78053842F002029A703CE05E280BD199
:10B2A800254B46F63E429A8045229A719A783E3856
:10B2B80042F002029A702EE07C280BD11E4B46F217
:10B2C80022029A8011229A719A785C3842F002021E
:10B2D8009A7020E0EC280BD1174B46F682429A80F0
:10B2E80045229A719A78CC3842F002029A7012E09C
:10B2F800A7280BD1104B46F6A2429A8045229A7194
:10B308009A78873842F002029A7004E0E02801D166
:10B31800541C03E018B1044B18550134E4B220461C
:10B32800BDE8F081C1160020F201002080840208E7
:10B33800A84702085D6B02081017002038B50A4BB1
:10B3480045F655151B78002405FB030507E0074B58
:10B3580022461978FFF728FF041B2D190446287880
:10B3680008B11F2CF3D938BD86160020C11600205D
:10B3780070B5002543F6FA44204604F04DF8064619
:10B3880004F1080004F048F816F0FF0F06D020F08A
:10B398007F0010F0FF0F01D00135ADB246F219035E
:10B3A8009C4201D00934E7E7284670BD38B5B0F9AA
:10B3B80000500B4C05EBC50505F5745502352846BC
:10B3C80004F02AF8C1B211F0800F07D0238828466C
:10B3D800013B01F07F01238004F014F8208838BD78
:10B3E80080160020454B2DE9F74F1B88444A044638
:10B3F80089461788DFF80C8123B14FF0000A0AE06C
:10B408009A4608E00529FBD198F8003043F0040378
:10B4180088F8003070E098F8003013F0030F0BD074
:10B4280013F0010F02D0B4F1FF3F05D103F002037E
:10B43800DBB21BB1012C01D03F19BFB23BB2B3F153
:10B44800FF3F04D0B3F57A7F08BF002701E040F240
:10B45800E7370FFA87FB0BEBCB0303F5725303F1C6
:10B468007A00019303F0D8FF10F0FF0F019B16D06C
:10B47800B9F1050F09D103F1820003F0CDFF20F0E7
:10B488007F0010F0FF0FC6D022E0B9F1000F1FD0E7
:10B4980003F1820003F0C0FF00F07F0618E00AF114
:10B4A800010AB4F1FF3F1FFA8AFA04D198F8003074
:10B4B80043F0010305E0012C05D198F8003043F072
:10B4C800020388F80030BAF57A7F0DD03D46A2E72E
:10B4D8004E4505D0B9F1000F02D0B9F1050F9AD148
:10B4E800BAF1000F05D000E03D46054A2DB21560BF
:10B4F80002E0034BC3F800B0BDE8FE8F80160020C1
:10B50800D8160020DC160020F0B503789BB05A1E30
:10B51800D2B26B2A0F4600F2C8805E01644AF31863
:10B528009B18644A45F655161278457806FB02368C
:10B53800E7213046F4F7ACFF0446F0B930467C21E9
:10B54800F4F7A6FF0446C0B930462521F4F7A0FF5A
:10B55800044690B930462421F4F79AFF044660B9AE
:10B5680030464021F4F794FF044630B93046F921BB
:10B57800F4F78EFF0446002876D0A41B0FB14E487E
:10B5880000E04E4831462246A619F5F7D9F930466B
:10B59800E721F4F77DFF30B128466946652246F673
:10B5A8008243FCF72DFC30467C21F4F771FF50B143
:10B5B800691EC9B201EB011101F5C041684622318B
:10B5C800112203F03AFF30462521F4F761FF38B124
:10B5D800681EC0B26946652246F63E33FCF710FC89
:10B5E8003046F921F4F754FF38B1681EC0B26946F5
:10B5F800652246F63E43FCF703FC30464021F4F74B
:10B6080047FF50B1691EC9B201EB011101F5E041D4
:10B6180068467C31112203F010FF30462421F4F7EC
:10B6280037FF50B10FB1244800E0244800192946DB
:10B638000222FCF7CDFC02340BE00FB11E4800E0FB
:10B648001E4800196946F5F797F86846F5F7F2F8C5
:10B658000419002F29D01A4B9A781C1942F00202BB
:10B668009A700023E37116E03046F5F7E3F80546D3
:10B678001FB9124831462A4615E0102810DD2A461F
:10B688000D483146F5F75CF90D4B9A785D1942F093
:10B6980002029A70EC7110200146FCF723FC04E0CA
:10B6A800084831461022F5F74BF91BB0F0BD00BF32
:10B6B8001A6F02088616002017170020B7240020EA
:10B6C80010170020020200200C4B1B7813F0010217
:10B6D80002D000200A4905E003F00200C0B218B108
:10B6E80008491046FCF74EBC03F00403DBB20BB16B
:10B6F8000549F7E705480121FFF706BFDC160020DA
:10B70800644F0208434F0208854F020803170020C0
:10B7180070B5124D124C00201249FCF735FB284633
:10B72800A1780222FCF754FCE81CE1780222FCF71D
:10B738004FFC05F1080021790222FCF749FC05F1CC
:10B748000B0061790222FCF743FCA17905F10E0098
:10B758000222BDE87040FCF73BBC00BFF2010020AC
:10B7680003170020F0FB01082DE9F3414F4F504C1F
:10B778003B689D7C237813F0010F2FD1022243F6FA
:10B78800F8410DF1060003F058FE4A4EBDF80630A8
:10B798004FF0FF3033602946FFF724FE237843F04B
:10B7A80001032370444B1B7813F0030F14D1B6F92F
:10B7B8000010424801EBC10101F572517A310922AA
:10B7C80003F03BFE3E4B1B881BB13046FFF7EEFDF6
:10B7D80010B90020FAF724F9FFF79AFF394E3378A9
:10B7E800552B0CD1DFF8D080FCF764FB98F80030BB
:10B7F8004FF0FF306FF3410388F800300CE0442B22
:10B808002AD1DFF8B480FCF755FB98F80030012006
:10B818006FF3000388F800302946FFF7E3FD98F836
:10B82800003013F0030F15D1224D2448B5F900104C
:10B83800092201EBC10101F572517A3103F0FDFDD6
:10B848001F4B1B881BB12846FFF7B0FD10B900201D
:10B85800FAF7E6F8FFF75CFFFFF736FF3378232B9C
:10B8680021D1154B1A7802F0FC026FF382021A708C
:10B87800FCF74CFC144B9A786FF341029A70134B07
:10B888001D782DB9FCF722FBFCF714FB3D600AE09C
:10B898002278013DEDB242F0060222701D700C4B79
:10B8A80053F825303B60BDE8FC8100BFA01600209E
:10B8B80001170020D8160020DC16002003170020EE
:10B8C800801600206816002010170020EF160020B0
:10B8D800F01600202DE9F0411646104A0F4653781D
:10B8E8000E21C3F342034B43117803F5EC433C3379
:10B8F8000B4D01F00701044603EB4101022203F05E
:10B908009CFDE81921780222FCF762FB6178A819EE
:10B918000222BDE8F041FCF75BBB00BFC616002061
:10B92800F2010020044B02225978044BC1F3420172
:10B9380018180131FCF74CBBC6160020F201002094
:10B9480010B5074B074C1B78074A03F0070304EBB5
:10B9580083031C88111814529B788B7010BD00BF8C
:10B96800C61600205D6B0208F2010020084B1B7808
:10B978009B0902D0012B06D102E01020054904E002
:10B988001020054901E005491020FCF7FBBA00BF6B
:10B99800C6160020A35B0208C45B0208E55B020828
:10B9A8002DE9F041DFF868800F4698F80010174D30
:10B9B800C1F382010446164605F10800013102224E
:10B9C800FCF706FB98F80010042201F01C0101F5B1
:10B9D8000A412431204603F030FDE819217802227B
:10B9E800FCF7F6FAF81C281861780222FCF7F0FA3E
:10B9F800A819A1780222FCF7EBFAF01CE1782818C4
:10BA08000222BDE8F041FCF7E3BA00BFF2010020D2
:10BA180084160020064B1B7803F08003DBB233B199
:10BA2800435C04482021C0180222F4F7B3BC7047D5
:10BA3800302A0020F20100202DE9F743484D494CF7
:10BA48002B6821789B68022203EB41010DF1060067
:10BA580003F0F3FCBDF806604FF46163B6FBF3F145
:10BA680003FB11663C22B6B2B6FBF2F302FB136687
:10BA78005FFA81F8DFB23A3A3B484146FCF7A8FA48
:10BA8800F6B2022239483946FCF7A2FA02223848AF
:10BA98003146FCF79DFA374BA9461B7813F0010F86
:10BAA8004BD0354B354D1878232804D12B78012BF2
:10BAB8003FD8013305E02A2805D12B78002B38D050
:10BAC800013B2B7035E0A0F13003DBB2092B01D923
:10BAD800432828D12B7833B941461122FDF724FF9A
:10BAE8005FFA80F80CE0012B05D139463B22FDF7BF
:10BAF8001BFFC7B204E031463B22FDF715FFC6B273
:10BB08003946324640460BF096FED9F80030ADF87B
:10BB180006009B6820780DF1060103EB4000022225
:10BB280003F085FC05E0532803D100232B70FDF7B3
:10BB3800DBFE13482978FFF76DFF65222078002384
:10BB48001049FCF75DF905200B21FCF7CBF92178AA
:10BB58000D4801310222FCF73BFABDE8FE8300BF25
:10BB6800A0160020C11600200202002008020020B2
:10BB7800100200200117002068160020CB160020B4
:10BB880001FC010817170020F301002073B5994B39
:10BB9800994D1A7812F0010F05D12A7812F038025F
:10BBA80004BF2A706A701A78924E42F001021A7025
:10BBB8002B78914C13F038023ED1904909785529D9
:10BBC80004D113F0070F2FD0DA1D0AE044290CD155
:10BBD80003F0070201323D3992FBF1F1C800411A26
:10BBE800521A62F3020323701EE053290AD1C3F3E9
:10BBF800C201013161F3C5032370637862F3430323
:10BC0800637011E023290FD1FCF780FA33787C4A5E
:10BC180043F0060333701378013BDBB21370794AA3
:10BC280052F82320784B1A6000207849FCF7AAF9CB
:10BC38001C20FFF785FEDBE0082A2CD17449002080
:10BC4800FCF7A0F90620FFF76DFE0C20FFF778FE41
:10BC58001521182201A8FFF73DFE684B1B78552BCC
:10BC680006D1637803F0FE03C3F34202013A07E00A
:10BC7800442B09D1637803F0FE03C3F34202013277
:10BC880062F343036370B3E0532B28D0232B40F0B7
:10BC9800AF802378A6E0102A51D15D490020FCF737
:10BCA80071F90620FFF73EFE0C20FFF749FE15212B
:10BCB800182201A8FFF70EFE6178564801F001012D
:10BCC800FFF7A8FE4D4B1878232801D02A2804D165
:10BCD8006378DA4362F30003D4E7532804D1237866
:10BCE800C3F3C202013280E0A0F13003DBB2092BBA
:10BCF80001D943287CD16B7802AA03F001033B21C8
:10BD0800D41883F001024B43172606FB023214F8BD
:10BD1800041CFDF709FE04F8040C6B780E22C3F32B
:10BD280042035343287803F5EC433C3300F0070003
:10BD380003EB400001A90C3A03F079FB58E0182AFC
:10BD48004DD133490020FCF71DF90620FFF7EAFD25
:10BD58000C20FFF7F5FDFFF709FE284B1B78552B44
:10BD680007D1237813F0C00F42D0C3F38112013AF0
:10BD780006E0442B07D123789A09012A38DC0132DE
:10BD880062F3871333E0232B04D12378C3F3C20271
:10BD9800023A2AE0532B2BD1FCF7B8F933781E4A24
:10BDA80043F006033370164B1648197840F82120E3
:10BDB800013119702378C3F3C201013161F3C5035E
:10BDC800C3F381112370104B11B1012904D101E093
:10BDD8001C3202E0114A00E0114A1A6008E0114AD8
:10BDE80000211170C3F3C202013A62F3C503237044
:10BDF8007CBD00BF01170020C61600206816002071
:10BE0800EF160020F0160020A0160020615B020843
:10BE1800825B020804FC010808FC010840FC0108D8
:10BE28005CFC0108CB16002073B5494B494D1A78C4
:10BE380012F0010F04D12A7812F0030208BF2A7009
:10BE48001A78434E42F001021A702B78414C13F0D5
:10BE580003022ED1404A1278552A03D1C3F3820235
:10BE6800013A04E0442A06D1C3F38202013262F3A4
:10BE78008403237017E0532A03D15A1C62F3010389
:10BE8800F7E7232A0FD1FCF741F93378334A43F017
:10BE9800060333701378013BDBB21370304A52F853
:10BEA8002320304B1A6001A810211B22FFF778FDD0
:10BEB8004CE0012A4AD101A810211A32FFF770FD7F
:10BEC800254B1878232804D12378C3F34112013273
:10BED80005E02A2807D12378C3F34112013A62F317
:10BEE800461323702CE0532804D12378DA1C62F31C
:10BEF8000103F6E7A0F13003DBB2092B01D943288F
:10BF08001ED12B7802AAC3F34113D4180C215A1C52
:10BF180003F001034B4302F001021F2614F8041C2E
:10BF280006FB0232FDF700FD04F8040C287801A98D
:10BF380000F01C0000F50A402430042203F077FAD0
:10BF480029780948C1F34111FFF764FD7CBD00BFA2
:10BF5800011700208416002068160020EF16002024
:10BF6800F0160020A016002078FC0108064B1B786C
:10BF780003F08003DBB233B1435C04482021C018CE
:10BF88000322F4F707BA7047302A0020F201002094
:10BF98004328F8B504460D46174606D1104B00262F
:10BFA8001A786FF3C3021A7000E00E462046FCF7B9
:10BFB800A5F890B10A4B303C1A780A2602F008011D
:10BFC800C9B2002918BF002506FB05466FF3C30256
:10BFD80036B21A70BE42A8BF3E4630B2F8BD00BFA6
:10BFE800011700202DE9F3416E4F6F4E3B7843F067
:10BFF80001033B70347844B94AF28E1003F00CFA0E
:10C008006A4B6B491860204617E0012C02D10020CA
:10C01800684912E0022C02D1002067490DE0032C88
:10C0280002D10020654908E0042C02D100206449AF
:10C0380003E0052C03D163490020FBF7A3FF317807
:10C04800D9B9614B1B78312B01D1013101E0302B7B
:10C0580005D1564B4AF28E10196003F0D3F95B4BA9
:10C068001A785B4B02F08002D2B20AB1202202E0B9
:10C078004E4A12683032DA776EE001290BD0022975
:10C088000CD003290DD004290ED04AF28A150529AF
:10C0980018BF00250AE04AF27A1507E04AF27E1531
:10C0A80004E04AF2821501E04AF286152946042284
:10C0B80001A803F0C2F9474B474A03F1100153F8AE
:10C0C800040B8B4242F8040BF9D1032243489DF834
:10C0D8000410FBF77DFF032241489DF80510FBF78C
:10C0E80077FF03223F489DF80610FBF771FF3E4893
:10C0F80003229DF80710FBF76BFF334B3B4C187876
:10C10800232804D12378022B22D8013304E02A28DB
:10C1180004D12378E3B1013B237019E0A0F1300387
:10C12800DBB2092B01D9432812D194F8008002AA66
:10C13800904418F8041CFF22FFF72AFF08F8040CA3
:10C14800207802AA131813F8041C281803F05AF9C7
:10C1580027482178FFF70AFF1B4B1B78532B1FD169
:10C16800224B00221A7033780133DBB2062B33706E
:10C1780004D0012B14D10D4B1B688BB1FDF7B4FB18
:10C18800002333703B781B4A43F006033B70137857
:10C19800013BDBB21370184A52F82320174B1A6080
:10C1A800BDE8FC8101170020C1160020D816002028
:10C1B800A5950208CE960208EF9602081097020885
:10C1C800319702085297020868160020302A00208A
:10C1D800F2010020BDBC0208020200200302002078
:10C1E800070200200B0200200F020020CB160020BF
:10C1F8007CFC0108EF160020F0160020A016002095
:10C2080070B5174C0D460646002120464FF4C17202
:10C21800F4F7C0F8FF2D0AD1B10001F5D641204648
:10C228003E31042203F009F923789BB970BDFE2D35
:10C2380001D1173E02E0FD2D02D10136267009E03A
:10C24800B60006F5D6403E30401903F0E5F8C0B216
:10C25800207020B10248BDE8704011F0F5BF70BDF4
:10C26800B01800202DE9F04112F020F860B110203C
:10C278008F49FBF787FE8F4B1B78432B40F0EE81ED
:10C28800BDE8F04112F034B812F022F8002826D0A8
:10C29800894C23786BB110208849FBF773FE8848D6
:10C2A8002D211030F4F7F4F8002800F0D781217818
:10C2B80010E010208349FBF765FE81482D211030DE
:10C2C800F4F7E6F80446002800F0C88112F018F8E0
:10C2D800014620468222BDE8F041FBF779BE7A4C40
:10C2E80043F6CC2223689B68934250D0774E744D16
:10C2F800307803EB800003F08FF80322014674487E
:10C30800FBF766FE2368986846F6A24398422BD04E
:10C31800203B984228D03378013000EB830003F0AB
:10C328007BF80322014605F11500FBF751FE23684F
:10C3380030789B68023303EB800003F06DF803222A
:10C34800014605F11900FBF743FE236830789B6826
:10C35800033303EB800003F05FF80322014605F185
:10C368001D00FBF735FE0EE02D2103225948F4F796
:10C3780011F82D2103225848F4F70CF857482D21BD
:10C388000322F4F707F820232B772B762B75544BD1
:10C398001B7813F0010F00F0BD80236843F6CC2210
:10C3A8009B68444D934261D04E4E484F327838785E
:10C3B800D31803EB800003F02FF84B4B01461860AD
:10C3C80028789846A0F13002D2B2092A01D9432828
:10C3D8000FD109B2BA22FDF7A7FA236832789B6811
:10C3E8000146C8F800003878D31803EB800003F042
:10C3F80009F82B782A2B04D1337813B1394A013B39
:10C4080013702B78232B0ED13378022B0BD822688C
:10C4180046F6824192688A4205D020318A4202D08B
:10C42800304A013313702B78552B01D0442B0FD190
:10C43800236831789B68A3F5D643B3F13E0248BF21
:10C44800A3F13B023B7803EBA202D0B2FFF7D8FE80
:10C45800264B1B7803F08003DBB23BB13278184BD4
:10C4680003EB820320225A749A74DA742B78532BC4
:10C4780006D023689A6843F6CC239A4240F0EE80AF
:10C48800FBF744FE236846F63E329B68934203D18D
:10C498000E4B0220197806E046F6A242934227D1B5
:10C4A8000A4B002019780131BDE8F04108F050BD71
:10C4B800BA83020868160020D4100020918202086E
:10C4C800F2010020DB830208A0160020C11600201C
:10C4D80003020020070200200B0200200F020020A8
:10C4E80001170020CB160020D8160020302A002083
:10C4F80046F68242934204D1594B01201978091813
:10C50800D2E746F63E42934240F0A880544B0320BF
:10C518001978C8E7236849F2EE429B6893423ED1F6
:10C528004F4E10204F49FBF72DFD31784E4D01EB52
:10C53800011101F51441EE311022284602F07DFF69
:10C548002B4605F110012A461078474F78B947491C
:10C55800FBF718FD3846E721F3F79AFF78B13178F1
:10C56800401B381801310322FBF732FD07E013F8AE
:10C57800010B10B9203003F8010C8B42E4D13C4D7B
:10C588002B782A2B03D13078FD21FFF739FE2B7841
:10C59800432B63D1307823680130C0B259E043F6A9
:10C5A800CC229342324E1AD010203249FBF7EAFCD3
:10C5B80033782A2B52D1304B1B689B68A3F5D6439E
:10C5C800B3F13E0248BFA3F13B02254BFF211B7884
:10C5D80003EBA202D0B2BDE8F041FFF711BE3378F9
:10C5E8001F4D552B04D12B78142B01D1033B2B70F5
:10C5F8003378442B05D12B78122B02D1184B1522F6
:10C608001A702B78DFF874805901C918414401F574
:10C61800725100207931FBF7B5FC08F56E511020F6
:10C6280071312F78FBF7AEFC3378112F8CBF0327BD
:10C6380000272A2B05D12878FE21C01BC0B2FFF79E
:10C64800DFFD3378432B09D12B78173BDF1B236899
:10C65800F8B2997CBDE8F04111F010BEBDE8F08158
:10C66800C116002099830208F20100208F69020890
:10C678006816002057830208A0160020A847020861
:10C6880010B50E4B1B78452B17D10D4B1A7842F07D
:10C6980006021A700B4A1378012B0ED80A490B4C64
:10C6A800086844F823000133137083680B60FBF7B4
:10C6B80063FBBDE81040FBF729BD10BD68160020DC
:10C6C80001170020EF160020A0160020F016002009
:10C6D80010B50C4B04462146D8790BF06EF868B1BA
:10C6E800094B1B5D543BDBB2012B09D820460AF0ED
:10C6F8005BFFD0F1010038BF002010BD022010BD43
:10C70800022010BDCE1600203D2C002008B50BF0ED
:10C7180043F8C0B208BD00002DE9F047634B644CF4
:10C728001A78994612F0010F624D65D02078FFF70C
:10C73800CFFF614A2B181178604F93F8A031604EF3
:10C7480044293870336090460AD12D2B08D038B967
:10C7580095F8A11101233B7031602078FFF7D6FFCF
:10C7680098F80030552B10D133682D2B0DD03B781D
:10C778005BB1013B514ADBB21370EB1893F8A0117F
:10C788004F4B20781960FFF7C1FF98F80030232B32
:10C7980019D14C4B20781B689B7C013B984212DADC
:10C7A800434B0130C0B21870FFF792FF3870281859
:10C7B80090F8A0313360444B9B7803F00203DBB25E
:10C7C8000BB1FBF783FB98F800302A2B14D12078A3
:10C7D80090B1374B0138C0B21870FFF779FF387045
:10C7E800281890F8A0313360374B9B7803F0020388
:10C7F800DBB20BB1FBF76AFB344EFDF775F8237813
:10C8080032789A4288BF337032780F32934202DD11
:10C818002E4A0F3B1370DFF8C48000273078381891
:10C82800C0B2FFF755FF281890F8A0310137102F34
:10C8380008F8013F07D0254B1A78224BBA181B6815
:10C848009B7C9A42EADB99F8003013F0010F13D071
:10C858001F4B1A781F4B02F08002D2B22AB12278FD
:10C8680031781032521A5F2105E02278317810327F
:10C87800521A13490968995413498B7803F0020333
:10C88800DBB253B120780731652246F63E43FBF709
:10C89800B7FA05200B21FBF725FB21780E4801315B
:10C8A8000222BDE8F047FBF793BB00BF0117002049
:10C8B800CB160020E0FA0108681600208216002036
:10C8C800D8160020A016002010170020C31600203C
:10C8D800302A0020F2010020F3010020010200208C
:10C8E8002DE9F041074610460D461446F3F7A2FF1E
:10C8F800C3B28046B3B1AB4214D80B4E20212A46AE
:10C90800F019F3F747FD2046F3F794FFC8EB050548
:10C918006D08EDB2EF1902462146F019BDE8F04165
:10C92800F3F790BCBDE8F081F2010020F0B5124B9E
:10C938001A1894781F46ECB10E7800233A189278AA
:10C948001A4112F0010F4FF001020BD0A6420D78E8
:10C9580003D09A4042EA050502E09A4025EA02051A
:10C968000D7004E09A400D7825EA02020A7001333E
:10C97800082BE3D1F0BD00BFCE16002031220023E2
:10C988000178194111F0010F02D00449C9180A753C
:10C9980001330132082BD2B2F2D17047F2010020E4
:10C9A800034670B50846674A31B11278532A40F0F9
:10C9B800C880533A1A7070BD1278302A24D162495F
:10C9C8001C780A7822400ED00A78024112F0010F32
:10C9D80005D0012282401C7824EA02021A70013034
:10C9E8000828F1D10CE00878104110F0010F04D0AC
:10C9F800012090401C78204318700132082AF2D197
:10CA08005248002113221AE0A2F13100C0B20728CF
:10CA180024D84D4A1278024112F0010F00F091809B
:10CA28001C7854FA00F212F0010F4FF001020AD0FC
:10CA380012FA00F024EA000444481C701232BDE8DF
:10CA48007040F3F7A7BC82404049441C4C741C78E2
:10CA580022431A70102246F682436EE0132A0BD046
:10CA6800552A17D13A4A3B491278122000FB021284
:10CA7800527812F0200F64D00024344D1946204615
:10CA88006C74FFF753FF304B9B78002B59D020462E
:10CA980029464FE0142A0BD02A2A16D12C4A2D49B0
:10CAA8001278122000FB0212527812F0200F48D0A0
:10CAB800264C0022194662740120FFF737FF224BEB
:10CAC800DB78002B3DD0012033E0152A0BD0232A38
:10CAD80016D11F4A1F491278122000FB0212527801
:10CAE80012F0200F2DD0194C002219466274022032
:10CAF800FFF71CFF144B1B79002B22D0022018E0F3
:10CB0800162A0BD0442A1CD1114A12491278122035
:10CB180000FB0212527812F0200F12D00B4C0022A8
:10CB2800194662740320FFF701FF074B5B7943B195
:10CB380003202146102246F6A243BDE87040FBF7C9
:10CB48005FB970BD68160020CE1600206A16002056
:10CB5800C4160020A72B00202DE9F04F87B09DF8C0
:10CB680040508046072D0E4605929A4637D100243C
:10CB780027463378234113F0010F2CD0012523B227
:10CB88004FF000080293512029462A462B4600956B
:10CB9800CDF8048002F0B4FC1B20414662194346DC
:10CBA800CDF80080F5F7DCFA37B9112039463A4656
:10CBB8002B460097F5F7D4FA534B204613F8242058
:10CBC80001276FF3000203F824201199F6F7F6F80D
:10CBD8002046F6F7CBFA0134082CCAD1F7E1012D2B
:10CBE80003780CD10BB90B7823B3FF2300930021F2
:10CBF800464B01911B780C200133029316E0022D5D
:10CC080009D10BB90B78ABB10021FF230093019137
:10CC1800029134200AE0062D0CD10BB90B784BB1E8
:10CC28000021FF23009301910291652004220B4605
:10CC380002F066FCBAF1010F98F800302BD13BB135
:10CC4800334B0020D979024653460090F5F788FA0D
:10CC580033783BB12E4B0120D9790022034600924C
:10CC6800F5F77EFA0020F6F79BF898F80030002BCD
:10CC78005BD0284B1978002957D1274B1B78002BFC
:10CC880053D0FF2300933A2001220B4601910291D1
:10CC980002F036FC49E063B1052D4FF0000102D1E6
:10CCA80000910F2001E000910B200A460123F5F7BF
:10CCB80057FA337883B1052D4FF0000106D11020C3
:10CCC8000A4601230091F5F74BFA12E00C200A46B8
:10CCD80001230091F5F744FA022D25D0032D01D147
:10CCE8000E4B02E0042D02D10D4B1F781DE0052DDF
:10CCF80001D10C4BF9E7012D01D1044BF5E7062DC5
:10CD08000CBFFF27002710E013130020F4130020A6
:10CD1800CE160020011300201F0E002064180020EA
:10CD28003B330020E42D0020FF2798F80030002B2B
:10CD380000F09D80914C237803F02003DBB26BB1A7
:10CD48008F4B197811F0010108D1FF230093282097
:10CD580001220B460191029102F0D2FB237803F0E5
:10CD68001003DBB273B1864B197801F00201C9B226
:10CD780041B9FF230093292001220B46019102911A
:10CD880002F0BEFBE37813F0010F0ED07C4B19784C
:10CD980001F00401C9B241B9FF2300932A200122FE
:10CDA8000B460191029102F0ABFBE37803F002031A
:10CDB800DBB273B1724B197801F00801C9B241B9FD
:10CDC800FF2300932B2001220B460191029102F0D0
:10CDD80097FBE37803F00403DBB273B1684B19786F
:10CDE80001F01001C9B241B9FF2300932C200122A0
:10CDF8000B460191029102F083FBE37803F00803EC
:10CE0800DBB273B15E4B197801F02001C9B241B9A8
:10CE1800FF2300932D2001220B460191029102F07D
:10CE28006FFB0CF061FD70B1554B197801F04001B2
:10CE3800C9B241B9FF230093492001220B46019151
:10CE4800029102F05DFBE37803F04003DBB273B1BB
:10CE58004B4B197801F08001C9B241B9FF23009307
:10CE68004E2001220B460191029102F049FB119BD1
:10CE7800444A1978444B51B198F80010117032782F
:10CE88001A7033780BB1542005E0522003E011707A
:10CE9800327853201A7002F0B1FE119B00241A78E0
:10CEA8003A4B1A7098F80030234113F0010F2DD037
:10CEB8002146059810F050FC0122014628B923B2FA
:10CEC800019000920293104605E0002123B20092DF
:10CED8000191029324200B4602F012FBBAF1010FD4
:10CEE80005D12B4B8020DA790521013208E0022D8B
:10CEF80007F1010202D18020072101E080200621EC
:10CF08002346F6F74BFC2046F6F704F9337823411D
:10CF180013F0010F57D000214FF0010B23B20293F9
:10CF280002205A460B46CDF800B0019102F0E8FA0B
:10CF3800DA45DFF868900CD119F8243013EA0B03AE
:10CF480034D1134A0520D1790093594404EB0B02DC
:10CF58002AE019F8243013F0010327D1022D1FD13C
:10CF68000C4B1B7803F02403042B04BF0A4B83F8F3
:10CF780000B000230093072014E000BF302A0020EF
:10CF8800B51400205F13002060130020D214002085
:10CF9800CE160020DC140020180E002013130020E9
:10CFA80000930620791C621CF5F7DAF811992046DF
:10CFB800F5F704FF2046F6F7D9F819F824306FF38F
:10CFC800000309F824300134082C7FF46BAF07B054
:10CFD800BDE8F08F2DE9F74F16469A463378044698
:10CFE8000F469DF830909DF834B09DF83820DFF852
:10CFF8007C8043B102EA03033370097898F8002073
:10D008008A18D31A0370164B00251D70217843F631
:10D01800ED2002F0F7F9494646F2A75002F0F2F97E
:10D02800104B31465D7052464B463846CDF800B03D
:10D038000194FFF791FD2046F8F72AFD23780A4866
:10D048000A4988F80030F6F73DF88AF8005035703C
:10D058003D70257003B0BDE8F04F02F0DFBC00BFA3
:10D06800001700201F0E0020B61400200113002016
:10D078002DE9F04180460E46174646F268650024C1
:10D088003846214610F068FB88B1294608220B482B
:10D0980002F0D3F90948414610F000FB074810F0A8
:10D0A8002EFB20B90123A340327813433370013497
:10D0B8000835082CE4D1BDE8F08100BFCA1400206F
:10D0C8002DE9F04387B08046894604A847F252010B
:10D0D800082202F0B2F900244046214610F03CFB39
:10D0E80038B301260223A719002100933BB200257B
:10D0F800029323200B460422019602F001FA3946D6
:10D1080032462B4611200095F5F72AF804202146CF
:10D118002A4633460095F5F723F8B9F1000F08D0F1
:10D1280004A8214610F018FB18B10548214610F054
:10D13800FDFA0134402CCFD107B0BDE8F08300BF21
:10D148003C13002010B50B4B0B4C024603CB206060
:10D1580061600A48114610F0CDFA2146074810F0E0
:10D168009DFA064810F0CBFAD0F1010038BF002034
:10D1780010BD00BF18200020C0140020CA140020D1
:10D188002DE9F04F744B754FF0221A703B788BB035
:10D198000B2B7DD1DFF8108298F80260012E06D99A
:10D1A8006F4900200BB0BDE8F04FFAF7EBBE6D4DAC
:10D1B80019D16D4B6D4A6E496E4800241C7014706D
:10D1C8000C70047088F8024000966B4E0194367813
:10D1D8000296FFF7FFFEFAF799FF2C600BB0BDE847
:10D1E800F04FFAF767BE65486149F5F76BFF644B86
:10D1F800644A03CB644E654B1278716019782B68CA
:10D20800532A30609B7C09D05A1E48BF9A1DD610FD
:10D2180001364E4306F5CA46A8363AE05C495748F7
:10D2280010F03CFA5548FFF78DFF044618B1052366
:10D2380088F80230BDE1082246F2A8514F4802F0B2
:10D24800FCF84E49534810F055FA082246F60A21D0
:10D25800304602F0F2F83146484810F040FA4748A4
:10D268000121FFF72DFF45483F49414AFFF700FFDD
:10D2780001230093404B01941B783E4802933C499C
:10D288003A4A394BFFF7A6FEFAF740FF2C6090E1C7
:10D298000026414B334D1A78404C12F0010F00F034
:10D2A800A380384B1A789846432A21D13B780B2B18
:10D2B8001ED13248217810F04FFAC8B1324821788F
:10D2C80010F04AFAA0B920780FFA86F909EBD000D5
:10D2D80002F0A2F82378012103F007029140304AB6
:10D2E80080EA0101116009EBD300C9B202F08AF8A3
:10D2F80098F80030232B10D12A682378927C013AC1
:10D3080093420ADA254A01331370264B9B7803F0BF
:10D318000203DBB20BB1FAF7D9FD98F800302A2BDB
:10D328000CD1237853B11D4A013B13701D4B9B78D8
:10D3380003F00203DBB20BB1FAF7C8FD98F800302E
:10D34800552B3DD129682278897C144B08398A42AB
:10D358002CDA08322BE000BF0D1700200017002040
:10D36800556A0208A016002069160020021700203E
:10D378000E170020A4160020CE160020D31400207B
:10D388001820002068160020F8120020C11600207E
:10D398004C1300205713002001170020CB16002043
:10D3A800D8160020101700201F0E002000221A7027
:10D3B800814B9B7803F00203DBB20BB1FAF786FDD1
:10D3C80098F80030442B0FD122787C4B072A9CBF59
:10D3D8002A68927C083A1A70774B9B7803F002030C
:10D3E800DBB20BB1FAF772FDFCF77EFA744A2378C8
:10D3F80011789046994288BF137012780F32934281
:10D4080002DD6F4A0F3B13702B684FF0000B93F847
:10D418001290CDF81CB0B9F10F0F9ABFC9F12009CD
:10D428005FFA89F94FF01009334638784FFA8BF2D2
:10D438000B2805D198F800105218D210614904E061
:10D4480098F8001052186049D2108E5C98F80010B5
:10D458004FFA8BF251180B2801F0070A13D118B2B2
:10D4680000EBE1000692059301F0D6FF5449069AB5
:10D478000978C0B2079051185448C910415C059BFF
:10D4880006EA01010991387898F8001008905218B6
:10D498003CE0DDF81CC04CFA0AF111F0010F4C49D0
:10D4A8000CD108980B280BD14A484FEAE20C10F827
:10D4B8000C0040FA0AF010F0010F01D12A2013E005
:10D4C800DDF824C04CFA0AF010F0010F04D00898D7
:10D4D8000B2801D14D3007E046FA0AF000F00100B0
:10D4E80000280CBFA520DB200AF1010A5FFA8AFA9E
:10D4F80001F809000BF1010B09F101090132BAF138
:10D50800080F5FFA8BFB5FFA89F903D0B9F1200F96
:10D51800BFD10CE0B9F1200F09D098F800204FFADC
:10D528008BF189182A68927C9142FFF67EAF2A49CE
:10D538000B7813F0010F17D02B68284A9B7C1278C0
:10D548000F2B02F0800298BFC3F11003D2B294BF30
:10D55800DBB2002342B1227898F800101032521A38
:10D568001B49CB185F21995413498B7803F00203A8
:10D57800DBB28BB10731652246F63E332078FAF7E5
:10D588003FFC2B689B7C102B02D905200B2101E066
:10D5980000200721FAF7A6FC2B689B7C102B08D9E2
:10D5A80021780F48013102220BB0BDE8F04FFAF79D
:10D5B8000FBD0BB0BDE8F08F10170020CB16002070
:10D5C800C31600204C130020AC130020F8120020D2
:10D5D800F2010020D314002001170020302A002077
:10D5E800F301002010B50A4CA37C4BB10020094977
:10D5F800FAF7C8FC084B1B78432B01D1433BA374B3
:10D60800A07C20B90549BDE81040FAF7BBBC10BDA5
:10D618006A160020D169020868160020B06902085D
:10D62800034B1A7801321A7001230370704700BF48
:10D63800001700200A4A10B500241470094A0A4B42
:10D6480014700A4A9C701470094A5C701470094A74
:10D658001470094A1470FAF759FD084B1C6010BD84
:10D66800CE160020691600201F0E00200217002089
:10D678000E170020A416002000170020A016002076
:10D688002DE9F041002386B08DF81730884B1B78C0
:10D69800012B00F0EA81874C874D237843B12B7822
:10D6A800002B40F0A680FAF731FD08232B70A0E08C
:10D6B8002A78072A00F29D80804A1278232A13D1FB
:10D6C8002B70FAF723FD7E497E4A0B7853B17E48CA
:10D6D800013B0478DBB244F0060404700B707B490C
:10D6E80051F8233013605FE2774B1A7812F0010F7C
:10D6F80004D101210A438DF817101A70F5F798F92B
:10D7080028B92B781BB90DF11700FFF789FFF5F73A
:10D718009DF930B92B78012B03D10DF11700FFF7D4
:10D728007FFFF5F7A1F930B92B78022B03D10DF162
:10D738001700FFF775FFF5F7A3F930B92B78032B1E
:10D7480003D10DF11700FFF76BFFF5F7A7F948B9FB
:10D75800F5F7C0F930B92B78042B03D10DF1170078
:10D76800FFF75EFFF5F7F4F930B92B78052B03D1F5
:10D778000DF11700FFF754FFF5F7DEF930B92B78F4
:10D78800062B03D10DF11700FFF74AFFF5F794F9BF
:10D7980030B92B78072B03D10DF11700FFF740FFA5
:10D7A8009DF817302BB32B78072B1FD8DFE803F031
:10D7B80004070C0F1215181B0020454901E04549C4
:10D7C8000020FAF7DFFB14E000204349F9E70020C6
:10D7D8004249F6E700204249F3E700204149F0E7D3
:10D7E80000204149EDE700204049EAE7FAF78EFCBE
:10D7F800DAE12B78304F082B40F0A280324B2F4FC4
:10D808001978984611F00101394E23D11322304678
:10D81800F2F7C0FD0123B374364A2378137003B9B5
:10D82800B374B37C13B1344B00221A70FFF7DAFEDD
:10D838003048B17CFFF7B4F898F8003003F0FD03E6
:10D8480043F0010388F800302C4B1A7812B13A7073
:10D8580000221A703B78002B5ED0FFF7C3FE2548E4
:10D86800B17CFFF79DF8234B1A78984622B1002027
:10D8780010211F4AFFF734F82378387898F80040C9
:10D888001F4924EA030252380A70C0B21D4A23EA2B
:10D898000403012813703FD8002C37D1002B35D052
:10D8A80001230093184B01941B78124802931FE13F
:10D8B8000D17002001130020001700206816002013
:10D8C800EF160020A016002001170020F0160020F7
:10D8D800126E0208F16D0208336E0208546E0208D7
:10D8E800756E0208966E0208B76E0208D86E0208B6
:10D8F8006A160020A4160020180E0020C516002065
:10D908000E17002002170020CE160020814B04229B
:10D918009A702B7801332B707F48FFF72FF8737CB0
:10D92800002B00F041817D4A127802F08002D2B2C9
:10D93800002A00F039817A4AD3182022DA7433E1B8
:10D94800092B31D1774806F0ADFBC6B2714C2EB326
:10D95800A378042B02D10020734903E0022B04D1E1
:10D9680072490020FAF70EFB02E00BB90433A370EA
:10D97800314602226A48FAF72BFB6D4B1E78232E9C
:10D9880073D03046FAF7BAFB002800F00D81312E2B
:10D9980040F00A812B7801332B7002E03B78013389
:10D9A8003B700823A370FFE00A2B40F0FD805D4820
:10D9B800002106F04DFBC4B2002C4CD0554F7B78AB
:10D9C8003E466BB95B4BD879F7F7C6FF10B903230E
:10D9D800FB704AE0BE2010F0ADFC7B7801337B7011
:10D9E800B3784C4A092B02D90020534915E010D1CD
:10D9F800504B00241C709470504B514A494946487A
:10DA080001251C7014700C70047000950194029428
:10DA18006FE0082B04D14B490020FAF7B3FA11E064
:10DA2800062B02D100204849F7E7042B02D1002039
:10DA38004649F2E7022B02D100204549EDE70BB930
:10DA480008339370B378082B0BD835482146022247
:10DA5800FAF7BEFA05E001230093364B01941B78D0
:10DA680042E0334F3C78232C02D1FFF7E3FD9BE0E3
:10DA78002046FAF743FB002800F09680303CE4B2D9
:10DA8800631EDBB2012B3C703AD8022C294D26D1FB
:10DA9800E879F7F761FF002839D02E48FFF752FBE5
:10DAA800002834D1082246F2A8512B4801F0C5FCC1
:10DAB800284929480FF0FDFD0822274946F2A850B9
:10DAC80001F0B5FC244925480FF014FE2148012136
:10DAD800FFF7F6FA1F481949124AFFF7C9FA012356
:10DAE8000024009301942B780B480E49144A0293A2
:10DAF800124BFFF76FFAFAF709FB194B1C6053E05A
:10DB0800032C51D10B4BD879F7F726FF50BB0C23C8
:10DB1800B37049E01F0E0020A4160020302A002010
:10DB2800F20100200E170020976A0208B86A02085E
:10DB380068160020CE160020556A020869160020D3
:10DB480002170020F2690208136A0208346A020800
:10DB5800766A0208D3140020F81200205713002018
:10DB6800A01600200024124821460FF0F5FD28B128
:10DB7800E02010F0DFFB204610F018FC0134402CA8
:10DB8800F1D1082246F60A200A4901F050FC002388
:10DB9800B3702B78084A01332B70084B1A60084B76
:10DBA8001A7842F006021A7006B0BDE8F08100BF8C
:10DBB800D31400205713002084FC0108A01600206D
:10DBC800011700201FB5044611B100200B4901E0E0
:10DBD80008460B49FAF7D6F9217810220139C9B25B
:10DBE80001EB011101F5C0412231684601F025FC25
:10DBF800102001466A46FEF773FE1FBDB8490208A9
:10DC0800FA4902080B4B1B78442B06D0552B037896
:10DC180001D013B17047013B01E003780133037071
:10DC280003780BB9403302E0412B01D1403B03702C
:10DC3800FFF7C8BF681600202DE9F74FDFF8C88145
:10DC4800DFF8D4A198F80030554643F0010388F86E
:10DC580000309AF80130624C23F07F039B46D3B121
:10DC680000206049FAF78EF95F482A21F2F710FC84
:10DC780018B121788222FAF7ABF92278002A40F00D
:10DC8800AB802B6862F3CF332B60584B1A7842F085
:10DC980003021A70A0E0DFF85491237099F800305D
:10DCA8004E4603F00202D2B20192514F002A40D0F0
:10DCB80013F0010813D058464E49FAF763F93B7838
:10DCC800232B20D14C4B4D4A4D481A600121FFF7B8
:10DCD80079FF337803F0FE036BF3410312E040460B
:10DCE8004849FAF74FF93B78232B0CD1424B434A6A
:10DCF80043481A600121FFF765FF337868F3000392
:10DD080068F3410333703B782A2B65D1337803F0ED
:10DD1800FE036FF3410333702B6843F400432B6019
:10DD28000F232370364B187803B0BDE8F04F0BF083
:10DD38009BB80AF0E3FF054600282DD001213048A2
:10DD4800FFF760FF3B78532B12D13378019A03F029
:10DD5800FD0362F300033370DAF8003043F4004344
:10DD6800CAF800300F232370254B18780BF07CF885
:10DD78003B78232B30D13378002203F0FD036FF377
:10DD8800000333701E4B1A70FAF7C0F91E4A137855
:10DD980043F00603137015E01C49FAF7F3F83B78D3
:10DDA800232B19D199F8003065F3410365F300037B
:10DDB80089F80030FAF7AAF998F8003043F006031A
:10DDC80088F80030124A1378013BDBB21370114A0D
:10DDD80052F82320084B1A6003B0BDE8F08F00BF4B
:10DDE800463400203C4A0208F2010020F82C0020AA
:10DDF800681600205D4A0208A0160020A0FC010851
:10DE0800CB1600207E4A0208011700209F4A02080C
:10DE1800EF160020F0160020302A00202DE9FF41DF
:10DE28002C4D2D4C2B7843F001032B70217801F0F9
:10DE38000401C9B211B92948FFF7E4FE284E337826
:10DE4800232B21D12378274F13F004080AD0224A24
:10DE58006FF382031370244B20483B600021FFF7C7
:10DE6800B1FE11E0FAF752F92B78204A43F0060385
:10DE78002B701378013BDBB213701D4A52F8233024
:10DE88003B60164B83F800803378532B1FD12378DF
:10DE9800052243F004032370104B16491C78013CFB
:10DEA800E4B204EB840000F5C840623001F0BFFA28
:10DEB80000201149FAF766F8FF2300210093013486
:10DEC800162004220B460191029401F019FBBDE8CB
:10DED800FF8100BF01170020F82C0020CB1600207E
:10DEE80068160020A0160020BCFC0108EF160020D0
:10DEF800F0160020D8FC01081B4A02082DE9F04161
:10DF0800984B04469A7812F0010F00F017811B888D
:10DF1800002B40F01381944D95F820303F2B40F2B0
:10DF2800D780012C14D1914B1B7803F00203DBB28C
:10DF3800002B00F0C48095F820208B4B402A03D199
:10DF4800013283F82020FBE0482283F82020B6E045
:10DF5800022C03D1482385F82030B0E0844E337872
:10DF680003F02002D2B28AB195F82020402A0DD1C0
:10DF7800032C0BD07F4B804A03F1100153F8040B9C
:10DF88008B4242F8040BF9D1412395E003F01003CA
:10DF9800DBB28BB195F82030412B0DD1032C0BD07F
:10DFA800764B754A03F1100153F8040B8B4242F883
:10DFB800040BF9D142237FE0F37813F0010F0FD05F
:10DFC80095F82020422A0BD16D4B6B4A03F11001C2
:10DFD80053F8040B8B4242F8040BF9D143236BE04E
:10DFE80003F00202D2B27AB195F82020432A0BD16D
:10DFF800644B614A03F1100153F8040B8B4242F859
:10E00800040BF9D1442357E003F00402D2B27AB1E9
:10E0180095F82020442A0BD15B4B574A03F1100195
:10E0280053F8040B8B4242F8040BF9D1452343E023
:10E0380003F00803DBB28BB195F82030452B0DD1E6
:10E04800032C0BD0514B4C4A03F1100153F8040B2D
:10E058008B4242F8040BF9D146232DE00BF044FC27
:10E06800A0B14B4B1B788BB195F82030462B0DD1C6
:10E07800032C0BD0474B404A03F1100153F8040B13
:10E088008B4242F8040BF9D1472315E0F37803F0EB
:10E098004003DBB29BB195F82030472B0FD1032CFE
:10E0A8000DD03D4B344A03F1100153F8040B8B4259
:10E0B80042F8040BF9D1482385F8203078E095F828
:10E0C80020300133DBB2472B85F820307FF629AFAB
:10E0D80095F82060472E04D9234B002683F820604A
:10E0E80001E00136F6B206F14007FFB212E02B4814
:10E0F80031460FF031FB08B1032C04D1284B9B5D4E
:10E1080023B1032C02D185F820600FE00136F6B266
:10E11800BE4203D03F2EEAD9402E07D1214B1E2202
:10E128001A70402385F82030BDE8F08195F820006A
:10E138001149652246F63E33F9F762FE012C37D1C4
:10E14800194B0D4A03F1100153F8040B8B4242F8A6
:10E15800040BF9D1044B93F820303F2B3CD9002015
:10E1680012493EE010170020F2010020021300209F
:10E17800302A0020F0500208171700201151020819
:10E18800325102085351020874510208955102088D
:10E19800452F0020B6510208F8510208AC130020A0
:10E1A80062130020CC160020DCA00208AE50020842
:10E1B800104BD87800F02000C0B220B1022C06D055
:10E1C80000200D490DE0032C01D10C4909E00C4B4E
:10E1D80093F820303F2B02D800200A4901E00A4971
:10E1E8000020F9F7CFFE10200146BDE8F041F9F70D
:10E1F80079BE00BF302A0020C9470208CF50020864
:10E20800F20100206C500208D751020810B5F9F746
:10E218007DFF084B1B7803F00403DBB22BB10649E2
:10E228000020BDE81040F9F7ADBE0220BDE810405F
:10E23800FFF764BE021300209E4E020870B5214B02
:10E2480006461B78204CF3B9257819E01F48294663
:10E258000FF082FA78B123689D4202D9FF2E02D0CE
:10E2680007E0FF2E02D19D4208D202E036B91DB95F
:10E2780013B9256012E00EB9013500E0AD19EDB211
:10E288003F2DE3D90AE0013B2021114810222360E9
:10E29800F2F780F800200F49F9F774FEF9F70AFE43
:10E2A80046F63E3320780C496522F9F7A9FD084D5A
:10E2B800216805F1100001310222F9F789FE2D23AA
:10E2C800AB7470BDC1160020D8160020A616002019
:10E2D800F20100204685020817170020F8B5534BB5
:10E2E800F02253481A700378044613F00E0518D12B
:10E2F800504A43F00203156000F8013B0FF0C6F9DD
:10E308002C464D4BE35C1BB14C4821460FF00EFAEE
:10E318000134402CF5D14A4B1A7842F001021A70A8
:10E32800F8BD13F00C0543D12E46444829460FF09A
:10E3380013FA08B10136F6B20135402DF5D11EB9F0
:10E34800237843F0040331E000253E482946EFB224
:10E358000FF002FA68B1384BEB5C53B13A4B013716
:10E368001F700020FFF76AFF237843F0080323702B
:10E3780002E00135402DE8D1344D3A212846F2F724
:10E3880087F838B1401BC0B2013028183146022244
:10E39800F9F71EFE2E4B1B78532B46D12A4B002033
:10E3A8001870FFF74BFF237843F008032370F8BD7C
:10E3B8006FF34103037003F00403DBB2244D23B170
:10E3C80000202449F9F7DEFD0DE02B78552B01D10B
:10E3D800FF2002E0442B02D10120FFF72FFF13207A
:10E3E8000D21F9F77FFD2B78232B1ED1227802F01F
:10E3F8000204D4B90E4902F0FB0264F3C3020A70A6
:10E408000C4A1460F9F782FE0D4B1A7842F00602A6
:10E418001A70114A1378013BDBB213700F4A52F895
:10E4280023200F4B1A60084B1C70F8BD0D170020F5
:10E43800A5160020D8160020881E0020A616002049
:10E448000117002003130020C1160020F20100204C
:10E4580068160020C7910208EF160020F016002069
:10E46800A0160020024800210922F1F793BF00BF3F
:10E47800DD16002070B50A46002405E01B19811A34
:10E488002A2501345D54E4B20E4D0F4B295D09B1C4
:10E498009442F3D1801A001918182021121BF1F7A1
:10E4A80079FF0A4B1E785EB1432E04D10CB1013CB2
:10E4B800E4B200232B553046F9F720FE00B12E5563
:10E4C80070BD00BFDD160020F20100206816002094
:10E4D80038B5184C184DA07800F01000C0B250B9EB
:10E4E8001649F9F74FFDFFF7BDFF236843F4801382
:10E4F80023600F232B702A782AB92368FF2062F340
:10E508001453236038BD0E48C5792DB91C20082145
:10E51800FFF7B0FF284638BD23680A496FF3145344
:10E5280008222360F2F7B6F900280CBF0120FF206B
:10E5380038BD00BF302A00200F170020014F020805
:10E54800DD160020ADBB0208F0B5634D85B06E78CE
:10E5580006F01006F6B2002E3ED1604B1A78604BDA
:10E56800013A53F822305F4A934204D15E4B1A783D
:10E5780042F0020207E002F11C018B4208D15A4B1B
:10E588001A7842F00402022161F3C7021A7019E0F6
:10E598003832934216D1FFF79BFF002800F09A808B
:10E5A8000128514C06D12378022243F0010362F37B
:10E5B800C70306E030464D49F9F7E4FC237866F3D3
:10E5C800C70323704A4B1A7842F001021A702B686D
:10E5D80043F480532B607DE0434E337813F0F80406
:10E5E80006D04449002005B0BDE8F040F9F7CABCA0
:10E5F80013F0070F4FD003F00202D7B287B12146BC
:10E6080012200CF0B9FAFF2300934320214604227C
:10E6180023460194029400F073FF0094162031E021
:10E6280003F00404E4B2A4B1394638460CF0A4FA65
:10E638000BF0F6FC07F00EFD0AF088FBFF230093B1
:10E648004420394604223B460197029700F058FFC0
:10E658001DE013F0010F1AD0012143F6FA400CF027
:10E668008BFA2046F7F7DCF9234B45201C80FF2363
:10E6780000932146042223460194029400F040FFAF
:10E6880000941520214601222346F3F769FD002056
:10E698001A49F9F777FC337803F0FA036FF341036B
:10E6A8003370174B1B78232B14D12B686FF30C3363
:10E6B8002B60F9F72BFD0E4B1A7842F006021A7000
:10E6C800064A1378013BDBB21370054A52F823203F
:10E6D8000C4B1A6005B0F0BD302A0020EF16002060
:10E6E800F0160020E0FC0108CA310020224F020881
:10E6F8000117002042950208801600202195020883
:10E7080068160020A01600201FB50446F7F746FA41
:10E71800A8B14B2001F072FAFF2300930121FF3BBF
:10E728000193392004220B460134029400F0E8FEDC
:10E73800064B01205A7842F004025A7004E0044B58
:10E748001888003818BF012004B010BDE82C00203C
:10E758005C340020F0B51E4E0024337A05460133A0
:10E7680085B00F46337210202146012223460094BB
:10E77800F3F7F6FC45B9FF230093019502974F2064
:10E78800294604222B4609E0012D09D1FF230093D5
:10E7980001940297502021460422234600F0B0FE3F
:10E7A800337A052B11D1FA33012100240093272055
:10E7B8000B4604220194029400F0A2FE044B1C7242
:10E7C80005B0BDE8F04001F0EBB905B0F0BD00BF01
:10E7D800CE1600202DE9F04F9D4B87B01A78804661
:10E7E80099461AB1012A40F0DB812AE0994B1A6850
:10E7F800994B9A4200F0D681F6F78CFE974B5B78DE
:10E8080003F02003DBB223B901F0F0F908B907F0EF
:10E8180021FC934B1A686FF310421A60914B1878D9
:10E82800F9F76CFC002800F0BD81FFF71BFE8E4B4A
:10E838003C221A70F9F7A0FA99F80030013389F8E8
:10E848000030894B1C787CB9884B08F101011A7893
:10E85800204664F3C30264F304121A70C9B2FFF7C6
:10E8680079FF89F800409DE1814D404607F02AFC78
:10E87800F9F72CFB00207F49F9F784FB7E4F2B78B2
:10E88800AA46FB1813F8313C23B91B200621FFF7D1
:10E89800F1FD87E1754A0B21137804A8C3F3C0047E
:10E8A800C3F3001603F0F7036FF304131370002388
:10E8B80089F80030062200F0C0FD2A78394604A8FD
:10E8C800303AF1F78DFC074620B100274FF01209C6
:10E8D8003D4629E049F2DB4000F09EFD0028F4D0D7
:10E8E800664D2F72F6F76EFF0446002840F05A81F5
:10E8F800634A584B21461A60FF2300930190029007
:10E9080004220820234600F0FBFD012223460E20A6
:10E9180021460094F3F724FC5A4B1A7842F004027B
:10E928001A700123AB713DE14946062204A800F0A4
:10E9380084FD9AF8002004A84F49303AF1F750FCBA
:10E94800002840F01E812846FFF7DEFE002840F030
:10E958002981DFF828B101218BF808002846F6F74D
:10E968003FFF8146F6F72EFFDA46002840F0B280D6
:10E9780048464549F1F712FEB0B901F04FF8354B5A
:10E9880014B916B9414A23E036B1414A1A60414BDD
:10E998001A786FF3410205E03F4A1A603D4B1A7836
:10E9A80066F341021A70D4E048463C49F1F7F6FD97
:10E9B80020B148463A49F1F7F1FD58B9002C40F02A
:10E9C800F180002E40F0EE8001F028F8354A214B06
:10E9D8001A60BEE048463449F1F7E0FD50B949F203
:10E9E800D940012100F00EFD1D4A136843F400537D
:10E9F8001360E3E748462D49F1F7D0FD38B9002CFC
:10EA080040F0D080002E40F0CD80294ADFE748460C
:10EA18002849F1F7C3FD38B9002C40F0C380002E17
:10EA280040F0C080244AD2E748462449F1F7B6FDB1
:10EA3800002840F08E8000F0F1FF002C40D0164AEC
:10EA4800044B1A60134B1A786FF34102A9E000BF18
:10EA58009F160020A016002034FD0108F62C002087
:10EA6800302A0020681600200F170020DC1600202E
:10EA780087160020A8470208DD160020CE160020C1
:10EA880050FD0108891C0020D7BC020880FF01083E
:10EA9800080102080117002024010208A9BC020885
:10EAA80094BE020840010208CDBC0208CFBC02088F
:10EAB8007801020866BE0208CC010208D1BC02082F
:10EAC800002E6FD0394A3A4B1A603A4B1A7864F3E1
:10EAD800410266E048463849F1F760FD064620B92C
:10EAE80000F09CFF002C5DD01BE048463349F1F74D
:10EAF80055FD002856D048463149F1F74FFD38B941
:10EB0800002C4FD12F4A2A4B8BF807501A6049E046
:10EB180048462D49F1F742FD064650B9A4B100F028
:10EB28007DFF2A4A224B1A60224B1A7866F341026B
:10EB380037E048462649F1F731FD20B148462549D6
:10EB4800F1F72CFD00B96CBB234A194B1A6000F091
:10EB580065FF07F56A506E308AF8075000F05CFCD4
:10EB68008AF800009AF8070000F5D440123000F047
:10EB780053FC8AF801001948F6F76AFF402D11D1B5
:10EB880007E00135EDB20137402D09F107097FF49F
:10EB9800CBAE08F101010020C9B2FFF7DBFD01E0AF
:10EBA80000221A7007B0BDE8F08F00BF0801020804
:10EBB800A016002001170020D1BC0208CFBC020813
:10EBC80066BE0208CC010208D7BC0208240102086C
:10EBD800A9BC0208CDBC0208E8010208CE16002034
:10EBE80038B51C491C4A0B6810789C7B8442144633
:10EBF80003D99D8915F0200F18D09A8912F0800F3B
:10EC080001D105E01C3B9A8912F0400FFAD000E0D0
:10EC18001C330B60002323700B689B8913F0200FB3
:10EC280006D00E4BDA790C4B1A7001E001301070E7
:10EC38000B4A002313700B4A13700B4A136843F4F2
:10EC480080731360F9F798F8084B1A7842F00602B7
:10EC58001A7038BDA0160020C1160020CE1600205C
:10EC6800831600207D160020302A0020011700207E
:10EC780010B51D4B1D4A1978184639B11468A48976
:10EC880014F0200F02D1013919701AE0136899891C
:10EC980011F0400F01D106E01C33998911F0800F63
:10ECA800FAD0136002E011491C3B0B6013689A7B91
:10ECB80002709B8913F0200F03D00D4BDA790A4BB1
:10ECC8001A700C4A002313700B4A13700B4A13680E
:10ECD80043F480731360F9F74FF8094B1A7842F040
:10ECE80006021A7010BD00BFC1160020A016002031
:10ECF800CE160020831600207D160020302A002022
:10ED080001170020084B094A1B68934203D002F5FB
:10ED18007C72934205D1064B1878003818BF012041
:10ED280070470020704700BFA016002034FD01087E
:10ED380001130020074B084A1B68934202D038325F
:10ED4800934205D1054B1878003818BF0120704749
:10ED580000207047A0160020CC01020801130020F3
:10ED68002DE9F04F8B4B8C4D1970A0F11103DBB2DC
:10ED7800012B87B00E46287020D8122804D1874B63
:10ED88001A8842F480521A80854B00245A7821460A
:10ED980042F010025A70FF23022200933D20FE3BEE
:10EDA8000194029400F0ACFB4D2000F027FF1220E4
:10EDB8004021012223460094F3F7D2F92B78522BF5
:10EDC8000DD1F3F711FF28B9F3F702FF10B9F3F7E4
:10EDD80023FF20B1734B1A7842F008021A70724B65
:10EDE800724C1B78002B2DD12168714A914229D091
:10EDF800704A23601370704A70481178037063F387
:10EE0800C30163F3000163F3071111706C4A1178B1
:10EE180063F3010111706B4A117863F3C501117036
:10EE2800694A1370694A117863F3410163F3000179
:10EE380063F382011170664A116863F30C31116043
:10EE4800644A13702368002B40F05781604F7B7829
:10EE580003F02003DBB273B15F4B93F80080B8F185
:10EE6800000F08D149F2D940414600F0CBFA3B687F
:10EE780068F34D333B60594B187810F01E0002D0F0
:10EE88000020574907E0574B93F803809946B8F19B
:10EE9800000F05D0544907B0BDE8F04FF9F772B834
:10EEA800524F97F801B0BA46BBF1000F2BD0BBF117
:10EEB800070F14D9F8F7FEFF4D49B878652246F6D2
:10EEC8003E43F8F79DFF3878072310F003007B7066
:10EED8000EBF484940464849F9F754F80CE0BBF1E1
:10EEE800020F09D8454B5B7823B1F8F7E3FF87F8A1
:10EEF80001806AE202237B701020014607B0BDE85A
:10EF0800F04FF8F7EFBF3E4FBB795BB187F806B01B
:10EF180000F0DCFB8E20594601225B46CDF800B09C
:10EF2800F3F71EF90020F3F73BFF234A2149137832
:10EF3800344843F00603137000230B7032492360F2
:10EF48000B70324989F800300370123303FB061C3A
:10EF58009CF802C093461CF0100F884604D1304636
:10EF68000593FFF737FC059B03FB06835B7813F0DB
:10EF7800100F04D02A78133AD2B2032A4AD913F0D0
:10EF8800200F7DD02B78442B44D041D8232B41D05F
:10EF98002A2B3EE0C416002068160020DC1400204E
:10EFA800E82C0020541300200D170020A016002084
:10EFB80084FC0108EF16002001170020CB16002062
:10EFC80084160020C6160020CD160020DC1600206E
:10EFD800302A00200C17002001130020453400209F
:10EFE8000B4802081F0E0020F96E0208C816002000
:10EFF8001717002013490208F248020810170020CA
:10F00800CE160020C5160020C1160020A72B002010
:10F01800552B35D17A4B1B78002B31D1794B93F88E
:10F028000080B8F1000F2BD143F6DB2000F0F4F993
:10F03800012825D13F23FB7189F8000043F62D30C4
:10F0480000F0EAF93870F87900F5D440123000F091
:10F05800E3F978706C48F6F7FBFC9BF80030304613
:10F0680068F341038BF8003007F02CF8F9F74EF8F5
:10F07800664B67482360674BC3F800802B780370A2
:10F088002B78432B0AD15F4B1B783BB9013389F8A6
:10F098000030614B3046236007F014F828781738A1
:10F0A800C3B2072B00F291815C4908F0CDFB9AF8B6
:10F0B80000105B4B60F301018AF8001001F00301B6
:10F0C800022900F082810122032041B100900192BF
:10F0D8009B7868309B1802930021033206E0009069
:10F0E80001929B786C200133029304220B4600F0B6
:10F0F80007FAFF238AF8013067E1474A934253D160
:10F108002878A0F14303DAB2122A25D8454A5BB21F
:10F118009A4021D5432840F05881394B1B78002B61
:10F1280040F0538100F084FC3F4B40B11A78032033
:10F138001109013191FBF0F000EB400007E01A786B
:10F1480007201109013191FBF0F0C400201A091AB7
:10F1580061F307121A7038E1F8F7D0FF002823D0BE
:10F16800314F3A7812F0F00308D163F307123A707E
:10F1780023602E4B1A7842F008020EE0102B13D1B0
:10F1880000F056FC80B13B786FF307133B70002307
:10F198002360264B1A7842F0100230461A7007B0E6
:10F1A800BDE8F04FFFF716BB214B1E211A781E4E03
:10F1B80061F346021A70337813F0010F134B3DD0F8
:10F1C80022689A420DD0A3F5AC63043B9A4208D05A
:10F1D800FFF798FD28B9FFF7ADFD10B9AA30F3F78E
:10F1E800DFFD2268134B9A4202D10020F3F7D8FDC5
:10F1F8002B78522B40F0AE800F4B53221A70A9E0A7
:10F20800011300209F160020CE160020E8010208F6
:10F21800C5160020F016002034FD0108CA1600208B
:10F22800C8160020002000C001170020DC160020AE
:10F238007E170020200202086816002022689A42E1
:10F248000DD0A3F5AC63043B9A4208D0FFF75AFDF2
:10F2580028B9FFF76FFD10B9AA30F3F7A1FD2B7895
:10F26800552B16D1FFF704FD3378594F43F00603A9
:10F278003370584B9B7803F00203DBB24BB1F8F7BD
:10F2880019FE23681868FCF759F83B786FF34103B7
:10F298003B702B78442B16D1FFF7A2FC33784C4FE8
:10F2A80043F0060333704B4B9B7803F00203DBB249
:10F2B8004BB1F8F7FFFD23681868FCF73FF83B7877
:10F2C8006FF341033B702B78522B09D1337800221E
:10F2D80043F001033370404B1A70404B45321A70AB
:10F2E8003F4B00271F702B78232B33D13D4B1F70CA
:10F2F8003D4B1F70F8F7DEFD33783C4943F00603B9
:10F3080033700B78324AFBB1394A013B1770394ADE
:10F31800DBB20B7052F82330374A23609B68934264
:10F3280002D107F03FFD15E002F5D2718B4204D1FE
:10F338000120014605F044FB0CE002F505729342FA
:10F3480008D12E4B1F7005E0117863F30711117077
:10F3580023603AE02A4B1B7813B10020F3F720FD15
:10F3680023681F7B17F00F0702D1FDF789F91BE00F
:10F37800012F02D1FAF762FC16E0022F02D1FAF748
:10F388008BFF11E0082F05D84FF09C53BB4001D5E7
:10F39800FBF72EFC042F03D123689B69984703E0F1
:10F3A800052F01D1FBF7EEF9337803F00203DBB246
:10F3B8001BB123681868FBF7C1FF33786FF341036B
:10F3C80033702B780BB1064A137007B0BDE8F08F85
:10F3D8000117002010170020CB1600206816002007
:10F3E80085160020CD1600200C170020EF160020EF
:10F3F800C1160020F01600203C020208AF160020BB
:10F408001F0E002007B502AB03F8011D19460122A3
:10F41800002303F0CFFF0EBD07B5002302A901F8B2
:10F42800013D012204F02EF89DF807000EBD08B535
:10F43800002303F0BFFF002008BD034610B50846AF
:10F448001446194604F01EF8E0B210BD10B5034684
:10F45800002484540846194604F014F8204610BDC8
:10F4680037B50546002400E01446012260190DF165
:10F47800070104F007F89DF80730621C203BDBB257
:10F488005A2BF1D920463EBDF8B50024194902226D
:10F4980011F8340001EBC4014000043100F571504B
:10F4A8000134FFF7C4FF5C2CF0D143F6B6301249A3
:10F4B80004220025FFF7BBFF48F6D8272C4615E0A5
:10F4C80007EB460004EB440100B259180222FFF78B
:10F4D800AEFF0136F6B2094B5A199278B242EFD80C
:10F4E800013480370335142CBFB201D00026F2E76F
:10F4F800F8BD00BFAC280208ABBC02088C2B020880
:10F508002DE9F347044615468A46022243F6F84198
:10F518000DF106001E46BDF930909DF828809DF833
:10F528002C70FFF78AFF2F4B2F499A78BDF90600F8
:10F538008A705A7800EBC000CA701A7900F57250C8
:10F548000A715A797A304A719A791B7845EAC61550
:10F558008A710C7081F80190CB710D7200B209228A
:10F56800FFF765FF1EB1214B1A8801321A80BDF8DA
:10F57800063001339BB2B3F57A7FADF8063002D37B
:10F588000023ADF8063002220DF1060143F6F840DB
:10F59800FFF74DFFBDF80600154B188000B200EBD1
:10F5A800C00000F5725000F17A05823000B2FFF712
:10F5B80033FF10F0800F03D00C4B1A88013A1A80E1
:10F5C80028B20021FFF71EFF0A4B03F8148003EB53
:10F5D80044046770BAF1000F02D00120F6F720FA50
:10F5E800BDE8FC87D0310020E616002080160020F8
:10F5F80022260020DB2300202DE9F743324B1D781B
:10F60800303DEDB2C5F10606F6B23EB305F112077C
:10F61800402413E008F101080FFA89F000215FFA8D
:10F6280088F8FFF7EFFE09F10109B0451FFA89F9DB
:10F63800F0D1013C0737E4B2BFB21CB1B9464FF074
:10F648000008E7E70B35013428B20021E4B20135A0
:10F65800FFF7D8FEB442ADB2F5D132E0122425B29C
:10F66800684629460622FFF7E8FE9DF8003043B1B8
:10F678009DF805302BB99DF803308DF804308DF8CE
:10F6880005300734062228466946A4B2FFF7CFFEA4
:10F69800B4F5E97FE3D168460B210622FFF7CDFEDA
:10F6A8009DF8003043B19DF805302BB99DF8033023
:10F6B8008DF804308DF805300B2069460622FFF7D7
:10F6C800B6FEBDE8FE8300BF8716002010B507F020
:10F6D80069FB09F0DDFB04F0B9FB04F0DFFAF3F78E
:10F6E80093FD9D48F6F7CEF943F6D120FFF794FE37
:10F6F8009A4B9B4C187043F6D020FFF78DFE994B20
:10F70800187043F6DC20FFF787FE974B187043F616
:10F71800E130FFF781FE954B187043F6E230FFF7B2
:10F728007BFE934B187043F6DA20FFF775FE914B7A
:10F73800187043F6D920FFF76FFE8F4B187043F609
:10F74800CF20FFF769FE8D4B187043F6CC20FFF7EA
:10F7580063FE8B4B187043F6D220FFF75DFE894B92
:10F76800187043F6DF20FFF757FE874B187043F6F3
:10F77800E820FFF751FE854B187043F6DD20FFF7B0
:10F788004BFE237801280CBF43F001036FF30003FD
:10F79800237043F6E020FFF73FFE237801280CBFD3
:10F7A80043F080036FF3C713237043F6E720FFF796
:10F7B80033FE774B01281A6843F6EA200CBF42F063
:10F7C80000526FF35D721A60FFF726FE6378012816
:10F7D8000CBF43F001036FF30003637043F66E211F
:10F7E80011226C48FFF729FE6B4800210322F0F72D
:10F7F800D1FD00246748235C312B03D122302146F8
:10F808000DF094FF0134112CF4D1224643F6F61181
:10F818006048FFF712FE224643F63A215F48FFF799
:10F828000CFE47F2740104225D48FFF706FE47F21A
:10F83800780104225B48FFF700FE0AF06DFEF6F738
:10F84800F1FB43F6E120FFF7E7FD574C237860F31F
:10F858000003237043F6E220FFF7DEFD237860F310
:10F868004103237043F6E420FFF7D6FD237860F3C5
:10F87800C303237043F6E620FFF7CEFD237860F339
:10F888004513237043F6E920FFF7C6FD237860F39C
:10F898008613237043F6E520FFF7BEFD237860F357
:10F8A8000413237043F6EB20FFF7B6FD237860F3CB
:10F8B800C713237043F6E320FFF7AEFD237860F308
:10F8C800820323703948FFF7A7FD394B1870394870
:10F8D800FFF7A2FD384B18703848FFF79DFD384BED
:10F8E80018703848FFF798FD374B18703748FFF7FE
:10F8F80093FD374B18703748FFF78EFD364B18705D
:10F908003648FFF789FD364B18703648FFF784FDF7
:10F91800354B18703548FFF77FFD354B1870FFF7EA
:10F928006BFE3448FFF778FD334B18703348FFF708
:10F9380073FD334B18703348FFF76EFD324B187068
:10F948003248FFF769FD324B18703248FFF764FD03
:10F95800314B187010BD00BF9B1600201A0E0020F6
:10F968007E170020190E00201C0E0020E412002033
:10F97800DA1000205E34002000000020C8140020A7
:10F98800861600201B0E00205B2B00208C2A0020EE
:10F99800302A00203D2C00205F2C00204E2C002017
:10F9A800482A00205E2A0020B5140020CE8AFFFFD6
:10F9B800452F0020CF8AFFFF722E0020D08AFFFF3C
:10F9C800422F0020D18AFFFF432F0020D28AFFFF59
:10F9D800742E0020D48AFFFFEB2D0020D58AFFFF6C
:10F9E80038180020DC94FFFF49150020DA94FFFF47
:10F9F8008716002014A2FFFF1B2A00208FA1FFFFFB
:10FA0800B524002091A1FFFF2026002090A1FFFF30
:10FA18001B260020858AFFFFC41C0020034B1E21E3
:10FA28001A7861F346021A70704700BF7E170020EB
:10FA3800024B187800F00100704700BF7E170020C5
:10FA4800014B1878C00970477E17002008B5FFF7EA
:10FA5800F7FF38B9044B1B7813F07E0F0CBF00205A
:10FA6800012008BD012008BD7E170020F8B546F624
:10FA7800AA742046FFF7D0FC2D2803DD20462D214F
:10FA8800FFF7C0FCA4F55856123E3046FFF7C4FCF9
:10FA9800414FC0B207EBC0000579C5F30015A5B901
:10FAA8000DE03D4B3D4953F83500F0F777FD20B99F
:10FAB80030462946FFF7A6FC07E00135EDB207EB13
:10FAC800C5031B7913F0080FEBD0013446F6EA732F
:10FAD8009C42CED143F6C4242046FFF79DFC2D2836
:10FAE80003DD20462D21FFF78DFC013443F6CC239E
:10FAF8009C42F1D1012143F6E120FFF783FC01216B
:10FB080043F6E220FFF77EFC012143F6E420FFF7ED
:10FB180079FC012143F6E620FFF774FC012143F646
:10FB2800E920FFF76FFC012143F6E520FFF76AFCA7
:10FB3800012143F6E320FFF765FC012143F6EB20A2
:10FB4800FFF760FC002143F6E020FFF75BFC002193
:10FB580043F6EA20FFF756FC002143F6EC20FFF7B6
:10FB680051FC012143F6DC20FFF74CFC002149F24F
:10FB7800DB40FFF747FC48F644200121FFF742FC31
:10FB880047F252042046FF21FFF73CFC013447F2BC
:10FB98005A039C42F6D1F8BD08040020929F02083F
:10FBA80010B506F041FA09F03DF9074B4FF416720B
:10FBB8001A80012147F26200FFF724FC4C20BDE8BF
:10FBC800104000F01BB800BF5C34002010B506F0F0
:10FBD80041FA09F0BBF8044B002147F26200198092
:10FBE800BDE81040FFF70EBC5C340020024B1888BB
:10FBF800003818BF012070475C340020542873B5C2
:10FC0800044663D83D4BDB7803F02003DBB2002BBE
:10FC180072D13F2801D80EF0B5FB394D35F8146084
:10FC2800002E69D1E10001F5D8416846B2310822B9
:10FC3800FFF703FC334821460DF08EFD50B1F3B2B7
:10FC4800072B07D03F2C05D80122B240D243D2B2AD
:10FC58002D4B27E01DF806300122542B08D0562BD7
:10FC680003D0532B284B1AD100E0284BB24007E0B1
:10FC7800B240254BD2B2195D42EA01011955234B16
:10FC8800195D0A431A55FFF7D3FE98B1204B1B782C
:10FC980083B13F2C0ED81E3325F814300AE0B24049
:10FCA800D243D2B2195D02EA01011955174B195D09
:10FCB8000A401A550136082EBCD1134B1A5D134B56
:10FCC8001B5D134318D125F8143015E0C10001F568
:10FCD800D8416846B2310822FFF7AFFB00231DF870
:10FCE80003202D2A05D001219940074A105D0143C0
:10FCF80011550133082BF2D17CBD00BF302A0020FA
:10FD08008217002010200020DA1B0020351A00205E
:10FD1800461500201FB500F017FD10B900F028FDAA
:10FD280048B10021FF2300930B2004220B460191C8
:10FD38000291FFF7E5FBAD220023D9B24D2909D086
:10FD4800012A07D90D48002119540D4819540D48A6
:10FD580020F8131001330132552BD2B2EDD1074BE5
:10FD6800002183F85510084B08481970084B0822E1
:10FD7800197005B05DF804EBF0F70CBBDA1B002036
:10FD8800351A0020821700209918002078180020C2
:10FD98008017002059B1064B0C2202FB0030437A31
:10FDA800C918837A417208300BB93C3383707047A5
:10FDB8005C200020072811D9094B1B5C022B0DD1B0
:10FDC8000838C0B2C308012100F0070011FA00F09A
:10FDD800044A0133D15C41EA0000D054704700BFA7
:10FDE800881E0020D42A0020044B0C2202FB00337A
:10FDF8000C3A5A729A72FFF7DDBF00BF5C200020F0
:10FE080010B50446FFF7F0FF034B0C2202FB043445
:10FE1800FF23637210BD00BF5C20002070B5104D39
:10FE2800002410482146E6B20DF096FC98B96B7A8A
:10FE38008BB10D4AA318A25C93F88030022A0AD02D
:10FE4800413BDAB2122A06D8084A5BB29A4002D578
:10FE58003046FFF7C9FF01340C35402CE1D170BDA5
:10FE68005C200020B6140020881E00200020008896
:10FE780010B50A4B0C2203EBD00393F88011084B02
:10FE880002FB00331C7A3CB900F0070051FA00F07D
:10FE980010F0010F18BF1A7210BD00BF881E002095
:10FEA8005C200020044B0C2202FB00331A7AFF2A44
:10FEB80001D1FF3A1A7270475C200020104B1B7862
:10FEC80013F0010F02D10F4B187818B10E4B03F540
:10FED80040720CE00C4B03F54072197A0C3301396F
:10FEE800C9B2FD2998BF01209342F6D17047197A0B
:10FEF80009B1FF2119720C339342F8D100207047E1
:10FF0800DC140020461500205C20002030B5044693
:10FF18001048007800F00200C0B2C8B10C2060435D
:10FF28000D4D285C904201D1994207D0984201D1E9
:10FF3800914203D0052A0BD1052B09D10C2303FBD1
:10FF48000455064821462B72BDE830400DF0F9BB38
:10FF580030BD00BFA51600205C200020A61600209A
:10FF68001FB50446214614480DF0F6FB002821D0A1
:10FF78000122022300210093A31802935C200B4660
:10FF88000192FFF7BDFA21460B480DF0DAFB214636
:10FF98000A480DF0D6FB214609480DF0C7FB074B70
:10FFA800E40804F5CA40195DA83004B0BDE8104063
:10FFB800FFF728BA04B010BD3C13002057130020E7
:10FFC800B61400202DE9F7438E480DF05FFBDFF8EB
:10FFD80058828D4E0024E5B2284603F0E1FF18F858
:10FFE800019F074618F8403C13B1022B3ED10FE0A1
:08FFF8002846FFF7F9FE21463F
:020000040801F1
:1000000084480DF0A2FB214683480DF09EFB21465B
:1000100082480DF09AFBC9E028464946F5F788F872
:1000200010B12846FFF7EEFD737AFF2B01D1FF3B9D
:100030007372737A4B4501D2F37A9BB173482146B0
:100040000DF078FBF37A002B40F0B080204604F0EE
:10005000D7FA052128460A460B46FFF75BFF2846DC
:10006000FFF7C6FEF37A002B40F0A0802846FFF78A
:100070007BFF9BE090B92846FFF7BAFE2146634814
:100080000DF058FB28463946F3F7B2FB002800F084
:1000900086803378002B00F082803AE0022814D169
:1000A0005A4821460DF046FB3378012B01D0737A74
:1000B0001BB928460121FFF771FE28464946F5F78E
:1000C00037F800286BD0284626E003280FD12846B1
:1000D000FFF78EFE21464D480DF02CFB28460121EE
:1000E000F3F786FB00285AD03378032B10E004285E
:1000F00015D12846FFF77CFE214644480DF01AFB37
:1001000028460221F3F774FB002848D03378042BEB
:1001100045D0052B43D04520FFF774FD3FE0012873
:100120003DD1737A4B4502D32846FFF761FE214645
:1001300038480DF00AFB214637480DF006FB2146F2
:1001400036480DF002FB2846FFF7B0FE3378012B4E
:1001500025D0052B23D02846FFF706FF33780BB1B7
:10016000032B07D12E4821460DF0FAFAB8B12046EC
:10017000012108E0042B09D12A4821460DF0F0FAAC
:1001800068B120460221F2F7E7F908E02648214647
:100190000DF0E6FA18B120460021F2F70DF92846D5
:1001A000394601220223FFF7B5FE37702146174872
:1001B0000DF0D6FA013401462846F5F7FDFB0C3662
:1001C000402C7FF40CAF194D09F05EFF2C68D4B9B8
:1001D00043F6D320FFF724F9C6B29EB14320FFF7C0
:1001E00011FD21460122234608200094F1F7BCFFAF
:1001F00001230E20214622460094F1F7B5FF4FF46B
:1002000061635E432E60BDE8FE8300BFD21B002009
:100210005C2000206C1E0020741E00207C1E00202C
:10022000031300203E150020E61400205C1C002073
:10023000C71E0020324AF8B59042054601D000237F
:100240001FE0304B1C78005D002808BF002401E04F
:100250000134E4B28C4207D2105D0028F8D02A485D
:1002600030F814000028F3D18C4201D1002242E082
:100270002649087808B9125D0A701C700B780EE0E8
:100280000133DCB28C4207D2EA5C002AF8D01E4A65
:1002900032F81320002AF3D18C422DD02B5D00269A
:1002A00013F0010F05D10136F6B2082E01D05B081C
:1002B000F6E7174F00213E702122164806EB06167E
:1002C000F0F76CF806F51671124801312022FFF79D
:1002D000B8F8387800F046F978B93B78012212FA7C
:1002E00003F3295D21EA03032B553978074B8A4034
:1002F000197821EA02021A70FF242046F8BD00BFD7
:10030000351A0020230E00208217002080170020BD
:100310009D1800203E18002070B50E46C11EC9B2BF
:100320000123002407E002FB03440A22534301385F
:10033000A4B2C0B2DBB230B1325C303AD5B2092DD2
:1003400001D88842EFD1451C202106221648F0F73B
:1003500025F8092CEDB204D9632C8CBF00230123AE
:1003600009E0022307E011490135C918013381F87A
:10037000A320DBB2EDB2052B09D8725DA2F13001EA
:10038000C9B20929EFD92C2AEDD02E2AEBD046F696
:100390000920FFF745F8844204DA5520BDE8704093
:1003A000FFF730BC70BD00BF6F1D0020CC1C0020CB
:1003B000F0B587B00446F0F741FA47F26301C5B2E1
:1003C000102201A8FFF73DF89DF804300BB1202B57
:1003D00003D1234B1E78022E08D9204601A9F0F73D
:1003E00065FC0746002838D001A80BE01D4B06EB42
:1003F0000616F61820463146F0F758FC0746002846
:100400002BD03046F0F71AFA3F1837B33F1B1DE0E8
:10041000E35D2C2B01D02E2B17D1E31913F8012CFF
:10042000303AD2B2092A10D85B78303BDBB2092BC4
:100430000BD80D4B1B7803F00803DBB263B1013F0F
:10044000F8B22146FFF768FF06E00137FFB26B1EE6
:100450009F42DDDB002700E00127384607B0F0BDF2
:10046000410E002000470208CC1C002008B50449BA
:10047000F0F798F8D0F1010038BF002008BD00BFA8
:10048000431C0020044A00231370044A1370044ADA
:100490001370044A13707047492F0020751C002008
:1004A000741C00208A1A002038B51C4B1C4A19788D
:1004B0001C4B19B100201870107038BD12789AB911
:1004C000194A107870B1194A117801F04004E4B269
:1004D00044B91C78844205D141F040011E2060F3EC
:1004E0000501117000221A701C7894B10F4B1D7811
:1004F00005F04005EDB22DB943F6D520FEF790FF8B
:10050000844208D10A4B01201A7860F301021A7064
:1005100038BD204638BD284638BD00BF751C0020B8
:100520008A1A0020492F002038180020442F00206C
:10053000762E002010B5F7F7C1FA084B00211A6893
:10054000074822F002026FF382021A601122EFF7CD
:1005500025FFBDE8104002F0DDBD00BF302A0020BD
:10056000311C0020F8B5344D07462B78A3F130023A
:10057000D2B2092A0CD92B2B0AD0002404E02E4B2E
:1005800020221A550134E4B22B5D202B02D106E063
:10059000002404E0002BF2D101E00134E4B22E5D2E
:1005A000202EFAD0254800211122EFF7F7FE002E69
:1005B0003DD0A6F13003DBB2092B02D8204A00203F
:1005C0000DE02B2EFAD00020F8BD013002F8013FDB
:1005D000C0B220232B5501341028E4B20FD02B5D7C
:1005E00033B1A3F13001C9B20929EED92B2BECD0DC
:1005F00028B9F8BD104B20221A550134E4B22B5D06
:10060000202B04D0002BF5D101E00134E4B22B5DA6
:10061000202BFAD00B4C0023072F237009D807F5A5
:1006200066505830FEF7FCFE20700120F8BD3046C1
:10063000F8BD0120F8BD00BF3E180020311C00208D
:10064000301C00202C18002038B540F25925002419
:100650000C4829462022FEF7FDFE2046FFF782FFC8
:1006600040B10948FFF702FF20B1012010FA04F45D
:10067000E0B238BD0134E4B21135082CE8D10020D5
:1006800038BD00BF3E180020311C002070B52A4B39
:100690002A4C1B7823B12A4B00201870207070BDA3
:1006A0002378ABB9264D2B78012B00D100BF013B3D
:1006B000DBB2012B0AD802F025FD01462148F0F7F4
:1006C0005FF8FFF7C1FF08B107F08CF800232B702B
:1006D0001D4B587800F00200C0B200282AD01A68DA
:1006E00043F6D5206FF349221A60FEF799FE144DA8
:1006F000C6B22B780BB902F0E5FC06239EB123703D
:100700002B780133DBB2B3422B7012D10F4B1A7826
:100710006FF301021A7002F0F5FC01460948F0F788
:100720002FF8012070BD23702B78304601332B70D9
:1007300070BD002070BD00BF492F0020741C002038
:10074000751C0020431C0020981C0020762E0020E1
:100750000023074A184632F8021F11B90549595CAF
:1007600008430133572BF6D1003818BF01207047DA
:1007700080170020DA1B00200023074A184632F8B1
:10078000021F11B90549595C08430133552BF6D1B5
:10079000003818BF0120704780170020351A00204C
:1007A00038B50C461546F0F749F8C0B207E0054BDE
:1007B0001A181B5D1219013C02F8013CE4B2AC426C
:1007C000F5D838BD8E320020F8B506460C460846EE
:1007D0001746002110221D46EFF7E0FD3278174B37
:1007E000002013F8011F914206D12146102246F63F
:1007F000A243F7F709FB12E001300428F1D10023EE
:1008000031211A463078184110F0010F02D0A1545E
:100810000132D2B201330131082BC9B2F2D13946CB
:100820002A462046FFF7BCFF0646054821464019E8
:100830003246EFF70BFD3046F8BD00BF9A16002098
:100840008E32002030B50378A121594301F538716B
:1008500085B00131A0221248FEF7FCFD1048EFF7E9
:10086000EDFF0024C5B217E00D4B1B5D242B01D119
:100870000C4806E0262B01D10B4802E0402B09D1A1
:100880000A482A4623466946FFF79EFF4519EDB2FE
:10089000041900E00134E4B2AC42E5D305B030BD48
:1008A0008E320020D2140020601300205F1300203D
:1008B00070B5244A03780546D31893F88030542B3A
:1008C00005D121482149EFF75BFF002405E0462BC5
:1008D0001D480CBF1E491F49F5E72878800000F528
:1008E000D6403E302018FEF79BFDC6B246B31648F0
:1008F000EFF7A4FFC0B29F281BD8013EF6B21D2E11
:10090000114B4FEA061108D8891901F5144118183E
:10091000EE311122FEF795FD0BE00F4A8919891877
:10092000181801F1100351F8042B994240F8042BD8
:10093000F9D1054809490134EFF78AFD042CCCD1DF
:1009400070BD00BF881E00208E320020A2800208E9
:10095000C380020881800208FF9E0208CBBC020807
:1009600038B52C4D2B782C46012B16D002D3022BF8
:100970004BD138E057212848FFF75CFC274BFF2874
:10098000187045D026482749EFF7FAFE264B1A780B
:10099000264B1A702B7801332B70214801F09CFBF9
:1009A000002836D01D4803783F2B02D8FFF780FF80
:1009B00010E0A3F15202D2B2022A02D8FFF742FF9E
:1009C00008E0A121594301F5387119480131A022ED
:1009D000FEF740FD16481749EFF73AFD237800204F
:1009E0000133237038BD01F097FB90B10F4901200E
:1009F0000978002310FA01F12B70084B064A1B7886
:100A0000D45C24EA0101D15438BD0020287038BDDF
:100A1000012038BD240E0020DA1B0020331A0020EC
:100A200088180020311C00209D1800209A180020F2
:100A30008E320020D3BC020808B502F089FA18B93A
:100A4000074B05225A7008BDF7F706F8232804D192
:100A5000034B07225A70233808BD012008BD00BF90
:100A6000240E002038B50124844000210A480B22BE
:100A7000EFF794FCE4B20025084BEB5C1C4207D076
:100A8000074B33F815301BB9034829460CF052FECA
:100A90000135552DF0D138BD2D180020351A002014
:100AA0008217002070B5012585400024EDB20A4868
:100AB00021460CF055FE20B1084BE25C22EA05020B
:100AC000E2540134552CF2D1034800210B22BDE839
:100AD0007040EFF763BC00BF2D180020351A0020CE
:100AE00010B50B4A137813F001000FD0094903F039
:100AF000FE0309780848002413F0040F44541370CF
:100B000003D0FFF70BF9012010BD012010BD00BF7D
:100B1000CE1B00203A1800207818002070B586B04F
:100B2000F6F79AFF002800F09A804E4B4E491A784B
:100B300088540132D2B2072A1A7001D907221A70DA
:100B40004A4E1A783378303B9A42C0F28580454B42
:100B500000221A7043F6E410FEF762FCC4B214B926
:100B60001224002509E0FFF76FFD10EA0401F7D118
:100B700008223D48EFF712FC70E00021072204A88C
:100B8000EFF70CFC0622214604A8FEF75AFC327847
:100B900004A8303A3449EFF781FE10F0FF0F38D146
:100BA0002846FDF7B5FD0146002857D104A80722C5
:100BB000EFF7F4FB2846F4F7D3FE20B92846F4F704
:100BC000E5FE00284AD02A4C002108222648EFF7EB
:100BD000E5FB0021FF2325700422009301350B461D
:100BE0001C2001910295FEF78FFC2078214D00F525
:100BF0006A506E30FEF714FC2870207800F5D4405F
:100C00001230FEF70DFC68702846F4F725FF02202D
:100C100025E00135EDB20734402DAED10021072289
:100C200004A8EFF7BBFB062240F2522104A8FEF70E
:100C300008FC0E4B0C491A7804A8303AEFF72EFE48
:100C40000021044608220848EFF7A8FB14F0FF0F24
:100C500014BF0120052002E0032000E0012006B0BF
:100C600070BD00BF611C0020801800208716002086
:100C700064180020CE160020044B054A1B784FF460
:100C8000416101FB032318180DF0E2BA861600201B
:100C9000E0AE0208024800214FF4C172EFF77EBBBC
:100CA000B018002010B504460548EFF7C7FD80B224
:100CB000B0F5C17F01D3013880B2014B1C5410BD87
:100CC000B01800202DE9F041FFF7E4FFA92646F611
:100CD00042350024174821460CF042FDE0B1E3B252
:100CE0003F2B16D8144BE31893F88030542B01D1C6
:100CF000FB2000E02520FFF7D5FF2F1F3846FEF729
:100D00008FFBC0B240B10137FFF7CCFFAF42F5D146
:100D100002E03046FFF7C6FF013401360435552C9A
:100D2000F6B2D7D1FC20FFF7BDFF0448BDE8F04183
:100D30000DF08EBA2D180020881E0020B01800205B
:100D4000F0B5734C85B06378072B00F27881DFE84B
:100D500013F00800370057008500C7000701300175
:100D6000690155216B48FFF765FA6B4BFF28187036
:100D700000F06A8169496A48EFF702FD694B6A4AE7
:100D80001D78012313FA05F01178684E40EA01013D
:100D90001170674A674F11786370674A735D3D70E1
:100DA000117023B943F6E010FEF73AFB7055634B20
:100DB0009B7803F02003DBB213B13B780122F2549D
:100DC0005C4B1878FFF74EFE5D480B210CF0A5FC3C
:100DD000F8B95C4B1B78002B40F03681504802F08C
:100DE00077F8002800F033814D495748EFF7C8FCE9
:100DF000022343F6E3106370FEF712FB534B1870A7
:100E00004C4B1878FFF72EFE4D480B210CF085FC5B
:100E100008B1062379E002F09BF8E0B102F0C2F8D5
:100E2000484D10B1494B1B782B702B780BB901F052
:100E30002BF902F0E7F8002800F009810323637022
:100E4000F6F73CFE43F6E210FEF7EAFA404B187064
:100E500002232B70FAE006236370F5E0FFF7ECFD48
:100E6000002800F0F480374B1B78002B40F0EE8018
:100E7000304B1878FFF7F6FD364B1D7815F003055B
:100E800023D104F0BDFF002800F0E18004F09AFFB8
:100E9000002800F0DC800AF003FF002840F0D28038
:100EA0002D4B93F8292093F82A1042EA012193F858
:100EB0002B2041EA0241024661F31702D3F82100D8
:100EC000D3F82510032304F05DFF244B1A7842F079
:100ED00014026FF345121A70FFF7F4FE042314E0B6
:100EE000FFF7AAFD002800F0B2800DF0E3F900281A
:100EF00040F0AC80164B1A780AB1013A1A701B7890
:100F000073B3104B02221A70032363709EE000BF7C
:100F1000240E0020351A0020321A0020311C002037
:100F20009F1800209D180020991800207818002094
:100F30002C1800203A180020CE1B0020302A002058
:100F40002D1800203D180020431C0020CF1B00203E
:100F5000601C0020762E00204C0C002084390020DC
:100F60003C4D0DF0C9F92A78012111FA02F23A4BF1
:100F70003A4E197821EA02021A70337803F0050319
:100F8000042B01D1FEF7CAFE337813F0010002D121
:100F90002A783349885403F00303022B04D1314BE0
:100FA0001A7842F010021A7001F0D2FF08B9062335
:100FB000637043F6E110FEF733FA264F2A4B284AB6
:100FC00018703B78D15C09B10139D154012515FA6B
:100FD00003F62649D25C087820EA06000870CAB9F0
:100FE0001D4E3178194111F0010F10D05B19FF210E
:100FF00000910192029329462B463B200332FEF7D3
:1010000083FA3B789D40337823EA050535703878BC
:10101000FFF748FD0023637001F0F4FFA0B901F071
:1010200033F811E00DF068F905236370FFF758FD00
:1010300060B90C4B1A7842F008021A7007E00020E1
:10104000607004E0284602E0012000E0002005B0C6
:10105000F0BD00BF3A18002099180020CE1B0020D8
:1010600078180020D11B00203D1800208017002098
:1010700008B5074B4FF441611A78064B01FB02316A
:101080004FF4C17209180448EFF7E0F808BD00BF3B
:1010900086160020E0AE0208B018002070B53B4C68
:1010A0002378032B67D8DFE803F0020A1946384B90
:1010B00003221A7001232370364B033A1A70344B03
:1010C0001B78002B5AD0344B1A7842F001021A7068
:1010D00023780022013323702E4B1A700DF0EAF8AA
:1010E00010B12E4B0A221A702B4D2B7813F0010FE2
:1010F0000CD00DF0DFF8064640B9FFF7BDFD2B78A8
:101100000A2266F300032B70244B1A70FFF706FDCA
:10111000032805D10DF0F0F82378013323702FE078
:101120001E4B187800282BD1194B1A78013A1A70E7
:101130000123237070BDFFF7F1FC184B05461B78A7
:101140000BB1012809D14FF4C170FFF795FD104B89
:101150001A78013A1A7001232370022D12D0052D3E
:1011600012D1FFF797FDBF20FFF79CFD0C480DF053
:101170006FF8FEF7D3FD0020207070BD012070BD18
:10118000002070BD284670BD002070BD3C180020B6
:101190009C180020611C0020D11B0020621C002034
:1011A000B01800200A4A13783BB1013BDBB2137040
:1011B000084A52F82320084B1A60084B08481A784E
:1011C00000216FF300021A704FF4C172EFF7E6B816
:1011D000341A0020641C0020601800203C390020D4
:1011E000B01800202DE9F0413A4D3B4F2B7823B940
:1011F0000DF060F808B103233B703B78002B62D1FF
:10120000364C2078002862D00DF054F800285DD1CB
:101210002B78FF2B07D12F4B1870FFF7C3FF2E4AF7
:10122000032313702370DFF8C8802D4E98F8003028
:10123000002B27D040460DF00BF800214FF4C1726F
:101240004046EFF7ABF8274A33681146934205D082
:10125000254A934202D0FF232B7034E025781F4AA1
:101260000120002D33D08B4204D1107001380CF0D6
:101270004BFB1CE01C498B4219D1107000200CF074
:1012800007FD14E02B78142253433268DFF84480C2
:10129000D118097979B9154B1B7823B14FF44170F6
:1012A000FFF7EAFC01E005233B7000232B70237855
:1012B000013B237007E0D058FFF7DEFC98F80030C0
:1012C000013388F800300120BDE8F0810120BDE83D
:1012D000F08100BF421C0020621C0020CD1B0020BA
:1012E00060180020580F002020100020341A002021
:1012F000B018002030B50F4A0F4913780D680F4C15
:101300008068022B44F82350086001D80133137021
:101310000B4B984204D10020BDE830400CF0F4BAE9
:10132000084B984204D10020BDE830400CF0B0BC1E
:1013300030BD00BF341A002060180020641C00205B
:10134000580F00202010002010B5154B1B6819798C
:10135000022903D113490870184617E012498B423D
:1013600003D1BDE810400CF0DDBB10498B4203D126
:10137000BDE810400CF022BD142101FB00321379AE
:10138000012B02D0032B0AD104E01046BDE8104027
:10139000FFF7B0BF034913690878117B984710BD68
:1013A00060180020D01B0020580F002020100020C3
:1013B0001D4BF7B51B68002504E01A7B14339542DA
:1013C00038BF15461A79002AF7D16846F6F78AFB26
:1013D000044608B1F6F772FB0DF1FF3620E0134B1F
:1013E00003221A70124A00231370124A16F8017F62
:1013F00013700CF081FF232F02D1FFF7D3FE11E011
:10140000303FFFB237B1AF4204D8013FF8B2FFF727
:101410009BFF07E0013C40F28640E4B2FFF728FE64
:10142000002CDCD10120FEBD60180020CD1B002067
:10143000621C0020421C002010B5104B00241A78BA
:1014400021466FF300021A700D4B0E4A1C700E4BB2
:101450000E481A600822EEF7A1FFFFF71BFC0C4BA9
:10146000FF221C700B4B1C700B4B1A700B4BFC3A81
:101470001C700B4B1A700B4B1C7010BD3C390020BC
:10148000D11B002010BC020860180020801800202A
:10149000611C0020621C0020421C00203C1800201F
:1014A000CD1B0020341A002070B5364CA378042BD5
:1014B00060D8DFE803F00320334E57000123A37008
:1014C000314B1B7803F00802D2B212B12D4A02212F
:1014D000917003F01003DBB203252C4E2BB1FFF704
:1014E000ABFF0020A570307070BDFFF7A5FF284B43
:1014F0001D700A233370254D287800282CD0F6F76C
:10150000ABFA232839D1FFF7EBFA20B100200523ED
:1015100060702B7070BD02232870A370FFF7BEFDB2
:10152000012803D10423A370013870BD022826D1FD
:10153000FFF7B0FB154B00251D700323A370154B5F
:101540001878F4F723FAD8B1134A144B28461A60D6
:1015500070BDFFF747FE10B90423A37070BDFFF7FD
:1015600027FF0AE000F090FD0CF0C6FE0023A370F8
:10157000012070BD0020A07070BD002070BD002053
:1015800070BD00BF240E0020D11B0020621C002073
:101590009C1800206418002060BC0208601800201D
:1015A0002DE9F041884D894C2B6826466FF3DB63AB
:1015B0002B6023786FF34513237001F0CFFD58B1F2
:1015C000834B1B7843B10220072106F05FFA237892
:1015D00043F02003237010E001F0A4FD90B17D4B97
:1015E0001B787BB97A4B1B7863B10220012106F08E
:1015F0004DFA337843F0200333702B6843F00063D7
:101600002B6010E008F074F910B10220012108E00D
:10161000297801F01001C9B211B10220014600E0A1
:10162000022006F033FA6C4C2378082B00F21C835E
:10163000DFE813F009001E002B0136015A017A0180
:10164000E60109020A030BF0E1FB08F007F9FEF7D7
:1016500071FFFEF717FF614B00229A700123237080
:101660005F4880210DF073F804F0D2FB0CF052FEBD
:10167000FF205C4E014608F069F9337803F00A0256
:10168000082A06D003F00502042A02D013F0300F16
:101690000DD0554B1B7803F00203DBB20BB104F005
:1016A000B7FB337803F0D3036FF304133370AB78D5
:1016B00003F00203DBB24BB1082323704B484C4BC1
:1016C0003C221A70BDE8F0410CF0C2BD494E33789F
:1016D00003F04003DBB223B908F022F9002800F040
:1016E000C382FEF7E1FE10B9FEF7D0FF70B101F042
:1016F000A1FC414B1A7842F008021A70374B0022C5
:101700009A70052323703D4B02321A706B7803F0F8
:101710000203DBB25BB1337803F04003DBB233B1D9
:10172000374B1A786FF301021A70062308E0FFF7AF
:101730000FF840B1337803F04003DBB21BB1022352
:101740002370BDE8F081F0F7C5FF2E4DFF2828700B
:1017500029D02D4B1B78002B40F08682012212FAF3
:1017600000F02A4B1A781043187043F6DF30FDF76B
:1017700057FE274B1870274808F00EF8204B1B78AF
:1017800003F00303022B00F06F822978224801EB5B
:10179000011101F56C5107232E3110222370BDE891
:1017A000F041FDF757BEFEF7E7FF002838D01B4891
:1017B00007F0F2FF124B1B7803F00303022B00F03B
:1017C00053820323BCE700BF302A0020E82C00200E
:1017D000C41C00204B34002077180020240E002069
:1017E00000100140843900201D2A00208B1A00209F
:1017F00062340020981C0020D11B002039180020E2
:10180000762E00203B1800209E180020E1120020B8
:101810009B180020422F0020311C0020722E002037
:10182000984B994C5A7860F386125A70257805F0D7
:101830001003DBB2002B00F01782337803F0400373
:10184000DBB2002B00F01082904B1B7833B963F3AE
:10185000041563F301052570BDE8F08115F00C0552
:1018600040F002822946062204F1A300EEF796FD1D
:10187000A01C2946A122EEF791FDF0236370237886
:1018800043F0040365F304135AE70221FF2008F034
:101890005DF8FFF765F8002800F0E68100234FE7C8
:1018A0007B4B1B7823B17B4B5B78012B3FF448AF1C
:1018B000794B1B7803F00303012B02D10220FF2197
:1018C00001E0FF20022108F041F8FFF739FA002873
:1018D00000F0CA8101F096FB002800F08E806D4B6D
:1018E00000229A70042323706B4B1B7803F00303D0
:1018F000012B02D10220FF2101E0FF20022108F08C
:1019000025F801F07FFB20B1FFF7CEFD002800F0A5
:10191000AB8101F077FB08B900F0B6FB0023237020
:10192000BDE8F0410CF0E8BC5B4D2B7803F00303FD
:10193000012B02D10220FF2101E0FF20022108F04B
:1019400005F804F05DFA002800F08E8104F03AFA00
:10195000002800F089810AF0A3F9002840F0848172
:101960002D784E4905F00305012D19D191F82A2053
:1019700091F8293043EA022391F82B2043EA0243ED
:1019800000F07F421A43D1F821000D23D1F8251031
:1019900004F0F8F9424880212A460CF0D8FE13E002
:1019A00091F82A2091F8293043EA022391F82B205C
:1019B00043EA024300F07F421A43D1F82100032397
:1019C000D1F8251004F0DEF9364B1A7842F01402F3
:1019D0006FF345121A702F4B00229A7001F012FB20
:1019E00030B1314B1B78002B40F03E810433A7E629
:1019F00001F038FB002840F037812070BDE8F0810D
:101A00000221FF2007F0A2FF284801F061FA01F04F
:101A100041FB10B9264B05221A7001F03BFB20B99F
:101A200001F096FA002840F01F81214B1E78002E0D
:101A300040F01A812B6866F349232B6000F024FBE9
:101A40002670BDE8F081144E337803F00303012BB8
:101A500002D10220FF2101E0FF20022107F076FFE2
:101A6000144B1F7867BB144D01222878134B82401A
:101A7000197821EA02021A70F0F75EFE2F702770C3
:101A8000BDE8F081702E0020CC1C0020C41C00207A
:101A90003D180020240E0020762E00204C0C002043
:101AA00000100140843900203918002066180020F9
:101AB00065180020311C00203B180020E112002096
:101AC0006A4B1A78984602F02002D2B29ABB337859
:101AD00013F0030F2FD104F093F9002800F0C48015
:101AE00004F070F9002800F0BF800AF0D9F807462A
:101AF000002840F0B9805E4B93F8292093F82A1013
:101B000042EA012193F82B2041EA0241024661F3A7
:101B10001702D3F82100D3F82510082304F032F976
:101B200098F8003067F3041367F38203DBB243F0E5
:101B3000200388F800304F4801F0CAF901F04AFA52
:101B4000002866D14C4B9B7803F01003DBB21BB925
:101B5000337813F0030F0BD0484B5B7803F0080386
:101B6000DBB2002B55D1337803F00303012B50D1A6
:101B700001F048FA002846D098F800303B4D03F0B9
:101B80002003DBB2002B35D1337803F00303012BA4
:101B900030D104F035F9002866D004F013F900289C
:101BA00062D00AF07DF8064600285DD1334B5B78A1
:101BB00003F00203DBB2EBB12D4B93F8292093F82D
:101BC0002A1042EA012193F82B2041EA0241024601
:101BD00061F31702D3F82100D3F82510102304F085
:101BE000D1F82B7866F3041366F38203DBB243F07B
:101BF00020032B70224B1878F0F7BCFD002833D05F
